:100000005446495312660115000008000000000024
:10001000000000800100000059529D1700001000F0
:10002000FF00000000000000400000000000000091
:1000300000000000010000000000000000000000BF
:10004000544643530000100000D50100CA54F63E48
:10005000000001200101100007011000090110003B
:100060000B0110000D0110000F0110001F01100006
:100070001F0110001F0110001F01100011011000CE
:10008000130110001F0110001501100003381000AB
:100090000F3910001901100019011000D599110035
:1000A00019011000831310008913100019011000AA
:1000B000190110006B341000190110008F1310008B
:1000C000273A1000F9021000ED1F1000190110006E
:1000D0000000000000000000000000000000000020
:1000E0000000000000000000000000000000000010
:1000F0000000000000000000000000000000000000
:1001000000000000000000000000000000000000EF
:1001100000000000000000000000000000000000DF
:1001200000000000000000000000000000000000CF
:1001300000000000000000000000000000000000BF
:1001400000000000000000000000000000000000AF
:1001500000F010F8FEE7FEE7FEE7FEE7FEE7FEE749
:10016000FEE7FEE7FEE7FEE701480047FEE7FEE7A1
:100170001F01100000F002F800F04AF80AA090E811
:10018000000C82448344AAF10107DA4501D100F052
:100190003FF8AFF2090EBAE80F0013F0010F18BFD5
:1001A000FB1A43F001031847B8B30100D8B30100AC
:1001B0000A4410F8014B14F00F0508BF10F8015B5A
:1001C000240908BF10F8014B6D1E05D010F8013B43
:1001D0006D1E01F8013BF9D1641E03D0641E01F8C5
:1001E000015BFBD19142E4D370470000002300245F
:1001F00000250026103A28BF78C1FBD8520728BF37
:1002000030C148BF0B6070471FB51FBD10B510BD92
:10021000DFF80CD0FFF7F8FF04F0DBFB19F0EEFB82
:100220000000012003B4FFF7F1FF03BC19F0EEFB5F
:1002300000210028D8BF704700BF491C8842FBDC62
:100240007047704770477047704770477047017834
:10025000002908BF704710F8011F0029FBD1704723
:1002600082B0010F8DF80010C0F303618DF801100A
:10027000C0F303518DF80210C0F303418DF8031051
:10028000C0F303318DF80410C0F303218DF805107D
:10029000C0F303118DF8061000F00F008DF8070071
:1002A00000206A46115C0A2934BF303137311154BD
:1002B000401CC0B2082828BF0020F3D3401CC0B2A5
:1002C0000828FBD302B0704782B001098DF80010F6
:1002D00000F00F008DF8010000206A46115C0A2929
:1002E00034BF303137311154401CC0B2022828BF0E
:1002F0000020F3D3401CC0B20228FBD302B07047E9
:1003000082B0010B8DF80010C0F303218DF80110AD
:10031000C0F303118DF8021000F00F008DF80300F8
:1003200000206A46115C0A2934BF3031373111543C
:10033000401CC0B2042828BF0020F3D3401CC0B228
:100340000428FBD302B0704712484FF6FF710160DA
:1003500070471048104A0021016012681020506157
:100360000E48012203685A6003684022DA6003687D
:100370004FF40C621A6102685161026840F6FF7125
:1003800011620068EA21016305A010F8011F00292D
:10039000FBD170470070002088AE1100B8AE11008C
:1003A00055415254204F50454E21210D0D00000063
:1003B0000B0ACAB2FA49D1F800C0CCF81C0043F4C9
:1003C000FE400B6858610868006840F00103086847
:1003D00003600868C06810F0010FFAD008688068F0
:1003E0000B6840F00100986002F07F024FF400407B
:1003F00040EA022208684261086800680B6840F021
:10040000010018600868C06810F0010FFAD0086891
:1004100080680B6840F001009860086842610868D5
:1004200000680A6840F0010010600868C06810F0B9
:10043000010FFAD0086880680A6840F001009060F7
:1004400008688069C0B2704700F07F0041EA00216F
:10045000D3480268516101680968026841F00101EE
:1004600011600168C96811F0010FFAD0016889684C
:10047000006841F001018160704700F07F014FF496
:10048000004040EA0122C64801684A6101680968E3
:10049000036841F0010119600168C96811F0010F9A
:1004A000FAD001688968036841F001019960016828
:1004B0004A6101680968026841F001011160016840
:1004C000C96811F0010FFAD001688968026841F02B
:1004D0000101916000688069C0B2704710B58C4618
:1004E0000446FFF7CAFF20EA0C01E0B2BDE8104065
:1004F000AAE7704770B5AA48002401210268C2F833
:10050000141302686FF0FE21C2F8201302689921CB
:10051000C2F8301300680321C161A248A24DA34E66
:1005200000684FF0010390F8800190B935F823007E
:10053000C0F307217F20FFF787FFF01890F8C0165F
:1005400015F82300FFF780FF5B1CB3F5A67FEDDBFA
:1005500070BD35F82300C0F3072C644505D0644610
:100560000CF00F017F20FFF76FFFF01890F8C01616
:1005700015F82300FFF768FF5B1CB3F5A67FE8DBE7
:1005800070BD10B504F02CFA854B84464FF0043052
:100590001968086219680014486219680120086126
:1005A000196888601968486000217F20FFF74CFFB8
:1005B00040210120FFF748FFBCF1050F18BF10BD17
:1005C00000201968C1F8100310BD754A00B5126803
:1005D0000321D16100284FF000014FF07F000AD0C5
:1005E000FFF732FF03210020FFF72EFF002108460E
:1005F0005DF804EB28E7FFF727FF012100205DF8F5
:1006000004EB21E7664A00B512680321D161002896
:100610004FF000014FF07F0006D0FFF715FF0121DA
:1006200000205DF804EB0FE7FFF70EFF0321002029
:10063000FFF70AFF002108465DF804EB04E758497C
:1006400000B509680320C86100217F20FFF7FCFE88
:1006500000205DF804EB10E7514900B5096803205C
:10066000C86100217F20FFF7EFFE082102205DF81E
:1006700004EBE9E64A490A68926C0123096803FA27
:1006800000F0104388647047704745490968896DD8
:1006900080F001000122801C02FA00F0084070473F
:1006A0003F480168496C026841F400615164016887
:1006B000496C006821F4006141647047384A0123A5
:1006C00003FA00F000291168096C03D0084311688F
:1006D0000864704721EA00001168086470473049D7
:1006E00000280868C06D0AD00A6840F00200D06592
:1006F0000868C06D096840F01000C86570470A6856
:1007000040F00100D0650868C06D096840F008003D
:10071000C86570472DE9F043DFF8849080462025B6
:10072000D9F8001009270220C861002404217F2085
:10073000FFF78AFEA44611E0BCF1030F03D0BCF121
:10074000060F0BD105E005217F20FFF77DFE002479
:1007500004E006217F20FFF777FE00240023002D10
:1007600088BF08EB4C1608D9F15C2046FFF76CFEF9
:10077000601C5B1CC4B29D42F6D80CF1010C6745AD
:10078000DAD8D9F800100120C861002404217F20A4
:10079000FFF75AFEA446002F1CD8BDE8F0830000E6
:1007A0008CAE1100F806002000000020B059002097
:1007B000BCF1030F03D0BCF1060F0BD105E00521FE
:1007C0007F20FFF741FE002404E006217F20FFF791
:1007D0003BFE00240023002D88BF08EB4C160AD9ED
:1007E000F01890F820112046FFF72EFE601C5B1CCD
:1007F000C4B29D42F4D80CF1010C6745D8D8CCE7BF
:1008000070B5CA49044603200968C8610425E9B2E5
:100810007F20FFF719FE0023E1B2D8B2FFF714FEE4
:1008200003F12000E1B2C0B2FFF70EFE03F1400079
:10083000E1B2C0B2FFF708FE5B1C202BECDB0CF032
:1008400062FC002808BF00246D1C072DDFDB70BD93
:10085000B64803210268D16102681121C2F8301341
:1008600000684FF00111C0F8201300217F20EBE554
:1008700070B50546002404F0B3F8022804D004F053
:10088000AFF8052804D007E00CF03DFC18B921E0D2
:1008900009F053FCF0B1A64C04F0A2F8A34B844637
:1008A0004FF004301968086219680014486219682A
:1008B00001200861196888601968486000217F205C
:1008C000FFF7C2FD40210120FFF7BEFDBCF1050F7F
:1008D00006D101E0974CDFE719680020C1F810034A
:1008E00019680320C861DFF850C201233CF82300D7
:1008F000C0F307217F20FFF7A7FDE95C1CF8230068
:10090000FFF7A2FD1CB1E118E85C81F8C0065B1C92
:10091000B3F5A67FEADB70BD844B00B519680320F0
:10092000C86100217F20FFF78FFD00210120FFF724
:100930008BFD00210320FFF787FD01217F20FFF7BA
:1009400083FD0A210E20FFF77FFD02217F20FFF7A4
:100950007BFD35210220FFF777FD78210720FFF787
:1009600073FD8B210420FFF76FFD0F217F20FFF720
:100970006BFD01210320FFF767FD19680120C1F815
:10098000140319681120C1F8300319684FF00110E1
:10099000C1F8200303217F20FFF756FD012100202D
:1009A000FFF752FD00210120FFF74EFD2121052018
:1009B000FFF74AFD04216D20FFF746FD08216E2058
:1009C000FFF742FD10216F20FFF73EFD01217F2040
:1009D000FFF73AFD08210020FFF736FD0421012032
:1009E000FFF732FD1868406C196840F400604864F5
:1009F0001868406C196820F40060486400BD4B49D9
:100A000000B509680320C86100217F20FFF71CFDA5
:100A100000210120FFF718FD01217F20FFF714FDC1
:100A200021210E20FFF710FD00212420FFF70CFDEF
:100A300000213420FFF708FD00213A20FFF704FDD4
:100A400000214420FFF700FD00214A20FFF7FCFCB5
:100A500000215420FFF7F8FC00215A20FFF7F4FC96
:100A600000216420FFF7F0FC00216A20FFF7ECFC76
:100A700002217F20FFF7E8FC55210220FFF7E4FC6C
:100A800029210320FFF7E0FC07210820FFF7DCFC09
:100A900020211620FFF7D8FC03217F20FFF7D4FC8C
:100AA000092103205DF804EBCEE47047234B0021BD
:100AB0001A46E0FB03214809C0EB00108000704794
:100AC00000207047002070470020704700207047CA
:100AD00008467047002070477047002070477047F5
:100AE0007047002070477047704700207047002013
:100AF0007047002070470020704770477047002003
:100B0000704770477047704700207047002070475B
:100B1000704770477047002070470020704770474B
:100B20000020704770477047704770478CAE1100C7
:100B3000B059002078080020000000205BB0055B61
:100B4000FC4910B509680320C86100217F20FFF728
:100B50007BFC02210020FFF777FC01210220FFF738
:100B600073FC0121BDE810400020FFF76DBCF14986
:100B700010B509680320C86100217F20FFF764FCDD
:100B800002210020FFF760FC01210220FFF75CFC3E
:100B90000121BDE810400020FFF756BCE64808B52B
:100BA00001684969C1F30721009101684969009A08
:100BB000C1F307219142F8D0DE480168D1F82C1327
:100BC000006841F00401C0F82C13FFF738FD00283D
:100BD00008BF08BD0020BDE80840FFF713BDD64898
:100BE00008B501684969C1F30721009101684969A5
:100BF000009AC1F307219142F8D0CE480168D1F89C
:100C00002C13006841F00401C0F82C13FFF717FD06
:100C1000002808BF08BD0020BDE80840FFF7F2BC6F
:100C200010B503F0DDFE052809D0C2480068D0F8F1
:100C30002C0310F0040F0CBF0120002010BDBF4892
:100C40000068006810BD70B50546FFF7E9FF012890
:100C500018BF70BD03F0C4FEB64C0326052827D08C
:100C6000FFF7BDFF012D18BF70BD2068406C2168E3
:100C700040F40060486400BF00BF00BF2068406CC3
:100C8000216820F4006048642068C66100217F204C
:100C9000FFF7DAFB02210020FFF7D6FB012102203B
:100CA000FFF7D2FBBDE8704001210020FFF7CCBB6D
:100CB0000020FFF7A7FCD8E710B5FFF762FC012082
:100CC000FFF7C1FF102004F0F4F90121052002F024
:100CD000EEFA0121062002F0EAFA99490120887013
:100CE00010BD10B5602002F038FB602002F028FB38
:100CF000904903200968C86410BD914A01465079A3
:100D0000002818BF0120002918BF01215171704728
:100D10008B4A1169106108467047894800210171AA
:100D2000C1700189874818F0CBBD85480021017149
:100D3000C1700189834818F0C3BD7E490028086846
:100D4000406C20F4407002BF0968486470470A682C
:100D500050640868426C7C480068037EC3F300134B
:100D600042EA43220B685A640A68526C007E0968A2
:100D7000C0F3C00042EA00204864704700B583B069
:100D800000208DF80000ADF8040003F029FE844631
:100D90000120FFF7D2FFBCF1020F1CBF03B000BD62
:100DA0000CF0B1F902281CBF03B000BD012061495D
:100DB0000968C86103217F20FFF746FB89210520D0
:100DC000FFF742FB67210620FFF73EFB4521072086
:100DD000FFF73AFB23210820FFF736FB03B0F12190
:100DE00009205DF804EBFFF72FBB2DE9F14F86B02A
:100DF000002004460190009003F0F2FD022806D086
:100E000003F0EEFD052808BF09F097F901E00CF0AA
:100E10007AF903F0E5FD4D49052804BF086802286A
:100E200005D0086820B1012818BF022800D101248C
:100E3000474848494FF0200800680969406BFF3176
:100E400000F5E03021F0FF01503004FB01051220D5
:100E50000026049001E0032E01D214271AE0F01EB0
:100E6000032838BF152715D3B01F032838BF16270E
:100E700010D3A6F10900032838BF24270AD3A6F10E
:100E80000C00032838BF252704D3A6F10F00032840
:100E900038BF26270198B84209D02648019739095A
:100EA0000068C16107F00F017F20FFF7CDFA0CF059
:100EB0002AF90024B8F1000F34D9380903902648E4
:100EC000A0FB06104008A0EB800000EB06092348B9
:100ED000A0FB06104008404200EBC00081190698B4
:100EE00000EB41100290069800EB461A0398012887
:100EF00036D0C4F11F0000EB49101FFA80FB01221D
:100F00006946284601F06EF96D1C03F069FD05285D
:100F100047D050E0202C45F10005E7D3601CC4B257
:100F20004445F7D3701CC6B20498864293D307B0E9
:100F3000BDE8F08F8CAE1100A8AE110090AE11008C
:100F40003005002064110020F8060020C8050020AC
:100F5000B4060020B8060020ABAAAAAA398EE3384E
:100F600004EB49101FFA80FB01226946284601F074
:100F700039F96D1C03F034FD0528009809D119F0EA
:100F80009DF94FF03332F74B19F0E8F919F052F9A7
:100F90000090C1B20AF804100BF0FF00FFF754FAFA
:100FA000BCE7009819F08AF9EF4AF04B19F0D6F92E
:100FB00019F040F90090029800992044C9B280F8D5
:100FC00020110BF0FF00FFF73FFAA7E7E849C860E0
:100FD000704710B503F004FD052802D0BDE81040AD
:100FE000FDE5FFF71DFE012818BF10BD0020BDE87C
:100FF0001040FFF707BB70472DE9F04F064683B05E
:101000000C460120FFF71FFE03F0EAFCD94D07460E
:101010004FF001084FF00009002C5CD003F0E0FC19
:10102000052810D0FFF7DBFD606800281CBF206892
:10103000002850D06FF0FE2A4FF0990B052F0AD0F0
:10104000022F22D038E0FFF7EBFD012804BF00207B
:10105000FFF7D8FAE8E709F070F80746D4E900107E
:10106000FFF706FC2868C0F81483022F04D0002F75
:1010700008BFFFF751FC1FE02868C0F820A32868CC
:10108000C0F830B3FFF7BBFC16E00CF03CF80746A5
:10109000D4E90010FFF7ECFB2868C0F81483022F96
:1010A00004D0002F08BFFFF7D3FB05E02868C0F885
:1010B00020A32868C0F830B32868C0F82893AC484B
:1010C000C6600CF020F8022802D00BF0ABFE10B97D
:1010D000A068FFF78AFE8DF80090ADF8049003F049
:1010E0007FFC84460120FFF728FEBCF1020F1ED1D1
:1010F0000CF009F802281AD12868C0F81C800321D6
:101100007F20FFF7A1F989210520FFF79DF96721CD
:101110000620FFF799F945210720FFF795F92321CC
:101120000820FFF791F9F1210920FFF78DF9904C84
:1011300084F8049084F8039021898F4818F0C0FB4C
:10114000C4F81090607900206071602002F005F909
:10115000602002F0F5F829680320C86403B0BDE8F8
:10116000F08F602002F0F0B810B5602002F0ECF8CB
:10117000BDE81040012066E57D48C06870477C48A6
:101180000078002818BF0120704738B5002400946B
:10119000FFF746FD002818BF38BD75480471C470BC
:1011A0000189754818F08CFBDFF8C8C1DCF8000035
:1011B000406CDCF8001040F40060486400BFDCF8CC
:1011C0000000406CDCF8001020F4006048646B4DB7
:1011D0006B48297800290168496914BFC9B2C1F375
:1011E0000721009120D001684969009AC9B2914253
:1011F000F9D000680221C161DCF80000D0F82C03AE
:10120000DCF8001020F00400C1F82C03DCF800002A
:10121000C0F81043FFF713FA002818BF38BD0120AB
:10122000BDE83840FFF7EEB901684969009AC1F39B
:1012300007219142F8D0002301684969C9B20091A1
:1012400001684969009AC9B29142F9D0591CCBB2E0
:10125000042BF1D301212970CBE770B503F0C0FB5B
:101260000025434C052803D02570BDE870408CE76D
:10127000FFF7D6FC002818BF70BD2571E5702189E5
:101280003D4818F01DFB25703A480168D1F82C1331
:10129000006821F00401C0F82C13BDE87040012063
:1012A000FFF7B0B9324901200870704770B503F0FC
:1012B00097FB2F4C0125052808D0FFF7B1FC00282B
:1012C00018BF70BD2570BDE870405EE7FFF7A8FC51
:1012D000002818BF70BD00202071E07021892648C9
:1012E00018F0EEFA2570BDE870400120FFF78AB9CA
:1012F0000120A8E470B51E4C0025E57003F070FBDA
:10130000052803D02570BDE870403EE7FFF788FC54
:10131000002818BF70BD2571E5702189164818F0A6
:10132000CFFA257013480168D1F82C13006821F01A
:101330000401C0F82C13BDE870400120FFF762B92A
:101340000B4A5169506108467047094880697047E7
:1013500007498861704706488069704704484078AB
:10136000704700003333FB3FCDCCCCCCCCCCFC3F22
:10137000300500208CAE110064110020AA05002069
:10138000A8AE1100FB4948707047012888BF70471C
:10139000F94900280868406E04D0096840F002004E
:1013A00048667047096840F00100486670470128A8
:1013B00088BF7047F04900280868406E04D009686B
:1013C00020F0020048667047096820F00100486676
:1013D0007047002000F0DABB012000F0D7BB10B549
:1013E000E44CE069401CE061E4480168096D006874
:1013F00041F004010165FFF753F9FFF72DF920785B
:1014000000281CBF0120FFF71EFC6069002818BFE0
:101410008047DB48016841F40061016010BD10B5F0
:101420000120FFF710FCBDE8104000F0FCBBD548E0
:101430007047D5487047CF48006A7047CD48406A2A
:101440007047CC48806A7047CA49002008624862E9
:1014500088627047CD4900EBC00001EBC0107047B7
:1014600048434FF6FF7101EA4000C24908817047C6
:10147000C74A107051707047C549085C7047F0B595
:101480000746A1B0202401210220FFF717F9C14D22
:1014900000216E46286830F8110026F81100491C1A
:1014A000A142F7D300210220FFF708F90121002013
:1014B000FFF704F90021002C09D9286806EB410246
:1014C00030F81100491CA2F840008C42F5D80021E8
:1014D0000846FFF7F3F8A2006946384618F04FF9BE
:1014E00021B0F0BD70B50E46A2490500E0B04FF046
:1014F000800008814FF020044FF001010CBF05204F
:101500000420FFF7DBF8A34900206B46096801EBD4
:10151000053101EB800202F58052D2F800C043F899
:1015200020C003EB800CD2F88020401CCCF8802037
:10153000A042EED3002D4FF0000114BF042005207F
:10154000FFF7BCF8E2006946304618F018F960B0C1
:1015500070BD70B5040087480E464FF00101058943
:101560000CBF05200420FFF7A9F88A482A46006826
:1015700000EB043000F58051304618F000F94FF0D0
:10158000000124B1BDE870400420FFF797B8BDE822
:1015900070400520FFF792B810B590B020220021CE
:1015A0000091019102910391049105910691079197
:1015B000089109910A910B910C910D910E91EC46B5
:1015C0000F9100EB410430F81130B4F8404223444D
:1015D0002CF81130491CC9B29142F2D35200614635
:1015E00018F0CDF810B010BDF0B5624F694EADF2F5
:1015F000844D00243D89002C4FF001010CBF0520D3
:101600000420FFF75BF830682A4600EB043000F551
:101610008051684618F0F8F8002C4FF000010CBF1C
:1016200005200420FFF74AF8641C022CE2DB0020AE
:10163000FFF7BDFE0120FFF7BAFE0DF2844DF0BDAD
:101640004E4A55490020136803EB8003D3F8C0309D
:1016500021F81030401C0728F5D31068D0F8E400BA
:1016600048827047454A4D4B002818BF00201DD0C6
:10167000116801EB8001D1F880110904090C18BF31
:1016800023F81010401C2028F2D30020116801EB31
:101690008001D1F880120904090C1CBF03EB400C37
:1016A000ACF84010401C2028F0D37047116801EBC3
:1016B0008001D1F800110904090C18BF23F810109B
:1016C000401C2028F2D30020116801EB8001D1F8E2
:1016D00000120904090C1CBF03EB400CACF84010CD
:1016E000401C2028F0D370472DE9F8430446002021
:1016F000009003F075F91F4E204F274D4FF0010861
:10170000052809D00BF0FFFC0028204648D0FEF742
:10171000BCFF00285ED066E02046FEF7B6FF40B969
:1017200084F001042046FEF7B0FF002808BFBDE8A2
:10173000F88316492046FFF70CFF0021386800EBBC
:101740008100D0F8C00025F81100491C0729F5D305
:101750003868D0F8E40068822046FFF783FF20460F
:10176000FFF725FE86F8048084F00100F070BDE8E4
:10177000F88300003005002088AE11008CAE110007
:101780006405002038110020411100206411002060
:1017900036050020B0AE110064160020E4150020CC
:1017A000FEF773FF40B984F001042046FEF76DFF99
:1017B000002808BFBDE8F883FE492046FFF7C9FEB0
:1017C0002046FFF7F4FD86F8048084F00100F070F5
:1017D000BDE8F88384F001042046FEF756FF002898
:1017E00008BFBDE8F883F3492046FFF7B2FE0021A9
:1017F000386800EB8100D0F8C00025F81100491CC2
:101800000729F5D3A4E770B5EB4D044668790028A5
:1018100004BFE878FFF768FF2879002808BF70BD8B
:10182000E44AAB6902F5A060A0F18001A06100204C
:10183000C4E9021020616061C4E90032012070BD7A
:10184000DD490020087170472DE9F14F82B000207A
:10185000009012204FF020080025019001E0032D98
:1018600001D214261AE0E81E032838BF152615D326
:10187000A81F032838BF162610D3A5F10900032896
:1018800038BF24260AD3A5F10C00032838BF25262B
:1018900004D3A5F10F00032838BF26260098B042D4
:1018A00009D0C648009631090068C16106F00F01F1
:1018B0007F20FEF7C9FD0024B8F1000F28D9029857
:1018C0004FEA161B00EB451ABD48A0FB0510400867
:1018D000A0EB80004719BB48A0FB05104008404220
:1018E00000EBC0000299284401EB4019BBF1010F45
:1018F00016D0C4F11F0000EB471080B2FEF7BDFD0B
:1019000009EB040181F82001601CC4B24445EDD309
:10191000681CC5B201988542A1D303B0BDE8F08F21
:1019200004EB471080B2FEF7A8FD0AF80400EBE7CD
:10193000012070477047002070472DE970431C4616
:1019400016460D468046FFF76BF95FEA00091CBF9B
:101950000120FFF778F92819A84288BF01210FD983
:1019600000234446B34238BF202C06D201FA04F2C9
:101970003A4218BF5B1C641CF4E76D1C8542EFD330
:10198000B9F1000F08BFBDE87083BDE87043B1E452
:101990002DE9F047994614460E460746089DFFF785
:1019A0003FF95FEA00081CBF0120FFF74CF903F084
:1019B00079F9DFF814C206EB0903B342CCF8000052
:1019C00088BF381913D93C460AE0DCF800100978C2
:1019D00025F8021BDCF80010491C641CCCF8001030
:1019E000844238BF202CF0D3761C9E42EBD3B8F152
:1019F000000F08BFBDE8F087BDE8F0477AE4704704
:101A000010B5FFF76AF86C49488110BD6A4AC1B247
:101A100000F470635289914288BF11464FF0640C04
:101A200001FB0CF1B1FBF2F11A0A02FB0C1189B2B5
:101A300010F4805F12BF08B2484200B2704700281D
:101A4000B8BF404280B2B4BF00214FF4805100F4CF
:101A500070621143584AC0B25289504341EA102083
:101A6000704708B50921732000F046F9BDF8001051
:101A700000F01F0021F0FF010843ADF800000D2128
:101A8000732000F039F9BDF8001000F01F0021F4B8
:101A90007F4141EA0020ADF80000BDF8000008BD1C
:101AA0007047FFF730B849484FF41071006800F5EF
:101AB000405017F005BF2DE9F84F12204FF02008D5
:101AC00000900BF020FBDFF800B102280CBF40486B
:101AD000404800F590600024CBF8000001E0032CA2
:101AE00001DA14261AE0E01E032838BF152615D3A4
:101AF000A01F032838BF162610D3A4F1090003281D
:101B000038BF24260AD3A4F10C00032838BF2526A9
:101B100004D3A4F10F00032838BF2626B24509D00C
:101B200026483109B2460068C16106F00F017F20E6
:101B3000FEF78AFC0025B8F1000F1EDD26484FEAAB
:101B4000161980FB0410A0EBE070A0EB80000719D1
:101B5000B9F1010F0EBF05EB4710C5F11F0000EBF7
:101B60004710DBF80020C0B212F8011BCBF80020B0
:101B7000FEF76AFC6D1C4545EADB0098641C844254
:101B8000ADDBBDE8F88F0020FEF79CBF70B50446C2
:101B900001280AD81148002C0168496E14BF41F091
:101BA000020141F0010100684166034DA869401C33
:101BB000A86115E064110020300500208CAE1100F2
:101BC000ABAAAAAA398EE338DC050020B0AE11001A
:101BD000B0590020780800205655555588AE1100A0
:101BE000296900291CBF20468847287800281CBF87
:101BF0000120FFF728F80648002C0CBF0221012124
:101C0000006801650348016841F02001016070BD72
:101C10008CAE1100640500200549002814BF002087
:101C20000120087070477047704770477047000088
:101C30005C050020704770B501F081FE2A4D2B4AEB
:101C40002B4B2C494FF0000C4C682CB1C1F804C050
:101C500001F07AFE204670BD287888B90888B0F572
:101C60007A7F9CBF401C0880EED930BF107838B115
:101C7000186800681C6820F00100206082F800C02D
:101C8000A1F800C0E0E710B501F059FE194844681A
:101C9000002C08BF30BFFAD00021416001F054FE93
:101CA000204610BD70B501F04AFE124D6C682CB193
:101CB0000020686001F048FE204670BD30BF01F092
:101CC00071FB0028F2D001F071FBA860EEE7002064
:101CD000704730BF704772B662B670477047704742
:101CE00072B662B67047000030060020420700203E
:101CF00090AE110060050020F84BC2081B681A6402
:101D000001F0FC0141EA002040F4704040F08040C6
:101D100000687047F14BC2081B681A6401F0FC02AE
:101D200042EA002040F4704040F08040890700689B
:101D3000C90EC840C0B27047E94900200870E749A1
:101D40000E2009680864E748007810F0800018BF8A
:101D50000120704710B44FEAD00CE04B1C68C4F867
:101D600040C001F0FC0141EA002040F4704040F026
:101D7000804002601868006C10F4007F04BF10BC43
:101D8000704700BF1868006C10F4007FF9D110BCD8
:101D90007047DFF848C310B4DCF800C0C308CCF8C3
:101DA000403001F0FC0343EA002343F4704343F066
:101DB0008043FF24D3F800C08B07DB0E9C402CEA45
:101DC000040C9A4010BC42EA0C02C3E7C6484FF428
:101DD000F4610268116101684968026841F002011A
:101DE00051600068032181617047BF4810B50268E7
:101DF0000021116002684FF4F461116101684968C3
:101E0000026841F0020151600068032181610722EC
:101E100008217120FFF7BDFF0E2001F084FA002198
:101E20000E2001F044FABDE810400E2001F063BA24
:101E3000AA4910B50968AD4808620722012170203F
:101E4000FFF7A7FFA84800210268116002684FF45D
:101E5000F461116101684968026841F00201516052
:101E6000006803218161072208217120FFF791FF9B
:101E70000E2001F058FA00210E2001F018FABDE8FA
:101E800010400E2001F037BA974800210268116017
:101E900002684FF4E06111610068012181617047BF
:101EA000914900200A6810600A6810610968886119
:101EB00070478D4806210268116002680221516056
:101EC00000688161704788480021026811600068DD
:101ED000816170478449002009680860704710B527
:101EE000814C08202168086021680220886107224F
:101EF00008217120FFF74DFF2068C06810F0080F1F
:101F0000FAD021680F20886010BD10B50446024643
:101F10000021F020FFF71EFF22460121F020FFF7ED
:101F200019FF22460021F120FFF714FF224601216C
:101F3000F120FFF70FFF22460021FC20FFF70AFFE8
:101F400022460121BDE81040FC2003E74FF48071D8
:101F500041EAD00261490B681A64654A42EA0022EC
:101F600010600868006C10F4007F08BF704700BF65
:101F70000868006C10F4007FF9D17047574A4FF49D
:101F8000807141EAD00112681164594941EA002088
:101F900000687047082270200021FAE600227020B5
:101FA0001146F6E64D480168496E026821F4007159
:101FB00051660168496E026841F48071516601689A
:101FC000496E026841F4806151660168496E00689B
:101FD00021F480614166002270201146D9E63F4815
:101FE0000168496E026841F4806151660168496E7A
:101FF000026821F4806151660168496E026821F42B
:10200000807151660168496E006841F40071416653
:10201000704732480168496E026841F48061516638
:102020000168496E006821F48061416670472B4861
:102030001B21026811640068016470472DE9F041BA
:10204000294C2068C1682B4801602068C0684FF0A7
:10205000000610F0100F0BD020481B2102681164FD
:102060000068016420688068216840F01000886082
:102070002068C06810F0080F05D0206880682168CB
:1020800040F0080088602068C06810F0040F0AD093
:102090002068806840F0040120688160FF220021F0
:1020A0007020FFF776FE2068C06810F0020F4BD05A
:1020B00020688068216840F0020088600E4D287812
:1020C000F0B316F0BFF90327DFF83080012817D0EE
:1020D00016F0B8F902281FD029E0000088AE1100E0
:1020E0006C05002000F20040A8AE11002222A26080
:1020F00000F00040FC060020430700208CAE1100D9
:10210000D8F80000C76100217F20FEF79DF900216B
:102110000320FEF799F90AE0D8F80000C761002112
:102120007F20FEF791F901210320FEF78DF9206849
:102130000068216820F0020008604FF4F46000E0BD
:1021400002E0216808612E702068C06810F0010F5D
:1021500008BFBDE8F08120688068216840F0010078
:102160008860BDE8F0810000704770B5FF4D0446FF
:10217000C0F30741286801F0D0FAC4F307212868AA
:1021800001F0CBFAE1B22868BDE8704001F0C5BAB1
:102190002DE9F041F64F0446164638680D46806A30
:1021A000396840F003008862DFF8C0830321D8F863
:1021B000000001F0B2FA2046FFF7D7FF0024002EFE
:1021C00007D9D8F8000001F0D6FA2855641CA642B9
:1021D000F7D83868806A396820F0030088620120E7
:1021E000BDE8F08170B514460D46064601F0B1FB1E
:1021F000224629463046BDE87040C9E72DE9F04146
:102200000024DC4D042601F0A4FB3246294620467A
:10221000FFF7BEFF04242F463D1D264601F099FB23
:10222000324629462046FFF7B3FF08242D1D042619
:1022300001F08FFB324629462046FFF7A9FF2025F3
:1022400007F10C0401F085FB324621462846FFF7D2
:102250009FFF0C3724243E1D042501F07AFB2A46FB
:1022600031462046FFF794FF2824361D01F071FB0C
:102270002A4631462046FFF78BFFBF4E07F10C047C
:1022800001F067FB2A4621463046FFF781FF371DE4
:1022900025462C1D042601F05CFB324621463846BB
:1022A000FFF776FF3E1D0424083501F052FB22465D
:1022B00029463046FFF76CFF4FF4FC342D1D0426F1
:1022C00001F047FB324629462046FFF761FF271DF4
:1022D0002C46251D01F03DFB324629463846FFF7C6
:1022E00057FFA64F2D1D01F034FB324629463846D4
:1022F000FFF74EFF3F1D2D1D01F02BFB32462946F7
:102300003846FFF745FF2E1D3F1D042501F021FB38
:102310002A4631463846FFF73BFF351D3F1D042650
:1023200001F017FB324629463846FFF731FF3E1DC4
:102330000425183401F00DFB2A4621463046FFF7EC
:1023400027FF8F4E8F4C012501F003FB2A462146C3
:102350003046BDE8F0411BE77047F8B50E00054672
:102360004FF0000417D0042269462846FFF710FFFB
:102370009DF800009DF801109DF8032008409DF88D
:10238000021011400840FF2801D00020F8BD641C55
:102390002D1DB442E7D30120F8BD2DE9F843914645
:1023A0000D468046002401F0D4FA0027B9F1000F51
:1023B00088BF6E4619D9042269464046FFF7E8FEF9
:1023C0000023F05CE95C88421CBF601C84B25B1C8B
:1023D000042BF6D32D1D7F1C08F104084F45EAD3CA
:1023E000002C1CBF0020BDE8F8830120BDE8F88365
:1023F0000120704770B55E4C06462068806A2168EF
:1024000040F003008862594D0521286801F085F9E4
:10241000286801F0B0F92168896A226821F0030177
:1024200091623070012070BD38B5514C2068806ACF
:1024300040F00301206881624C4D0521286801F0BD
:102440006CF9286801F097F92168896A226821F0FF
:10245000030191628DF8000010F0010018BF012007
:1024600038BD10B5424C2068806A216840F00300F6
:1024700088623E480621006801F04FF92068806AB2
:10248000216820F003008862012010BD70B5054668
:10249000FFF7CAFF00281CBF022070BDFFF7E1FF55
:1024A000334C2068806A216840F0030088622F481E
:1024B0002021006801F031F92846FFF756FE206818
:1024C000806A216820F003008862FFF7ADFF28B121
:1024D00000BF00BFFFF7A8FF0028F9D1012070BDA1
:1024E0002DE9F84F8046032701F033FADFF880909A
:1024F000DFF878A0FFF798FF10BBFFF7B2FFD9F81D
:102500000000806AD9F8001040F0030088622021A2
:10251000DAF8000001F001F94046FFF726FED9F88D
:102520000000806AD9F8001020F003008862FFF7ED
:102530007BFF28B100BF00BFFFF776FF0028F9D16D
:1025400045464FF480660024042269462846FFF77A
:102550001FFE9DF800009DF801109DF80320084023
:102560009DF8021011400840FF280DE0A4AE1100B4
:1025700088AE11008416002068C0010010F8010028
:10258000043003007005002006D0381EA7F10107B3
:10259000B0DC0220BDE8F88F641C2D1DB442D3D3FB
:1025A0000120BDE8F88F2DE9F04117460E4604469C
:1025B000FFF73AFF00281CBF0220BDE8F081FFF7BB
:1025C00050FFDFF80C84D8F80000806AD8F80010BB
:1025D00040F003008862FF4D0221286801F09DF859
:1025E0002046FFF7C2FD0024002F06D9315D286880
:1025F00001F093F8641CA742F8D8D8F80000806A6C
:10260000D8F8001020F003008862FFF70DFF28B112
:1026100000BF00BFFFF708FF0028F9D10120BDE887
:10262000F0812DE9F043C1B08846814603276E460C
:1026300001F08FF94FF4807241464846FFF7B3FF2F
:10264000002445464FF4807269464846FFF7A0FDD6
:10265000305D295D884205D07F1EE9D241B002205D
:10266000BDE8F083641CB4F5807FF1D341B0012054
:10267000BDE8F0832DE9F041D74C0646D44FDFF892
:1026800054836068C0B00D4650B1D8F8000001F026
:1026900044F86268FF2AB8BF501C1BDA606035E05E
:1026A00001F057F9FFF7DDFE3868806A396840F0BD
:1026B000030088620221D8F8000001F02EF83046AD
:1026C000FFF753FD2946D8F8000001F026F86068AE
:1026D000401CE3E7002060603868806A396820F0B9
:1026E0000300886200244FF4807269463046FFF789
:1026F0004FFD68462A5D015D914203D040B0022043
:10270000BDE8F081641CB4F5807FF3D340B00120B4
:10271000BDE8F08170B50C46054601F01AF9B4F534
:10272000807F88BF70BDAA490A68926A096842F032
:1027300003028A62A7480321006800F0EEFF2846E2
:10274000BDE8704011E5A348006801F014B8A04846
:102750000168896A006821F003018162704770B5E1
:102760000C46054601F0F5F821462846BDE87040C4
:102770004FF480720CE570B5954D04462868806A68
:10278000296840F003008862924E9F21306800F073
:10279000C4FF306800F0EFFF2070306800F0EBFFFE
:1027A0006070306800F0E7FFA0702868806A2968D0
:1027B00020F003008862012070BD70B5044601F06E
:1027C000C8F8834D2868806A296840F00300886251
:1027D000804E9F21306800F0A0FF306800F0CBFFF2
:1027E0002070306800F0C7FF6070306800F0C3FFF1
:1027F000A0702868806A296820F0030088620120A0
:1028000070BD2DE9F047DFF8C89104461746D9F8A6
:1028100000008846806AD9F8001040F00300886202
:102820006C4D0321286800F078FF2046FFF79DFCDF
:102830000024B4EB970F18D2286800F09CFF0646DE
:10284000286800F098FF46EA0026286800F093FF09
:1028500046EA0046286800F08EFF46EA006048F825
:102860002400641CB4EB970FE6D3D9F80000806A0B
:10287000D9F8001020F0030088620120BDE8F0873D
:1028800070B514460D46064601F063F82246294607
:102890003046BDE87040B4E710B5FFF7C5FD00282D
:1028A0001CBF022010BDFFF7DCFD494C2068806A88
:1028B000216840F00300886246486021006800F00B
:1028C0002CFF2068806A216820F003008862FFF7EF
:1028D000ABFD28B100BF00BFFFF7A6FD0028F9D16E
:1028E000012010BD10B501F034F8FFF79DFD002860
:1028F0001CBF022010BDFFF7B4FD354C2068806A74
:10290000216840F00300886232486021006800F0CE
:1029100004FF2068806A216820F003008862FFF7C6
:1029200083FD28B100BF00BFFFF77EFD0028F9D16D
:10293000012010BD70B50C46054601F00AF80026CE
:1029400001F007F84FF4807221462846FFF720FC7B
:10295000761C04F5807405F58075102EF0D30120E7
:1029600070BD2DE9F047C0B08846814600F0F1FF08
:102970004FF0000A464603276D4600F0EAFF4FF489
:10298000807231464846FFF70EFE00244FF48072F5
:1029900069464846FFF7FCFB295D305D814205D062
:1029A0007F1EEAD240B00220BDE8F087641CB4F577
:1029B000807FF1D30AF1010A08F5807809F5807962
:1029C000BAF1100FD6D340B00120BDE8F087000067
:1029D00088AE1100A4AE1100700500202DE9F04F63
:1029E00081B00546ADF5804D000514468846000DC2
:1029F000EB4633D02F466FF30B07BA465E4600F026
:102A0000A8FF4FF0000900F0A4FF4FF48072314698
:102A10003846FFF7BDFB09F1010906F5807607F599
:102A20008077B9F1100FEED3C5F30B00C0F58056D7
:102A3000A64288BF264658443246414616F09FFEBD
:102A40005046FFF74DFD022850D059465046FFF73B
:102A500088FF02284CD03544B044A41BB4F5805FF5
:102A600019D34FF480524146584616F088FE284646
:102A7000FFF736FD022839D059462846FFF771FF87
:102A8000022835D0A4F5805405F5805508F5805806
:102A9000B4F5805FE5D21CB3D9462E4600F059FF4D
:102AA000002700F056FF4FF4807259463046FFF77A
:102AB0006FFB7F1C06F580760BF5807B102FF0D323
:102AC00022464146484616F05AFE2846FFF708FDC2
:102AD00002280BD049462846FFF743FF022807D0BB
:102AE000012001B00DF5804DBDE8F08F0A20F8E718
:102AF0000B20F6E710B5ADF5806D0446AAB1684627
:102B000016F03DFE2046FFF7EBFC022802BF0A202C
:102B10000DF5806D10BD69462046FFF782FD022845
:102B200002BF0B200DF5806D10BD01200DF5806DED
:102B300010BD70B50646FFF777FC00281CBF0220C9
:102B400070BDFFF78EFCB44C2068806A216840F0AD
:102B500003008862B14D0121286800F0DEFD314696
:102B6000286800F0DAFD2068806A216820F0030000
:102B70008862FFF759FC28B100BF00BFFFF754FC83
:102B80000028F9D1012070BDF8B500F0E2FEA24D99
:102B90002868806A296840F0030088629F4E0521FA
:102BA000306800F0BAFD306800F0E5FD2968896AF8
:102BB0002A6821F00301916240F040048DF8004042
:102BC000FFF732FC002818BFF8BDFFF74AFC286861
:102BD000806A296840F0030088620121306800F0B3
:102BE0009CFD2146306800F098FD2868806A2968BD
:102BF00020F003008862FFF717FC002808BFF8BD2B
:102C000000BF00BFFFF710FC0028F9D1F8BD70B578
:102C100005460024FFF708FC40B1AC4201D9002072
:102C200070BD641CFFF700FC0028F6D1012070BDC8
:102C300070B5794C06462068806A216840F0030030
:102C40008862764D0921286800F067FD286800F049
:102C500092FD2168896A226821F003019162307037
:102C6000012070BD38B5FFF7DFFB002836D1FFF734
:102C7000F8FB694C2068806A40F00301206881629B
:102C8000664D2F21286800F048FD2068806A216881
:102C900020F003008862FFF7C7FB28B100BF00BF28
:102CA000FFF7C2FB0028F9D12068806A216840F054
:102CB000030088620921286800F02FFD286800F0D1
:102CC0005AFD2168896A226821F0030191628DF81A
:102CD000000010F0020F1CBF012038BD022038BDDB
:102CE0004E4810B50421006800F017FD012010BD0A
:102CF00070B5FFF799FB00281CBF022070BD464C41
:102D00002068806A216840F003008862434D0521F5
:102D1000286800F002FD286800F02DFD06462068B6
:102D2000806A216820F0030088622068806A216838
:102D300040F003008862FFF794FB0121286800F04F
:102D4000ECFC26F04001286800F0E7FC2068806A6F
:102D5000216820F003008862012070BD70B505462F
:102D6000FFF762FB00281CBF022070BDFFF779FB54
:102D7000294C2068806A216840F003008862274857
:102D80005221006800F0C9FC2846FFF7EEF92068E0
:102D9000806A216820F003008862FFF745FB28B1B4
:102DA00000BF00BFFFF740FB0028F9D1012070BD34
:102DB00010B50446FFF738FB00281CBF022010BDE9
:102DC000FFF74FFB1548D821006800F0A6FC20460D
:102DD000FFF7CBF910480168896A006821F0030108
:102DE0008162FFF721FB28B100BF00BFFFF71CFB8A
:102DF0000028F9D1012010BD084810B5B92100689C
:102E000000F08BFC012010BD044810B5AB21006818
:102E100000F083FC012010BD88AE1100A4AE1100AB
:102E2000012101FA00F042490A6810430860414953
:102E3000096808607047012101FA00F03C490A68FE
:102E400022EA000008603B49096808607047384979
:102E5000096821FA00F000F001007047344A116857
:102E600021FA00F313F0010F4FF0010303FA00F011
:102E7000304B05D021EA00001060196808607047E7
:102E8000084310601968086070472A490968096892
:102E900021FA00F000F00100704726490A685268E4
:102EA0000123096803FA00F0104348607047214984
:102EB0000A6852680123096803FA00F022EA000058
:102EC000486070471B490A68126A0123096803FABF
:102ED00000F010430862704716490A68126A01231D
:102EE000096803FA00F022EA0000086270471149FD
:102EF000086840680A6840F00100012350600868D3
:102F000040680A6840F002005060094A106840F0CA
:102F100001001060D1F800C0CCF80000106840F04B
:102F2000020010600968086003480068C3607047C9
:102F30007805002080AE110088AE11007047704700
:102F4000B24810B502683F21D16002680021916447
:102F50000068C0F8B41003210A2000F0A8F9BDE809
:102F600010400A2000F0C7B9A84A13681860136817
:102F700059604843116888607047A44A1368186014
:102F800013685960484310F0010F18BF401C1168C6
:102F9000886070479D490968C1F8B40070479B4933
:102FA00018B10968012088647047096800208864A6
:102FB000704796480168C968006841F00201C16025
:102FC0007047DFF848C210B4DCF800402062DCF83B
:102FD00000004162DCF800008262DCF80000C3629D
:102FE000DCF8001001200863DCF80000406B10F0F2
:102FF000010F09D000BF00BF00BF00BFDCF8000018
:10300000406B10F0010FF5D110F0020018BF4FF027
:10301000FF3010BC70477D480168C968006821F026
:103020000201C160704779480168C968006841F0D1
:103030000101C1607047754BD3F800C0CCF8200087
:10304000186841621868826219680120086418686B
:10305000406C10F0010F08D000BF00BF00BF00BFE0
:103060001868406C10F0010FF6D110F0060018BF80
:103070004FF0FF30704765480168C968006821F06B
:103080000101C160704761480168C968006841F08A
:103090000401C1607047027C017B02F03F0241EAFB
:1030A00002415A4A136899651368016859621368A6
:1030B0004168996213688168D962136801211965B2
:1030C0001168496D11F0010F08D000BF00BF00BFAB
:1030D00000BF1168496D11F0010FF6D11368DB6D67
:1030E00083821368DB6D1B0CC38213681B6E038322
:1030F00013681B6E1B0C438313685B6E838312681B
:10310000526EC2F30E42C28311F0020018BF4FF09C
:10311000FF3070473D480168C968006821F004012C
:10312000C160704701684FEA314238490B68C3F803
:103130009C200A684068C2F8A0000868C068096856
:1031400040F02000C8607047304A13681862106869
:10315000416211680120C1F890001068D0F8980011
:1031600010F0010F09D000BF00BF00BF00BF106802
:10317000D0F8980010F0010FF5D110F0060018BF3C
:103180004FF0FF30704721480168C968006821F09E
:103190002001C16070471D480168C968006841F09E
:1031A0001001C1607047A3F1050C184B10B41C68E6
:1031B000C4F888C0D3F800C0CCF820001868426278
:1031C0001868816219680120C1F880001868D0F879
:1031D000840010F0010F09D000BF00BF00BF00BF86
:1031E0001868D0F8840010F0010FF5D110F0060037
:1031F00018BF4FF0FF3010BC704704480168C96821
:10320000006821F01001C1607047000094AE110009
:10321000234810B502680121116602681021516728
:10322000026841F206015166026800219166026857
:103230000A21C2F8881002689021C2F8841001683F
:10324000D1F88410026841F00101C2F884100268CC
:103250004FF48171116600680166032000F04BF89D
:103260000021032000F023F80E490220096888623B
:10327000002010BD10B5032000F048F808484FF4B6
:1032800080710268116602680021116600681021D1
:103290008167002010BD04490020087070470000BD
:1032A00084AE110090AE11007C050020704700F044
:1032B0000303DA004FF0FF0C0CFA02F24FF0050C9A
:1032C0000CEBC303994000F00C03002808DA3048E7
:1032D00000681844436911409343194341617047A2
:1032E0002C4800681844D0F8003311409343194328
:1032F000C0F80013704700F01F01012202FA01F12B
:10330000244A4009126842F82010704700F01F015B
:10331000012202FA01F11F4A4009126802EB800003
:10332000C0F88010704700F01F01012202FA01F17D
:10333000184A4009126802EB8000C0F880117047FB
:10334000144909680860704712490968C1F880008B
:10335000704710480068006870470E490968C1F856
:10336000800170470A4800688068704708490A6809
:1033700092680968886010467047054A126892682A
:1033800000F1100352F8230042F8231070470000A8
:1033900078AE110074AE11007047704770477047E7
:1033A000704770470020704700207047002070472A
:1033B000704770471B4A1168106008467047704795
:1033C00018484068704710B500F0ACF81648042162
:1033D0000268C2F8881002684FF6FF71C2F88C10BC
:1033E00072B600684FF40071016662B610BD72B625
:1033F0000D484FF400310268116662B60068D0F8DB
:10340000040268B14FF6FF71081A0649074A88603E
:10341000A0F50840B93890423CBF4FF00110C86099
:1034200000F085B88005002098AE1100372B1A00F7
:103430001A4801684969026841F4007151610168E4
:103440000969026821F006011161016809690068D3
:1034500041F0100101617047104801680969026874
:1034600021F00601116101680969026841F0040157
:10347000116101680969006841F01001016170473C
:103480000649096888607047BFF34F8F03490448B5
:103490000968C860BFF34F8FFEE7000078AE1100E7
:1034A0000400FA05022824BF00207047874B53F818
:1034B000202043F820101046704770B5844C2068D7
:1034C000006F824D10F0010F06D021680120C86600
:1034D0002868002818BF80472068006F10F0020F8E
:1034E00008BF70BD02202168C8666868002808BF50
:1034F00070BDBDE870400047754810B502680221F4
:103500001165036801221A6603680322DA660068FF
:1035100041650920FFF7EFFE0221BDE810400920B8
:10352000FFF7C5BE6A490220096808657047684907
:1035300002200968486570470020704764480168A8
:10354000096F11F4007F04D000684FF440710166E8
:10355000704700684FF480710166704710B55C4C8D
:103560002068C06F10F0020F4FF0010018BF032059
:10357000226850670520B1FBF0F022684FF4057116
:103580000009C2F8801016F099FE524A524B16F00C
:10359000E5FE16F04FFE2168C1F884002068006F38
:1035A00010F4007F04D021684FF44070086610BD0D
:1035B00021684FF48070086610BD45480168096FA6
:1035C00011F4807F04D000684FF4407101667047A9
:1035D00000684FF40071016670473D4B30B41A68C3
:1035E000D26F12F0010F1DBF0322D3F800C0CCF838
:1035F00074204FF0020C04BF1A68C2F874C04FF078
:10360000020C00EB4005C5EBC0104FF49674C1EB03
:10361000C0004C4300EB8000304904EB4010A1FB9C
:103620000010C0080521B0FBF1F00022B0F5803F8A
:1036300005D3511C4008CAB2B0F5803FF9D242EA26
:103640000C211A6841F01001C2F888101968C1F8FD
:103650008C001868006F10F4807F05D019684FF453
:103660004070086630BC704719684FF400700866F7
:1036700030BC704716480168096F11F4003F04D050
:1036800000684FF440310166704700684FF48031A4
:10369000016670470E480168096F11F4803F04D03D
:1036A00000684FF440310166704700684FF4003104
:1036B0000166704706480068006FC0F3002070473D
:1036C00003480068006FC0F3402070479405002055
:1036D00098AE11007B14AE47E17A843FCDCCCCCCC0
:1036E00030B40025DDE9024C056001F00F0141EA2C
:1036F0008C1101600168D2B241EA0221016023F419
:103700007F41016110214160416804F004021143CE
:103710006FF3CF11416030BC7047C26812F0010FE7
:1037200018BF8160C16811F0100FFBD1C16811F0A2
:10373000040F08BF70478168C16811F0040FFAD107
:1037400070470023002A0BDD11F803C0C0F808C041
:10375000D0F80CC01CF0100FFAD15B1C9342F3DBC5
:10376000C16811F0040F08BF70478168C16811F08B
:10377000040FFAD17047FF22C16811F0100FFBD17E
:103780008260C16811F0100FFBD1C16811F0040F05
:10379000FBD08068C0B270470023002AD8BF7047B2
:1037A00010B4FF24D0F80CC01CF0100FFAD18460C4
:1037B000D0F80CC01CF0100FFAD1D0F80CC01CF0DF
:1037C000040FFAD0D0F808C001F803C05B1C9A427D
:1037D000E7DC10BC7047416841F002016FF3CF1184
:1037E00041607047416821F4C17121F47E4141601C
:1037F0007047000070470248006840687047704793
:1038000088AE11002C4900200A68906009680860A1
:103810002A494860704710B5274C216848602168E4
:10382000002088600221401EFFF741FD216807202B
:103830000860BDE8104006F087BA1F4900200968FB
:10384000086006F085BA1D49087070471B4800786B
:10385000704710B506F07CFA174900200968086027
:1038600010BD1648806870472DE9F041134C0027C1
:1038700005466780A0684FF47A71B0FBF1F00E4EF8
:10388000401E31684860306887600221C81EFFF71B
:103890000EFD31680720086006F056FA6188A942DB
:1038A000FCD330680760BDE8F04106F051BA044926
:1038B000484302498860704770AE11009C050020A3
:1038C00040420F00704770B52C4C05464FF40D5028
:1038D0002168886621680320C866216828484866F0
:1038E00021684CF27100086621682648C1F8800002
:1038F000216842F24630886602210020FFF7D7FC9B
:103900000020FFF7F8FC002D08BF70BD2068806E16
:1039100042F2413108432168886670BD174810B5EE
:1039200002680121916700684FF40D518166002003
:10393000FFF7ECFCBDE810400020FFF7F4BC0F4996
:1039400001200968486770470C49012009688867A9
:1039500070470A494CF271000968086670470748C9
:1039600081B04CF27101026811660168096F02684A
:10397000D1660068006F009001B070477CAE110006
:1039800007383937009C1C9110B500210A20FEF73A
:10399000F5FA8B49887110BD024670200121FEF7AF
:1039A000F8B9024670200021FEF7F3B92DE9F04185
:1039B0000024254672201421FEF79EF9064610F0D9
:1039C000010F18BF012416F0020F18BF44F00204C3
:1039D00016F0040F18BF44F0040416F0080F0DD0C1
:1039E000784844F008040168D1F82C13006841F0CD
:1039F0000401C0F82C130020FCF704FE16F0100F91
:103A000018BF44F0100416F0200F6D4F06D044F09C
:103A1000200400210A20FEF7B1FAB87124B1702009
:103A200001212246FEF7B5F9300A10F0010F18BF48
:103A30001025040A14F0010F4FF0010607D045F0DD
:103A400020053E7000210A20FEF798FAB871200A7E
:103A500010F0010F1CBF45F040057E7025B17020AD
:103A600000212A46FEF795F9B8799C281CBF002052
:103A7000B870BDE8F08199E710B500210A20FEF783
:103A80007DFAC0B200224E499C2804BFCA700A7059
:103A900008D0C878401CC0B2C870032882BFCA7062
:103AA000012010BD002010BD10B5454C6079401CB0
:103AB000C0B26071142818D900210A20FEF75EFAFE
:103AC000A279C0B20021824204BF217161710CD081
:103AD0006079401E60712079401CC0B220710328BB
:103AE00003D921716171012010BD002010BD10B5F6
:103AF000C9200021FEF700F9002010BD70B5742424
:103B0000002133222046FEF744F901210D462A46C2
:103B10002046FEF73EF902212A462046FEF739F9F3
:103B200003212A462046FEF734F97020012177222E
:103B3000FEF72FF90C20FFF7DEFB00210C20FFF72A
:103B4000B6FBC82000211422FEF723F91C4C0020EC
:103B50000146A0700A20FEF711FAA07170BD70B581
:103B6000FFF7A2FF20B10020FFF765F9FEF737FA53
:103B7000134C00252078B0B100210A20FEF7FEF991
:103B8000C0B29C2804BFE57025700CD0E078401CC2
:103B9000C0B2E070032806D9E57025700020FFF759
:103BA0004AF9FEF71CFA6078002808BF70BD6570FE
:103BB0000020FFF740F9BDE87040FEF710BA0000A2
:103BC000A80500208CAE110070B5FE4C00254FF406
:103BD000906125706570FC4815F072FE4FF490619D
:103BE000FA4815F06DFE4FF49061F94815F068FE43
:103BF0006560A5708021F74815F062FEBDE8704051
:103C00008021F54815F05CBEEE488078002818BF8A
:103C100001207047EB484078002818BF012070470A
:103C200070B50546ED48EE490078097800FB01F4CF
:103C3000FFF79AF9E64A2B46A2F510610846FFF70E
:103C4000C0F962002946E24815F099FDDD490120DE
:103C5000487070BD2DE9F0411D4616460F4680465E
:103C6000069C00F0BDFE022802D109F04CFA28B1F2
:103C700000F0B6FE052808BF06F05FFAFFF75EF910
:103C800021462846FFF779F93A4631464046FFF784
:103C9000D2F9BDE8F041FFF752B9CA484068704711
:103CA000D04A10B5127801469200CA4815F067FD57
:103CB000C4490120887010BD2DE9F04FDFF804934E
:103CC000002689B099F8018099F80270B346FDF793
:103CD0008BFCC5480168496C026841F4006151647D
:103CE00000BF0168496C006821F400614164BF496C
:103CF0000220096808660020FCF7FFFFFDF7ADFA17
:103D000005F06DFB01280BD06846FDF77CFD00280F
:103D1000F6D0684605F0C3FF029870B11FB10CE001
:103D20004FF0010B66E00146AE4800788200A948DA
:103D300015F025FD012089F802000198002851D0D6
:103D4000B8F1000F4ED1044699F8000090BBD9F8A5
:103D500004507DB3A14800780790A14890F800A0D6
:103D600000F03EFE022802D109F0CDF928B100F0A2
:103D700037FE052808BF06F0E0F9FFF7DFF85146E7
:103D80000798FFF7FAF821462A460846FFF753F945
:103D9000FFF7D5F8DFF858A29AF80000022804BF10
:103DA000284605F015FE9AF80000092804BF2046B1
:103DB00005F00EFE2546894889490078097800FB00
:103DC00001F4FFF7D1F8824A2B46A2F510610846AC
:103DD000FFF7F7F8620029467D4815F0D0FC012076
:103DE00089F80100FDF72CFD761C042E88D3BBF169
:103DF000000F03D089F8018089F802700120FCF7D8
:103E000022FF7A4802210068016609B05846BDE8E1
:103E1000F08F6C48002101704EE738B50F2100F09B
:103E2000AEFE684C012806D100202070FFF744FF49
:103E3000009000F027FF607800281BBFA0780028C2
:103E40000020012038BD0F2138B500F098FE5D4CF0
:103E5000012806D100202070FFF72EFF009000F00F
:103E600011FF607800281BBFA078002800200120E7
:103E700038BD0021534841708170704752487047E7
:103E80005248704770B505464FF490614E4815F0A2
:103E900017FD4FF490614E4815F012FD494C29462C
:103EA0004948227800F057FB22782946BDE8704047
:103EB000474800F050BBF0B4484A434B0021147807
:103EC0008C4603F510650022002C13D933F91160DC
:103ED00030F91170BE4253F81160B4BFB61CB61E63
:103EE00043F8116033F9116045F81160491C521C08
:103EF000A242EBD30CF1010CBCF1020FE3D3F0BCF6
:103F00007047002818BF01202E49487070472DE9DE
:103F1000F04FDFF8B0A083B05FEA000872D0002550
:103F20004FF410792C4600F05BFD052808BF0125F1
:103F300005D009F0E8F800280CBF2E4C2E4C2F4875
:103F40002F4F00687969806BFF3100F5E03021F078
:103F5000FF01503005FB010600F042FD022807D1A9
:103F600009F0D1F820B97869FF3020F0FF0006444D
:103F700000F036FDDFF864B0022803D109F0C3F881
:103F8000002856D000F02CFD052802D106F0D5F807
:103F9000B8B10025771C304601226946FEF722F9A8
:103FA0007E1C012201A93846FEF71CF90198002C5D
:103FB000C1B2009861F31F2000B2414628F81500F5
:103FC00021E036E0B0050020C8160020481B002084
:103FD000C81F0020482D0020C82D0020BA05002051
:103FE000BB050020C10500208CAE110088AE110079
:103FF0002D06002078080020B0590020B4060020CB
:10400000B806002010E018BF24F815006D1C4D45BF
:10401000C0D3FF489BF80020FC4B0078504342007F
:10402000184615F0ACFBF948CAF8040003B0BDE827
:10403000F08F4023002084466146424628F810C095
:10404000002C18BF24F81010401C9842F4D3F048FC
:1040500011469BF800200078EE4B50434200184672
:1040600015F08DFBEB48DFE710B509F04CF802289E
:10407000E94BE74AE5480AD01B781278E7495A43EA
:10408000520015F07CFBE649E048486010BD1B7803
:104090001278E4495A43520015F071FBF3E710B56A
:1040A000DF4C002804BF606010BDDFF860C3DA4950
:1040B0000B78D7490A7801465A435200604615F0FA
:1040C0005EFBD248606010BDD7487047002818BF1B
:1040D0000120D34988707047D149002200284A70D6
:1040E0008A7018BF01200870E6E510B54FF44C3017
:1040F0001422CE49FEF776F8CC4810BD10B54FF427
:104100004C301422C949FEF76DF8C848006810BD4C
:1041100010B54FF44C301422C449FEF763F8C3487D
:1041200010BD0268B2F1FF3F15D0052904BFC07A67
:10413000704728DC012904BF00797047022904BFB9
:10414000007A7047032904BF407A7047042904BFEE
:10415000807A704727E0052913D007DC012922D097
:1041600002291CBF032904290BD01CE0142912BF0B
:1041700015292D207047162904BF282070471729BC
:1041800011D100207047142904BF007B7047152906
:1041900004BF407B7047162904BF807B70471729F6
:1041A00004BFC07B7047FF20704770B5C0B00024CB
:1041B0004FF48071684615F083FBFF224FF44C36B4
:1041C000511C684615F052FBFF21254661F3070597
:1041D0002D22214662F3070162F30F2128224BF6BC
:1041E000BB3062F3174164F31F61CDE90005CDE9EF
:1041F000024104943046FEF7FBF869463046FEF76C
:1042000010FA40B070BD2DE9F04FC1B00446DDE9B1
:104210004A9887489A4693460D4601602068B0F157
:10422000FF3F08BFFFF7C1FFD4E901106BF30700A0
:104230006AF30F20266869F31740D4E9037465F325
:10424000070168F31F600D468046FF22511C684637
:1042500015F00CFBCDF80880CDE90374CDE90065BD
:104260004FF44C342046FEF73BF969462046FEF7F2
:10427000D8F9012818BF002041B0BDE8F08F2DE922
:10428000F04F174688468146C1B000244FF44C30A9
:1042900014226649FDF7A6FF644B1D68B5F1FF3F88
:1042A00002BF204641B0BDE8F08FFF22D3E902A44F
:1042B000511C6846D3F810B05E6815F0D7FA69F360
:1042C000070468F30F2467F31744012060F31F64A9
:1042D000CDE902A4CDE900564FF44C34CDF810B02E
:1042E0002046FEF7FDF869462046FEF79AF941B0F0
:1042F000BDE8F08F2DE9F04F4E4F0025C1B07E4252
:10430000A8464FF44C3014224849FDF76BFF474C48
:10431000172120462368FFF704FF84461421204616
:10432000FFF7FFFE4BF6BB3140B28B4204D1BCF12C
:10433000000F0FD12D280DD02160FF20207100200B
:1043400020726072A072E0722D21217361732821A6
:10435000A173E07314212046FFF7E3FE40B20390FF
:1043600015212046FFF7DDFE40B2029016212046BF
:10437000FFF7D7FE40B2019016212046FFF7D1FE8D
:10438000404240B20090FCF7F7FE10F0020F7CD0E4
:104390001F48294A4FF0000990F800C01E480078D5
:1043A0000028C8BFACF1010A1EDD0021BAF1000FE0
:1043B00016DD01F1010B01FB00930BFB009B32F8B2
:1043C000133032F81BB0A3EB0B031BB2002BB8BFAA
:1043D0005B421BB24345C8BF9846491C5145E8DBC8
:1043E00009F101098145E0DB02994145B8BF45F07B
:1043F00002054FF00009CA46BCF1000FC8BFA0F18A
:10440000010B34DD0021BBF1000F17E04824002030
:10441000BB050020C8280020BA050020780800202D
:10442000B0050020B0590020482D0020482E002063
:1044300070050020F1D8FFFFC816002013DD0AFB2D
:10444000001332F813E002EB43035B88AEEB030387
:104450001BB2002BB8BF5B421BB24B45C8BF99468D
:10446000491C5945EBDB0AF1010AE245CADB039915
:104470004945B8BF45F004054FF0000ABCF1000FF4
:1044800015DD002300280EDD00E018E00AFB0031F6
:1044900032F91110B942C8BF0F46B142B8BF0E463B
:1044A0005B1C8342F0DB0AF1010AE245E9DB01987B
:1044B000B84202DB0098B04201DD45F0080509F082
:1044C000FF0040907042C6B2274808F0FF08FFB2D4
:1044D00005602068B0F1FF3F08BFFFF766FED4E932
:1044E000020A4099D4E9009B61F3070068F30F20AA
:1044F00067F3174066F31F600646FF22246965F3E1
:10450000070B511C684615F0B1F9CDF80090CDE9C4
:1045100003A4CDE901B64FF44C342046FDF7E0FF8B
:1045200069462046FEF77DF81D208DF800004120E9
:104530008DF8010000208DF802508DF804008DF8F0
:1045400003008DF8050006226946072008F012FADC
:1045500041B0BDE8F08F054A1378054A12785A43F6
:10456000520015F00CB9000070050020BA050020BB
:10457000BB0500202DE9FF4F87B0002006903220B8
:104580004FF000091446CDF80C900590FE484FF00E
:10459000FF3A4F460678FD48C8460078CDF80090AF
:1045A000CDF80490049000F01BFA05280CBF1E25DE
:1045B0001425FFF763FC029004984FF0000C0028CC
:1045C000C8BF4FF0020E64DD0021002E51DD0CFB50
:1045D0000610079A80B232F910B0AB45C4BF09F19A
:1045E00001020FFA82F934F91020AA420EDD039B72
:1045F0005B1C1BB203935245C4BF059B9A4205DD69
:104600001FFA8CF301938BB292460093029B33F90D
:1046100010309A1A12B2BBF1000F13DA002AB8BF99
:104620005242002BB8BF5B4293420BDA1BF1640F7E
:10463000BCBF0A9BA3F800E0079A32F81030089A32
:1046400022F8103034F91020002A0ADA9742B8BF55
:10465000174612F1460FBCBF08F101001FFA80F89F
:1046600003E0089B002223F81020481C01B2B1424D
:10467000ADDB0CF101000FFA80FC04988445A3DB4C
:10468000B8F1640F02D90A9807210180002FB8BF42
:104690007F42574514DCB9F1000F1CBF0398002876
:1046A0000ED0A6F101094FF000081FFA89F7BAF100
:1046B000000F01DD069838B10BB00120BDE8F08F86
:1046C0000BB00020BDE8F08FDDE9000101FB060E14
:1046D00034F91E3003EBD370B3F1FF3F4FEA6000B3
:1046E000B8BF404202B201FB06F01FFA80FC0098FE
:1046F00000B28346012839DB0CEB000189B2002BA4
:1047000018DD34F911A004EB410131F9021CBAEBB8
:10471000010A06D50029B4BFC1F1000A8A469245B4
:1047200004DB0029B8BF4942A9421BDA401E1FFA28
:1047300080F81BE016DA34F911A004EB410131F9DD
:10474000021CAAEB010ABAF1000F06DD0029B4BF72
:10475000C1F1000A8A469245E8DB0029B8BF494208
:10476000A942E3DB401E00B20128C5DACB4536DAA8
:104770000CEB0B0080B2002B16DD34F9101004EBAB
:104780004000B0F90200091A05D50028B4BF414223
:104790000146914204DB0028B8BF4042A84218DA23
:1047A0000BF1010087B21AE013DA34F9101004EBB0
:1047B0004000B0F90200091A002905DD0028B4BF45
:1047C000414201469142EBDB0028B8BF4042A8427B
:1047D000E6DB0BF101000FFA80FBCB45C8DB01984B
:1047E000DDF808C000FB068083B201983CF913C0D5
:1047F00000FB067034F8133082B2ACEB03031DB239
:104800000298029B1FFA8EF130F9110033F9123031
:1048100034F8111034F81220411A9A1A09B212B25F
:104820004C1B48BF6C1A8D1A48BF551A61190CB23F
:10483000B0EB0C0148BFACEB0001C21A48BF1A1A1A
:10484000881800B28442B8BF4FF0FF30BFF634AFD3
:104850000BB0BDE8F08F2DE9F05FDFF834A18046A2
:104860000026DAF80000374690F8241100291CBF12
:10487000B0F8300100286CD0FCF76DFDDAF80010BC
:1048800091F82411B0FBF1F201FB1200002860D175
:1048900001F084FC5FEA00095BD03E4800781028F4
:1048A00004BF484605F094F837484FF0000C4446E2
:1048B00090F800B03548634690F800E0BEF1000F74
:1048C00019DD34F9020B0125BBF1010F10DD34F9BC
:1048D000022B101A01B20029B8BF494208B2604544
:1048E00002DD84461E462F466D1C10465D45EEDBFC
:1048F0005B1C7345E5DBDAF80020B2F83001844533
:1049000027DB06FB0B7008EB400338F8101033F878
:10491000023CC91A39F8103009EB400009B230F8EE
:10492000020C181A081A00B20028B4BF434203460A
:104930000029B8BF49428B420BDA0028B8BF404279
:10494000B2F83211884204DA01F032FC0020BDE8EE
:10495000F09F0120BDE8F09F70B515460E46044655
:1049600008F0D1FB002C18BF70BD042818BF052823
:1049700006D00748006890F82400A84288BF70BDA0
:104980003046BDE8704007E0BA050020BB050020B6
:10499000F80600202D060020FFF782B970B51546F5
:1049A000044608F0B0FBB4F1FF3F0AD0002C18BF5A
:1049B00070BD002D08BF70BD2846BDE87040FFF7F0
:1049C0002FB9002D08BF70BD2846BDE87040FFF725
:1049D00059BA10B506F03EFD06F0D8FD002010BD16
:1049E000AC4800787047AB480078022805D005280D
:1049F0001CBF0020704705F0A0BB08F084BBA54990
:104A00000870704710B50446072C28BF10BDDFE8BA
:104A100004F016040810160C0800084600F044F9CB
:104A20000DE0084608F064FB09E0084605F07AFB53
:104A300005E0084607F0FEFF9749012008709548F9
:104A4000047010BD954900200968B1F8641011F494
:104A5000807F08BF7047FDF7EEB8904900200968D5
:104A6000B1F8641011F4807F08BF7047FDF70BB9EF
:104A70008A4900200968B1F8641011F4806F08BFFA
:104A80007047FDF724B98349487800281CBF401EB1
:104A90004870704710B572B6FEF740FFBDE8104091
:104AA000FEF7F2BC10B57E48FDF7A2FC72B6FEF729
:104AB00035FFBDE81040FEF7E7BC76480069704757
:104AC0007448C068704773494861704771484069CD
:104AD000704710B5FCF77DFAFBF70CFDFCF701F908
:104AE000FFF7C2FABDE81040FCF7E5BF10B5FCF7D0
:104AF00070FAFBF7FFFCFBF782FFFCF7F2F8BDE86A
:104B00001040FCF7D8BF30B5ADF2844D05464FF4E8
:104B10009061684614F0D4FE5E4C2846256106F08C
:104B2000ADFBE060F0B10278A2704178E17083786B
:104B30002371531C03F0FE0363710023E37123729E
:104B40004FF0120C84F806C004F10A0C8CF8003007
:104B50008CF80130007860721046FCF781FC0DF291
:104B6000844D30BD4D480068B0F8640010F4807F7B
:104B700018BFFDF788F800200DF2844D30BDF0B568
:104B8000ADF2CC4D0F4604464FF49061684614F0E8
:104B900097FE404D20462C6106F070FBE86000282F
:104BA00051D00278AA7041780446E9708078287163
:104BB000501C00F0FE0068710020E871287212237A
:104BC000AB7105F10A0318705870207868721046AE
:104BD000FCF746FC0DF59061204606F06CFB608A00
:104BE0006E6900281CBF7043060B002017F0040FED
:104BF00018BF062017F0080F18BF40F00200616AC6
:104C00000840DDF88014CDF8C014DDF89C14CDF810
:104C1000C414DDF89014CDF8C8140DF59861FCF7B4
:104C2000EBF9DDF88C0420B13346EA78A97805F079
:104C3000BDFD6421304605F06CFE287802280FD0B7
:104C4000052810D017E015480068B0F8640010F48B
:104C5000807F18BFFDF717F800200DF2CC4DF0BD96
:104C600008F051FA01E005F068FA022804BFDDF807
:104C70009404FFF74CF9002001F08FFA0DF2CC4DAF
:104C80000120F0BD10B5FCF76FFA02490020C860A2
:104C9000012010BDB80500203A070020F8060020CA
:104CA00000FE1100F9487047F94948707047F8480C
:104CB00040787047F74810B4F74A0168914218D11C
:104CC0004168B1F5887F14D80022D0F808C00346A7
:104CD0001146B2EB9C0F24BF10BC704753F8214023
:104CE000491C2244B1EB9C0FF8D3002A04BF10BC2E
:104CF0007047002010BC70474FF4FC30FDF7F0BB4C
:104D00002DE9F0410446E3480E46E34F0168B942FD
:104D100013D14168B1F5887F0FD80023D0F808C0BF
:104D200001461A46B3EB9C0F08D251F82250521C90
:104D30002B44B2EB9C0FF8D303B10020002558B1EF
:104D4000B0E80E10A4E80E10B0E80E10A4E80E10A3
:104D50000FC884E80F0016E0FF223021204614F02F
:104D600085FD4FF48870C4E900703020C4E9020565
:104D7000AA20C4E904054FF0FF30E062A062A561FB
:104D80006062C4E9075066B94FF4FC30FDF7A8FB38
:104D9000C248056045608560C56005614561856103
:104DA000C5610120BDE8F081B94901204870704714
:104DB000B74900200870704770B5ADF5107D044606
:104DC000FFF77EFE054614F0020F04BF0DF5107DBF
:104DD00070BD0426FFF707FE002818BFB04C08D0AE
:104DE00095F92C102246304606F08AFA0DF5107D12
:104DF00070BD6C462046FCF727FDF1E770B50D4607
:104E000006461024FFF75CFE16F0020F18BF0524BB
:104E10002A46102C28BF70BD002A08BF70BD204450
:104E200090F928102046BDE8704006F069BA2DE9D7
:104E3000F04F87B08146122000244FF0200A274609
:104E40000090FFF7CDFD022802D108F05CF930B1E7
:104E5000FFF7C6FD052804D105F06FF908B9022057
:104E600000900098002500289CBF07B0BDE8F08F97
:104E70000026BAF1000F7CD98A4A681EA2FB0031D5
:104E80004908A1EB810108440590E81E0490A81F81
:104E90000390C01E0290C01E0190A2FB05104008A6
:104EA000A0EB8000A5F10F0B00EB0508FFF798FDC4
:104EB000022803D108F027F900283AD0FFF790FD27
:104EC000052803D105F039F9002832D0032D38BF69
:104ED000142417D30498032838BF152412D3039839
:104EE000032838BF16240DD30298032838BF242482
:104EF00008D30198032838BF252403D3BBF1030F3F
:104F000038BF2624A7420AD06748C4F303112746B6
:104F10000068C16104F00F017F20FBF795FAC4F32C
:104F2000031001281CBFC6F11F0000EB481018D168
:104F300027E0002D0CBF14242424A74209D05A488E
:104F4000210927460068C16104F00F017F20FBF7AB
:104F50007BFA2009012814D00598C6F11F0101EB46
:104F6000401019F8011BC0B2FBF76EFA761C5645CB
:104F70009CD300986D1C8542FFF47AAF07B0BDE862
:104F8000F08F06EB4810ECE72DE9F84F83464048D8
:104F90004FF0000A0C46B0F904804FF012092027A8
:104FA00050460091FCF756FA0546CBF10706FFF78D
:104FB00017FD022802D108F0A6F830B1FFF710FD66
:104FC000052804D105F0B9F808B94FF00209BBF182
:104FD000000F1CD0002E55DB4FF0000CB9F1000F74
:104FE00049D9012101FA06F3701E01FA00FB0021E4
:104FF000002F3CD935F8020B2278A0EB080000B254
:105000005FEAD21E23D0002827DA2EBB1BE0002344
:10501000B9F1000F2FD90021002F10D935F8022B3C
:105020002078A2EB080212B2502AC8BF40F08000DC
:1050300040F04000491C04F8010BB942EED35B1C60
:105040004B45E8D317E010F1280F05DB0AE00028F4
:1050500003DD0EB9282805DD9A43002EC4BF4BEAB4
:105060000200C2B204F8012B491CB942C2D30CF1B0
:10507000010CCC45BBD30098FFF7D9FE002E08BF2A
:105080004FF0010A5046BDE8F88F0000482F00207D
:10509000D005002000F8110054435246A816002005
:1050A00088310020ABAAAAAA8CAE1100FD498880E5
:1050B000704770B5FB4EFC49F08009680320C86159
:1050C0000425E9B27F20FBF7BFF90024B179E0B2F3
:1050D000FBF7BAF904F12000B179C0B2FBF7B4F9DB
:1050E00004F14000B179C0B2FBF7AEF9641C202C8A
:1050F000ECDB6D1C072DE4DB70BD2DE9F04F89B0B2
:105100000026FBF766FFE849072009680865E748BD
:10511000016841F0200101600020FFF7CAFFE1496A
:105120004FF4006088804FF41071E14814F0C8FB20
:105130000020FBF7E2FDFCF7B9F800252C460795A7
:10514000FFF751FC04F04BF901281DD06846FCF72D
:105150005AFBB8B10120FBF7D0FD684604F09FFD73
:105160006D1C012D0ED00025D1492046FFF70CFF04
:10517000072C1ED00020FBF7C0FDFCF761FBFCF7FD
:1051800095F8641C002EDDD0FFF72DFCC54AC948F8
:10519000C74BD0600020D16813F800C0401C01F854
:1051A00001CBD160B0F5107FF5D3079800283CD132
:1051B00035E012200890BB4800274FF0200BB0F9D3
:1051C00004603846FCF746F90546BA460024BBF1B0
:1051D000000F18D9304615F05AF8B74AB74B15F0FA
:1051E000BDF88946804635F9022B901B48BFB01A9E
:1051F00015F04DF842464B4615F0AEF938BF7F1C0E
:10520000641C5C45EFD308980AF1010A8245DDD39E
:10521000002F4FF001061CBF01200790B4E7002EBD
:105220001EBF002009B0BDE8F08F012009B0BDE825
:10523000F08FF0B587B000260120FBF704FD9B48F6
:10524000016841F0200101600020FFF732FF95491D
:105250004FF4006088809A490020C1F88000C1F8AE
:105260008400C1F88800C1F88C00C1F89000C1F832
:105270009400C1F89800C1F89C00C1F8A000C1F8E2
:10528000A400C1F8A800C1F8AC00C1F8B000C1F892
:10529000B400C1F8B800C1F8BC00FBF72EFDFCF764
:1052A00005F800252C462F4604F099F8012835D042
:1052B0006846FCF7A8FA78B30120FBF71EFD6D1CC9
:1052C000012D24D000257F492046FFF75DFE072CE5
:1052D00006D00020FBF711FDFBF7E8FF641C1BE084
:1052E000002420252046FCF7B5F8002130F9022BD8
:1052F000A2F26662B2F54D7F88BF641C491CB1EB17
:10530000450FF3D3002C08BF01260DD106E0002085
:10531000FBF7F3FCFBF7CAFF002EC5D027B9002E20
:105320001EBF002007B0F0BD012007B0F0BD2DE981
:10533000F04F83460021ADF5137D634890910C46F4
:1053400000780F460D46022808BF012703D0052824
:1053500004BF02240427DFF850914FF0010A00F047
:10536000A1B9204605F08AFF002800F09A81008943
:1053700000EA0B0626F0CC0030F47C4000F091816E
:10538000DFF84881D8F800004069D8F8001040F4F0
:1053900000704861D8F800000069D8F8001020F0CB
:1053A00006000861D8F800000069D8F8001040F045
:1053B000100008613CB1012C35D0022C71D0032CB7
:1053C00055D000F0FDB802210846FFF71BFB012075
:1053D000FBF739FC05F0BBFD0F212046FFF7CFFBA3
:1053E000002800F05E81D9F80000406CD9F8001068
:1053F00040F40060486400BF00BF00BFD9F800005F
:10540000406CD9F8001020F400604864FBF7AFFB53
:1054100005F086FD012007F06EFF0020FBF76DFC14
:10542000FCF70EFACCE000210220FFF7EBFA012096
:10543000FBF709FC0F212046FFF7A1FB002800F035
:105440003081D9F80000406CD9F8001040F40060B9
:10545000486400BF00BF00BFD9F80000406CD9F815
:10546000001020F400604864FBF781FBA8E00021F5
:105470000520FFF7C7FAFBF7ACFDD8F8000000697C
:10548000D8F8001020F006000861D8F80000006984
:10549000D8F8001040F004000861D8F80000006956
:1054A00016E03EE0D00500208CAE1100640500201F
:1054B00088310020482F00209A9999999999B93FED
:1054C00048330020C83300202506002078AE1100A4
:1054D000D8F8001040F01000086112F042FF0F21D0
:1054E0000220FFF74CFB00287ED0DFF884850720E0
:1054F000D8F800108860D8F8001004204860022115
:105500002020FBF7ADFF0020FBF7F7FBFBF7A5FE24
:10551000D8F800000068D8F8001040F001000860DA
:105520004EE002210520FFF76DFAFBF752FDD8F897
:1055300000000069D8F8001020F006000861D8F8D3
:1055400000000069D8F8001040F004000861D8F8A5
:1055500000000069D8F8001040F01000086112F057
:1055600000FF05F0DDFC0F210320FFF708FB0028FA
:105570003AD0DFF8FC847F20D8F800108860D8F893
:10558000001002204860D9F80000406CD9F80010E3
:1055900040F400604864012007F047FCD9F800009F
:1055A000406CD9F8001020F400604864FBF755FE09
:1055B000D8F800000068D8F8001040F0010008603A
:1055C0009098002868D116F0010F27D00120FBF732
:1055D0003AFB0020FBF7B1FBFFF705FA98B1FCF7A7
:1055E00003F8FF210F2000E05BE0FFF786FD2AEAC9
:1055F000000005430020FBF780FB0120FBF79DFB2B
:10560000909888BB0AE0FBF7EFFFFF210F20FFF720
:1056100010FE2AEA000045EA4005EBE716F0060F07
:1056200022D0FFF7E0F902281ED1FEF7CDFA0020C4
:10563000FEF752FD0120FBF706FBFEF71FFC0646B6
:10564000FFF73EFA0523320004D090F92D101846DA
:1056500005F056FEFEF712FCFEF721FDFEF70EFCEC
:105660004FF4906114F00AF9FFF72AFA80460420FB
:105670009190FFF7B8F9002818BFFE4E20D098F996
:105680002C103246919805F03BFEFB490020087033
:10569000FA490870FBF7E1FDFFF7A2F9F84880F836
:1056A00000A0641CBC4203D2909800283FF459AE7D
:1056B000F449002008700DF5137D2846BDE8F08FF1
:1056C0006E463046FCF7C0F8D9E770B5ED48CCB06F
:1056D0004578FFF785F901287ED1EB480068B0F9DD
:1056E0003610B0F9340005F087F915F0020F74D0C8
:1056F000002140A8FFF704FB4598401C459040F26C
:105700007770FFF714FEC0B2032810D0002804BF42
:1057100045F25000449012D0012808BF4AF25010C0
:105720000CD0022808BF45F2A10007D007E04AF2DA
:10573000A11044904698401C469008E04490479839
:105740000022401C47902121072007F0EAF840ACD6
:1057500005F085FD40B181694891C1694991416970
:105760004A91C0684B9005E04FF0FF304B904A9053
:1057700049904890C54840904FF48870419030203F
:10578000429000204390A3682246014652F820C070
:10579000401C6144B0EB930FF8D34E42FF22511CE2
:1057A0006846E66014F062F8A268F4E804018DE847
:1057B00047000FCC04AE86E80F0094E80F0008AE57
:1057C000203C86E80F004FF4FC306946FCF729FFC7
:1057D000AF4922680A6001E021E00CE062684A609B
:1057E00022698A606269CA60A2690A61E2694A61E3
:1057F000226A8A610CE015F0010F09D040F22220E4
:10580000FFF795FD20B900222121072007F089F834
:10581000FEF72FFB2A464021072007F082F84CB004
:10582000BDE8704003F0D7BD70B50C4699490546F8
:1058300003200968C86101217F20FAF705FE0021D5
:105840007520FAF701FE01217620FAF7FDFD6021AF
:105850000820FAF7F9FD00210920FAF7F5FD3021BB
:105860000A20FAF7F1FD00210B20FAF7EDFD0521E2
:105870000E20FAF7E9FDE1B22620FAF7E5FDE1B2E4
:105880002720FAF7E1FDE1B22820FAF7DDFDE1B2C9
:105890002920FAF7D9FDE1B22A20FAF7D5FDE1B2C5
:1058A0003020FAF7D1FDE1B23120FAF7CDFDE1B2B7
:1058B0003220FAF7C9FDE1B23320FAF7C5FDE1B2B3
:1058C0003420FAF7C1FDE1B23620FAF7BDFDE1B2AE
:1058D0003720FAF7B9FDE1B23820FAF7B5FDE1B2A9
:1058E0003920FAF7B1FDE1B23A20FAF7ADFDE1B2A5
:1058F0004020FAF7A9FDE1B24120FAF7A5FDE1B297
:105900004220FAF7A1FDE1B24320FAF79DFDE1B292
:105910004420FAF799FDE1B24620FAF795FDE1B28D
:105920004720FAF791FDE1B24820FAF78DFDE1B288
:105930004920FAF789FDE1B24A20FAF785FDE1B284
:105940005020FAF781FDE1B25120FAF77DFDE1B276
:105950005220FAF779FDE1B25320FAF775FDE1B272
:105960005420FAF771FDE1B25620FAF76DFDE1B26D
:105970005720FAF769FDE1B25820FAF765FDE1B268
:105980005920FAF761FDE1B25A20FAF75DFDE1B264
:105990006020FAF759FDE1B26120FAF755FDE1B256
:1059A0006220FAF751FDE1B26320FAF74DFDE1B252
:1059B0006420FAF749FDE1B26620FAF745FDE1B24D
:1059C0006720FAF741FDE1B26820FAF73DFDE1B248
:1059D0006920FAF739FDE1B26A20FAF735FD0221B4
:1059E0007F20FAF731FD6A210220FAF72DFD8E2182
:1059F0000420FAF729FDF3210720FAF725FD0421F9
:105A00000820FAF721FD15B1012D05D008E0042189
:105A10000620FAF719FD03E008210620FAF714FD25
:105A200003217F20FAF710FD21211020FAF70CFD49
:105A300000211120FAF708FD00211220FAF704FDD9
:105A400000211320FAF700FD00211420FAF7FCFCD6
:105A500000211520FAF7F8FC01211620FAF7F4FCD2
:105A600002211720FAF7F0FC0021182014E00000B2
:105A700090AE11008831002038070020390700203F
:105A80003A070020D0050020F80600205443524673
:105A9000A81600208CAE1100FAF7D6FC00211920C0
:105AA000FAF7D2FC00211A20FAF7CEFC00211B20C5
:105AB000FAF7CAFC01212020FAF7C6FC2021212098
:105AC000FAF7C2FC00212220FAF7BEFC00212320B5
:105AD000FAF7BAFC00212420FAF7B6FC00212520B1
:105AE000FAF7B2FC01212620FAF7AEFC00212720AC
:105AF000FAF7AAFC02212820FAF7A6FC00212920A7
:105B0000FAF7A2FC00212A20FAF79EFC00212B20A4
:105B1000FAF79AFC01213020FAF796FC0021312097
:105B2000FAF792FC20213220FAF78EFC0021332074
:105B3000FAF78AFC00213420FAF786FC0021352090
:105B4000FAF782FC01213620FAF77EFC002137208B
:105B5000FAF77AFC00213820FAF776FC0221392086
:105B6000FAF772FC00213A20FAF76EFC00213B2084
:105B7000FAF76AFC01214020FAF766FC0021412077
:105B8000FAF762FC00214220FAF75EFC2021432054
:105B9000FAF75AFC00214420FAF756FC0021452070
:105BA000FAF752FC01214620FAF74EFC002147206B
:105BB000FAF74AFC00214820FAF746FC0021492068
:105BC000FAF742FC02214A20FAF73EFC00214B2062
:105BD000FAF73AFC01215020FAF736FC0021512057
:105BE000FAF732FC00215220FAF72EFC0021532054
:105BF000FAF72AFC20215420FAF726FCBDE8704071
:105C000000215520FAF720BC10B50322FD490628D3
:105C100028BF10BDDFE800F00327FDFCFBFA086891
:105C2000C26101217F20FAF70FFCAF210820FAF7AB
:105C30000BFC73210A20FAF707FC0A210E20FAF761
:105C400003FC02217F20FAF7FFFB00210720FAF76F
:105C5000FBFB1F210120FAF7F7FB1021BDE81040E4
:105C60000620FAF7F1BB0868C26101217F20FAF72C
:105C7000EBFB0D210E20FAF7E7FB87210820FAF74E
:105C8000E3FB6E210A20FAF7DFFB02217F20FAF7FF
:105C9000DBFB71210720FAF7D7FB6A210220FAF714
:105CA000D3FB8E210420FAF7CFFB03217F20FAF7E4
:105CB000CBFB61211020FAF7C7FB00211120FAF776
:105CC000C3FB00211220FAF7BFFB00211320FAF7D3
:105CD000BBFB00211420FAF7B7FB00211520FAF7CF
:105CE000B3FB01211620FAF7AFFB06211720FAF7C4
:105CF000ABFB00211820FAF7A7FB00211920FAF7C7
:105D0000A3FB00211A20FAF79FFB00211B20FAF7C2
:105D10009BFB01212020FAF797FB60212120FAF755
:105D200093FB00212220FAF78FFB00212320FAF7B2
:105D30008BFB00212420FAF787FB00212520FAF7AE
:105D400083FB01212620FAF77FFB00212720FAF7A9
:105D50007BFB06212820FAF777FB00212920FAF7A0
:105D600073FB00212A20FAF76FFB00212B20FAF7A2
:105D70006BFB01213020FAF767FB00213120FAF795
:105D800063FB60213220FAF75FFB00213320FAF732
:105D90005BFB00213420FAF757FB00213520FAF78E
:105DA00053FB01213620FAF74FFB00213720FAF789
:105DB0004BFB00213820FAF747FB06213920FAF780
:105DC00043FB00213A20FAF73FFB00213B20FAF782
:105DD0003BFB01214020FAF737FB00214120FAF775
:105DE00033FB00214220FAF72FFB60214320FAF712
:105DF0002BFB00214420FAF727FB00214520FAF76E
:105E000023FB01214620FAF71FFB03E03FE039E0C6
:105E100033E02DE000214720FAF716FB002148204F
:105E2000FAF712FB00214920FAF70EFB06214A205F
:105E3000FAF70AFB00214B20FAF706FB012150205C
:105E4000FAF702FB00215120FAF7FEFA0021522056
:105E5000FAF7FAFA00215320FAF7F6FA60215420F3
:105E6000FAF7F2FA0021BDE810405520FAF7ECBA33
:105E7000AA21BDE810400020D6E45521BDE810401D
:105E80000020D1E4AA21BDE810400120CCE4552136
:105E9000BDE810400120C7E410B5FDF7EFFF044650
:105EA000FDF7EEFF2146BDE810404FF4906213F07D
:105EB00066BC2DE9F0415448047854480578FDF754
:105EC000DFFF0646FDF7DAFF0022002D98BFBDE890
:105ED000F0810021002C10D902FB04FC06EB4C03DE
:105EE00000EB4C0C11F0010F1CBF33F811702CF8B3
:105EF0001170491CC9B2A142F4D3511CCAB2AA42C2
:105F0000E7D3BDE8F08100B5ADF2844DFDF7B8FFF1
:105F100001464FF49062684613F031FC6846FDF785
:105F2000B1FF0DF2844D00BD2DE9F04F83B012207A
:105F30000190384836494FF020090024C16001E043
:105F4000032C01DA14261AE0E01E032838BF1526B8
:105F500015D3A01F032838BF162610D3A4F10900BB
:105F6000032838BF24260AD3A4F10C00032838BF25
:105F7000252604D3A4F10F00032838BF2626B345F5
:105F800009D020483109B3460068C16106F00F010D
:105F90007F20FAF759FA0025B9F1000F2ADD1E48D3
:105FA0004FEA161A80FB0410A0EBE070A0EB800013
:105FB00000EB0408BAF1010F0EBF05EB4810C5F164
:105FC0001F0000EB481087B21249C86810F8012B77
:105FD0000092C860F8B21146FAF736FA00BF00BF67
:105FE00000BF00BF00BFF8B20099FAF72DFA6D1C90
:105FF0004D45DFDB0198641C8442A1DB03B0BDE8A2
:10600000F08F00008CAE1100BA050020BB05002007
:10601000482F0020D0050020565555552DE9F84F42
:10602000DFF8D8B174484FF02008CBF80C001220EC
:106030000024009001E0032C01DA14261AE0E01E8F
:10604000032838BF152615D3A01F032838BF1626EE
:1060500010D3A4F10900032838BF24260AD3A4F1E1
:106060000C00032838BF252604D3A4F10F00032811
:1060700038BF2626B24509D061483109B2460068CA
:10608000C16106F00F017F20FAF7DEF90025B8F1B3
:10609000000F1EDD5B484FEA161980FB0410A0EBD1
:1060A000E070A0EB80000719B9F1010F0EBF05EBFE
:1060B0004710C5F11F0000EB471080B2FAF7DDF979
:1060C000DBF80C106D1C454501F8010BCBF80C10EA
:1060D000EADB0098641C8442ADDBDBF80C00BDE811
:1060E000F88F4648C08870472DE9F043002787B0F5
:1060F000B946FAF76EFF41494FF400608880FAF71D
:106100000CFE0020FAF7F9FD00254FF05A0828464A
:10611000FEF7CFFFFBF7A1F803F061F96846FBF744
:1061200072FB28B3684603F0BAFD002420262046FF
:10613000FBF790F9002130F9022BA2F26662B2F56A
:106140004D7F88BF641C491CB1EB460FF3D3ACB143
:10615000454515D2FAF73DFFA8B26D1CFEF7A9FF21
:10616000FBF77BF806F0CFFF002808BFFBF78CFE9B
:10617000002FD1D0B9F1000F0BD104E00127F9E7CE
:10618000FAF727FF05E0002F1EBF002007B0BDE88B
:10619000F083012007B0BDE8F0837047174881689D
:1061A00000291BBF017811F0020F0020C068704762
:1061B00015481249006890F825218878401CC0B223
:1061C0008870824228BF70470020887001210846ED
:1061D000FEF718BC10B506F096FF074902284FF4E9
:1061E000107204D0BDE81040084813F0C8BABDE8EA
:1061F0001040074813F0C3BA482F0020D0050020F4
:106200008CAE110056555555F8060020F80C0020AC
:10621000305E002003F00702FD4B012A04BF02207C
:10622000587104D0022A04BF5A79022A01D00020F2
:106230007047F84A127802700120087003205871E4
:10624000012070471FB513F0070F069804D003F024
:106250000702022A08D004E0012202A9112003F05B
:106260009AF804B0002010BDE94B5A79052A0DD1E7
:10627000DA8982423CBF521CDA8192B2824205D155
:106280000020D881012008700320587104B001203B
:1062900010BD1FB513F0070F04D003F0070002284C
:1062A00008D004E0012202A9112003F074F804B020
:1062B000002010BD0120087004B010BD1FB513F000
:1062C000070F04D003F00700022808D004E00122E1
:1062D00002A9112003F05FF804B0002010BD0120D6
:1062E000087004B010BD1FB513F0070F04D003F001
:1062F0000700022808D004E0012202A9112003F0BF
:106300004AF804B0002010BD0120087004B010BD90
:106310001FB513F0070F04D003F00700022808D0C0
:1063200004E0012202A9112003F035F804B0002096
:1063300010BD0120087004B010BD2DE9F00703F076
:1063400007050027B24EDDF81CC0012D08BFF781FC
:106350000DD013F0070FAE4BDFF8BC82DFF8BC9214
:10636000DB8903F10104A4B205D0022D16D0BDE8EB
:10637000F0070020704763453CBFD9F80000C254C5
:10638000F481644524D1D9F80000D9F80010407890
:10639000097800EB0120A8F80E0019E0B8F80E20EB
:1063A000D9F80050120A63452A70D9F8005098F8BD
:1063B0000E206A7004D2D9F80020D25C0270F481F9
:1063C000F089604504D1F7810120087003207071C5
:1063D000BDE8F007012070471FB513F0070F04D088
:1063E00003F00700022808D004E0012202A91120CE
:1063F00002F0D1FF04B0002010BD0120087004B0ED
:1064000010BD1FB513F0070F04D003F007000228DA
:1064100008D004E0012202A9112002F0BCFF04B060
:10642000002010BD0120087004B010BD1FB513F08E
:10643000070F04D003F00700022808D004E001226F
:1064400002A9112002F0A7FF04B0002010BD012016
:10645000087004B010BD1FB513F0070F069804D0E4
:1064600003F00702022A08D004E0012202A9112049
:1064700002F091FF04B0002010BD654B5A79052A47
:106480000DD1DA8982423CBF521CDA8192B282423B
:1064900005D10020D881012008700320587104B074
:1064A000012010BD0020704708B503F00700012847
:1064B00006D18DF80000024669460B2002F06BFF02
:1064C000002008BD08B503F00700012807D100200F
:1064D0008DF80000012269460B2002F05CFF0020CD
:1064E00008BD10B503F00700012808BFFEF7D2FA77
:1064F000002010BD08B503F00700012807D10320D4
:106500008DF8000001226946002002F044FF0020BF
:1065100008BD08B503F00700012807D103208DF856
:10652000000001226946002002F035FF002008BD6E
:1065300070B403F007020024354BDDF80CC0012ACB
:1065400002D0022A08D004E005205871DC811C63C7
:106550009C8270BC002070475A79052A11D1DA89D3
:10656000624506D22E4DAD68D600F5400570501C30
:10657000D881D889604504D1DC81012008700320CE
:10658000587170BC012070471FB513F0070F08D178
:106590009DF80800F02807D0012202A9072002F088
:1065A000FAFE04B0002010BDFEF7A6FBF9E71FB508
:1065B00013F0070F04D1012202A9104602F0EBFEEE
:1065C00004B0002010BDF0B403F00705104E012DFB
:1065D00004BF0020F08117D013F0070F114BD3F840
:1065E00000C00B4BDB8903F10104A4B202D0022DE1
:1065F0001AD009E0002B08BF8CF8EB2003D0012B48
:1066000008BF8CF8EA20F4810020F0BC704700003D
:10661000E80500202C0600208C100020BCAE1100E4
:10662000A8160020F8060020002B04BF9CF8EB10F1
:10663000017006D0012B04D19CF8EA2002700120E1
:106640000870F4810120E0E730B403F0070CF84C47
:10665000BCF1010F04BF0020E08118D013F0070F38
:10666000F34BDB8903D0BCF1020F13D00FE073B9F9
:10667000A271082A0BD2DFE802F004070704040421
:1066800004044FF4906001E04FF41070E06230BCFD
:1066900000207047E64A002BD26A04BF110A01703D
:1066A00004D0012B02D1027001200870581CE08137
:1066B00030BC01207047F8B5054603F007000026FE
:1066C000DB4C0F46012807D013F0070F2346DB8968
:1066D00006D0022828D025E005206071E68121E05F
:1066E00003BBA2714FF49060A0824010082A19D217
:1066F000DFE802F004060A0E10121416CD4810E06E
:10670000CD492163A0820DE0CC492163A08209E03C
:10671000CB4806E0CB4804E0CB4802E0CB4800E0A1
:10672000CB4820630020F8BD6079052847D1206B55
:10673000002844D0C749BE4A0968928A91F8EB10F4
:10674000012918BF032906D0694693422DD213F0C0
:10675000030F21D118E0934227D213F0010F07D085
:1067600094F82C002870E06A000AE062581C1BE0D4
:10677000AF49A079C989042821F0010214BFB648A5
:10678000B648805EE062EBE70422FBF72BFD009841
:10679000E062206B001D206394F82C002870E06AF2
:1067A000000AE062E089401CE081E089A18A884219
:1067B00005D1E68101202663387003206071012035
:1067C000F8BD2DE9F84303F007020026984D089C18
:1067D0000F468046012A02D0022A06D002E0052098
:1067E0006871EE810020BDE8F883687905281CD126
:1067F000E889A04211D2FCF7FEFFAC208DF8000022
:106800007A208DF8010070208DF80200EA891DF8C9
:10681000020088F80000501CE88180B2A04204D138
:10682000EE8101203870032068710120BDE8F883F3
:106830002DE9F04182B003F0070200267C4D089C50
:106840000F468046012A02D0022A07D002E0052026
:106850006871EE8102B00020BDE8F08168790528FA
:1068600021D1E889A04216D2FCF7C5FF53208DF84C
:10687000000045208DF801007A208DF8020070207C
:106880008DF803008DF80460EA891DF8020088F88D
:106890000000501CE88180B2A04204D1EE810120AA
:1068A00038700320687102B00120BDE8F0812DE945
:1068B000F00388B003F007020027DFF87481DDF8E9
:1068C00038C0012A09D04446E489651CAEB2022AC8
:1068D0000DD013F0070F2FD004E0052088F8050035
:1068E000A8F80E7008B00020BDE8F003704798F8D3
:1068F0000520052A1BD164450ED2594D00226B4656
:1069000015F8029003F80290521CD2B2202AF7D355
:106910001A5D0270A8F80E60B8F80E00604506D146
:10692000A8F80E7001200870032088F8050008B050
:106930000120BDE8F0037047644538BFA8F80E6039
:10694000B8F80E00604508BFA8F80E70CAE72DE938
:10695000F007DFF800C183B003F0070ADCF800C0DD
:106960000A9A0027BCF81640BCF81450DFF8C08023
:10697000BAF1010F0ED0C4464FF00109BCF80EC0A9
:10698000BAF1020F0CF10106B6B20DD013F0070FE9
:1069900040D004E0052088F80500A8F80E7003B088
:1069A0000020BDE8F007704798F80530052B2CD182
:1069B00094451FD2230A8DF800308DF804304FEA39
:1069C000152A12238DF808308DF801408DF8054006
:1069D00020238DF802A08DF806A08DF809308DF8DF
:1069E00003508DF807508DF80A701DF80C300370B5
:1069F000A8F80E60B8F80E00904206D1A8F80E7004
:106A000081F80090032088F8050003B00120BDE85C
:106A1000F00770471348944580F8009038BFA8F8F5
:106A20000E60B8F80E00904208BFA8F80E70B6E7E6
:106A3000E805002054B0020054D8020054DC0200E3
:106A400054C8020054D0020054C0020054B80200DE
:106A500054EC0200F80600200069002000710020BC
:106A600008340020680700202DE9F04383B08046F9
:106A700003F007000026FF4D0A9C0F46012802D0B4
:106A8000022807D002E005206871EE8103B00020E3
:106A9000BDE8F083687905282DD1E8894FF0010918
:106AA000A04220D20021B220FBF726F98DF8000089
:106AB000010A8DF80110010C8DF80210000E8DF8FE
:106AC00003007A208DF804001F208DF805000420B3
:106AD0008DF807008DF80690E8891DF8001088F8F9
:106AE0000010401CE88180B2A04204D1EE8187F8FA
:106AF00000900320687103B00120BDE8F0832DE908
:106B0000F84303F007020026DA4D089C0F46804642
:106B1000012A02D0022A06D002E005206871EE8127
:106B20000020BDE8F8836879052814D1E889A042DF
:106B300009D26846FBF741FEEA891DF8020088F891
:106B40000000501CE88180B2A04204D1EE810120F7
:106B50003870032068710120BDE8F88310B403F099
:106B60000701DFF810C3012906D013F0070FC24B4D
:106B700008D0022910D00CE00020ACF80E00ACF8D0
:106B8000100006E0BCF80E0019680A54401CACF86E
:106B90000E0010BC00207047BCF810101A68525C40
:106BA0000270481CACF8100010BC01207047F0B512
:106BB00083B003F0070201270025AF4CAD4EDDF88E
:106BC00020C0012A04D0022A00F0C68000F09DB83F
:106BD000FCF711FE012202A912200295FBF702FB2D
:106BE0000520707121687A2008702068477021683C
:106BF00021208870A14822680168897CD1700068D2
:106C00002268017C1171017E11F0040F0ED0C18A3F
:106C10002268090A51712268817D9171818A2268F6
:106C2000090AD1712168007D08720DE0818A22680D
:106C3000090A51712268017D9171C18A2268090A8D
:106C4000D1712168807D0872042269461046009542
:106C5000FBF7C8FA2168009848722268010A91720D
:106C60002268010C000ED172216804220873694663
:106C700014200095FBF7B6FA216800984873226843
:106C8000010A91732268010C000ED1732168087407
:106C90000298009500283BD0042201A948200195C4
:106CA000FBF7A0FA019804225030019069461C308D
:106CB000FBF798FA2168009848742268010A9174D9
:106CC0002268010C000ED174216804220875009519
:106CD00001A948200195FBF785FA0198042250305C
:106CE000019069462C30FBF77DFA216800984875C1
:106CF0002268010A91752268010C000ED175216885
:106D000008762168FF204876F58103B00020F0BDA9
:106D1000042269465A48FBF765FA216800984874CE
:106D20002268010A91742268010C000ED174216856
:106D300004220875694653480095FBF753FA216809
:106D4000009848752268010A91752268010C000EAE
:106D5000D17521680876D4E77279052A0ED1F289B7
:106D6000624504D223689B5C0370501CF081F0895B
:106D7000604503D1F5810F700320707103B00120CD
:106D8000F0BD30B403F007043B4B3A4D029A4FF08C
:106D9000000C012C02D0022C38D034E002206871A3
:106DA0003948A5F80EC00168880A444211EB8424D2
:106DB00018BF401C404201EB8000C01C20F00300C3
:106DC0003249B0F5003F014414D8CC78086864F328
:106DD0001F602F4CA0420DD10020002A13D901EBD7
:106DE000000C1C689CF804C004F800C0401C8242DF
:106DF000F5D808E00020002A05D9196801F800C07C
:106E0000401C8242F9D830BC002070476C79022CBB
:106E100010D1EC89944204D21B681B5D0370601C86
:106E2000E881E889904205D1A5F80EC001200870DC
:106E30000320687130BC0120704738B503F00702A9
:106E40000D4C00250B4BDDF810C0012A02D0022AA0
:106E50007ED086E0022058710E48DD8100680E4920
:106E6000884245D10D480168226811700168226886
:106E7000090A15E0E8050020BCAE1100F806002064
:106E80005CC001006CC0010000FE1100E8FF0F00B3
:106E900034CD12AB8416002054464953901600207E
:106EA000517001682268090C917001682268090E0E
:106EB000D17041682268117141682268090A5171D4
:106EC00041682268090C917141682268090ED171EC
:106ED00081682268117281682268090A517281688A
:106EE0002268090C917280682168000EC87238E02F
:106EF0000422694620200095FBF774F92168009868
:106F00000422087000982168000A487000982168DF
:106F1000000C887000982168000EC8706946242013
:106F2000FBF760F92168009808712268010A517125
:106F30002268010C000E917121680422C871694613
:106F40002820FBF74FF9216800980872010A00E039
:106F500009E0226851722268010C000E91722168CA
:106F6000C872002038BD5A79022A0FD1DA896245E9
:106F700004D22468A45C0470501CD881D889604570
:106F800004D1DD810120087003205871012038BD33
:106F900070B503F007020025FA4CFB4BDDF810C07A
:106FA000012A03D0022A0DD0002070BD02205871A2
:106FB000DD8104F013F9002814BF802040202168EF
:106FC0000870F1E75A79022A0FD1DA89624504D2B2
:106FD0002468A45C0470501CD881D889604504D111
:106FE000DD810120087003205871012070BD70B54B
:106FF00003F007020025E34CE34BDDF810C0012A43
:1070000002D0022A10D00DE002205871DD8100204C
:10701000FBF73BFF05460120FBF737FF216845EAF8
:1070200000100870002070BD5A79022A0FD1DA8949
:10703000624504D22468A45C0470501CD881D889AD
:10704000604504D1DD8101200870032058710120C2
:1070500070BD30B403F007020024CA4DCA4BDDF8FE
:1070600008C0012A02D0022A09D005E00220587186
:10707000DC8129685520087030BC002070475A799F
:10708000022A0FD1DA89624504D22D68AD5C057001
:10709000501CD881D889604504D1DC81012008705A
:1070A0000320587130BC012070472DE9F84303F0EC
:1070B00007020026B34DDFF8D082089C4FF001098B
:1070C000012A02D0022A2CD028E004F0C8F88769EF
:1070D000022088F80500A8F80E6004226946002006
:1070E000FBF780F8A948009981420FD1286880F801
:1070F0000090296804204870286887702968380A39
:10710000C870286846712868867107E00020002C46
:1071100004D929680E54401C8442FAD80020BDE8E6
:10712000F88398F80520022A14D1B8F80E20A2425C
:1071300005D22B689B5C0370501CA8F80E00B8F8B1
:107140000E00A04206D1A8F80E6081F8009003203E
:1071500088F805000120BDE8F883F8B503F00702C0
:10716000884C0025884EDDF818C0012A02D0022A7A
:1071700070D06CE004F073F800282ED084480168C9
:107180002268117001682268090A5170016822683A
:10719000090C917001682268090ED170416822685B
:1071A000117141682268090A517141682268090C0D
:1071B000917141682268090ED1718168226811724B
:1071C00081682268090A517281682268090C9172EB
:1071D00080682168000EC87236E0042269466D4856
:1071E0000095FAF7FFFF21680098042208700098C4
:1071F0002168000A487000982168000C8870009887
:107200002168000EC87069466348FAF7EBFF2168F1
:10721000009808712268010A51712268010C000E61
:10722000917121680422C87169465C48FAF7DAFF57
:107230002168009808722268010A51722268010CC4
:107240009172010E2068C17202207071F5810020D8
:10725000F8BDFFE77279022A0FD1F289624504D2A4
:1072600023689B5C0370501CF081F089604504D159
:10727000F58101200870032070710120F8BD38B538
:1072800003F007023F4C00253F4BDDF810C0012AF8
:1072900002D0022A4FD04CE0022058714048DD81D4
:1072A00001683A4A91421ED14168226811704168D2
:1072B0002268090A517041680A0C21688A70416885
:1072C0002268090ED1708168226811718168226874
:1072D000090A517181682268090C917180682168DE
:1072E000000EC87125E00422694610460095FAF7A1
:1072F00079FF216800980422087000982168000A2C
:10730000487000982168000C887000982168000E71
:10731000C87069460820FAF765FF2168009808716F
:107320002268010A51712268010C000E91712168D6
:10733000C871002038BD5A79022A0FD1DA89624516
:1073400004D22468A45C0470501CD881D88960459C
:1073500004D1DD810120087003205871012038BD5F
:107360002DE9F04F85B0934603F00702DFF818903F
:10737000DDF838C0012A15D013F0070F19D0022A02
:1073800076D070E0BCAE1100E805002054464953A9
:107390009C16002068C001006CC0010070C0010094
:1073A00084160020022089F805000020A9F80E00AC
:1073B00059E0002440274FF001081BF0010F28D0AE
:1073C000BA46042203A95046FAF70CFF042201A989
:1073D0004820FAF707FFFB490398884240D10198FB
:1073E0000025B5EB900F10D20AEB85000422694608
:1073F000FAF7F8FE0098032D044408BF06466D1CFA
:107400000198B5EB900FEFD304B93446B8F1000FF3
:1074100026D01BF0020F1DD00020042202A9FBF78A
:107420002FFAE949029888421AD10025B5EB970F47
:107430000DD2A80004226946FBF722FA0098062D17
:10744000044408BF06466D1CB5EB970FF1D3002C22
:1074500008BF3446B8F1000F18BFC9F82C4002D15C
:107460000020C9F82C0005B00020BDE8F08FFFE730
:1074700099F80520022A1AD1B9F80E2062450AD2DD
:10748000C2F10303D9F82C40DB0024FA03F30370A4
:10749000501CA9F80E00B9F80E00604507D1002075
:1074A000A9F80E0001200870032089F8050005B036
:1074B0000120BDE8F08F10B503F00700012804D1CA
:1074C000002211461E2001F066FF002010BD70B59D
:1074D000044603F00700BD4D0E46012804BF0020FE
:1074E000E88119D013F0070F02D0022816D013E05C
:1074F000E889B74B03283CBF19680A54401C80B286
:10750000E881032808D1186890F9022090F9011049
:1075100090F90000FCF7B3FE002070BDFCF7F8FD09
:107520000246E88930B101280AD002280ED003288B
:1075300012D018E014211046FCF7F3FD207012E081
:1075400015211046FCF7EDFD20700CE016211046C9
:10755000FCF7E7FD207006E017211046FCF7E1FD7F
:10756000207001203070E889401CE881012070BD46
:1075700013F0070F04D003F00702022A05D002E03F
:1075800092490020C88100207047924A1268027018
:1075900001200870704730B403F007030024DFF8BF
:1075A0002CC2029A012B02D0022B0BD007E005203F
:1075B0008CF80500ACF80E4020208CF8060030BC9A
:1075C000002070479CF80530052B14D1BCF80E3014
:1075D000934205D29CF806500570581CACF80E007A
:1075E000BCF80E00904206D1ACF80E4001200870A5
:1075F00003208CF8050030BC012070472DE9F043D2
:1076000083B003F00705724E704FDDF828C04FF0CD
:107610000008012D0AD013F0070F3B46DB8903F168
:107620000104A4B211D0022D22D01DE001A96846A8
:1076300002F0BAF805207871316801980870316855
:1076400000984870A7F80E800EE0634502D23068BB
:10765000C254FC81F889604506D1A7F80E803068D5
:107660000178407802F097F803B00020BDE8F0837D
:107670007A79052A0ED1634503D23268D25C027052
:10768000FC81F889604505D1A7F80E8001200870BB
:107690000320787103B00120BDE8F08370B503F0DA
:1076A00007000024494D4A4EDDF810C0012803D0E0
:1076B00013F0070F06D043E0EC81306804703068A7
:1076C00044703DE0E889604503D233681A54401C99
:1076D000E88180B2604533D13FA001220068EC818F
:1076E0000A703168C2B20978914229D13168C0F379
:1076F00007204978814223D11C2600244FF48015AD
:1077000005EB0430FAF7ECFE022808BF70BD601CE0
:10771000C4B2B442F4D3032600244FF48E1505EB13
:107720000430FAF7DDFE022808BF70BD601CC4B249
:10773000B442F4D32948FAF7D3FE022808BF70BD3B
:10774000002070BD10B503F00700012808BF02F04B
:107750000BFB002010BD70B503F007041B4D012C7E
:1077600009D013F0070F2B46D3F82CC0DB8908D0C3
:10777000022C17D014E00020E88105F0CCF8E86274
:107780000EE0002B04BF1002E86206D0012B04D1EA
:107790004CEA0200E86205F0B7F8E889401CE8818D
:1077A000002070BD002B04BF4FEA1C21017005D0E2
:1077B000012B03D180F800C001200870581CE8811B
:1077C000012070BD5446435354464953E8050020F8
:1077D000BCAE11007005002055AC000000FE110089
:1077E00070B5064603F00700FB4C0D46012808BFA4
:1077F00000200DD013F0070F02D002280BD008E0B4
:10780000E089002804BF104610F0BAFDE089401C52
:10781000E081002070BD10F0B0FD307001202870B4
:1078200070BD70B503F0070CEB4D0E460446BCF17D
:10783000010F06D013F0070F07D0BCF1020F17D0CD
:1078400014E00020E881288210E0E889002804BFC5
:107850001002E86207D0012805D1E86A1043E86207
:1078600080B2FDF726FCE889401CE881002070BD4D
:10787000288A02280CD2FEF734FC2A8A002A04BF88
:10788000000A207004D0012A02D12070012030703B
:10789000288A401C2882012070BD10B513F0070F04
:1078A00004D003F00702022A08D005E0002A14BF22
:1078B0000120002009F011F8002010BDC74A92F8FD
:1078C0005420D20802700120087010BD00207047BB
:1078D00070B503F007020026C14CBF4DDDF810C0A3
:1078E000012A02D0022A15D012E005F06FFC2168AF
:1078F0000870FDF775F82168487003F033FB2168C4
:107900008870FDF770F82168C87005206871EE81F5
:10791000002070BD6A79052A0FD1EA89624504D238
:1079200023689B5C0370501CE881E889604504D1A2
:10793000EE810120087003206871012070BD70B5D0
:10794000064603F007000D4602281CBF002070BD4C
:1079500001F03BFD002814BF0124002401F038FD94
:10796000002814BF02220022224332700120287016
:1079700070BD30B403F00703994A0024964DDDF83A
:1079800008C0012B02D0022B4AD046E09549086876
:10799000954B98422FD14868B0F5887F2BD8C8689E
:1079A000FF282EBFFF20C868C0B21368187008698E
:1079B000FF283ABF0869C0B2FF20136858704869B1
:1079C000FF283ABF4869C0B2FF20136898708868E2
:1079D0001368000AD8708869136818718869136879
:1079E000000A58718869030C1068837188691168EE
:1079F000000EC87110E010680470106844701068C0
:107A000084701168FF20C87011680871116848718E
:107A1000116888711168C871EC8130BC0020704712
:107A2000EB89634504D21268D25C0270581CE8816D
:107A3000E889604502D1EC810120087030BC01204A
:107A400070472DE9F04103F007010025624C06461E
:107A5000012904BFE561E58101D0022902D000209F
:107A6000BDE8F081207F5E4F00F00701E1812078C2
:107A7000084304D1386802F0F7F901202070E18949
:107A8000052928BF25703868405C3070E069401CCB
:107A9000E0610120BDE8F08170B503F00702002528
:107AA0004F4B4D4CDDF810C0012A02D0022A08D0FD
:107AB00005E0186802F0D8F905206071E581002022
:107AC00070BD6279052A0FD1E289624504D21B6834
:107AD0009B5C0370501CE081E089604504D1E58126
:107AE0000120087003206071012070BD70B503F0A3
:107AF00007020025384C012A02D0022A11D00EE0DC
:107B0000052060710021E581084601F04DFE4FF629
:107B1000FF7101EA4000608201F052FEA061002086
:107B200070BD6279052A16D1E289B4F812C06245A7
:107B300007D212F0010F1CBFA37903700DD0501CA7
:107B4000E081E089604506D1E581012008700320CD
:107B5000607101F043FE012070BDA66922F00103AF
:107B6000F35A1E0A0670A371E9E77FB51C460E465C
:107B7000054613F0070F08D103F030FB28B10122AE
:107B800002A91F2001F007FC03E004F0070002280F
:107B900002D004B0002070BD01F0DFFE287001208B
:107BA000307004B070BD2DE9F04103F007020027EA
:107BB000094E88460546012A02D0022A16D007E05F
:107BC00005207071F7810A20708201F0F9FDB06123
:107BD0000020BDE8F0810000E80500208C100020A6
:107BE000BCAE1100A81600205443524670790528F7
:107BF00018D1F289708A824208D212F0010F1CBF9C
:107C0000B079287010D0F089401CF081F089718A19
:107C1000884207D1F781012088F8000003207071A5
:107C200001F0DCFD0120D4E7002401F096FE0128DC
:107C300004D1F089B16920F001000C5A200A2870A3
:107C4000B471E0E77FB50D46044613F0070F04D08A
:107C500003F00700022808D004E0012202A90A204C
:107C600001F099FB04B0002070BD05F0AFFA207060
:107C70000120287004B070BDF8B503F0070200259C
:107C8000FF4C0E460746012A02D0022A0ED00BE016
:107C90000520607103F0B7FC206300281ABF44F28E
:107CA0006440A082A582E5810020F8BD60790528A6
:107CB00022D1E289A08A6946824214D212F0030FCF
:107CC00008D10422206BFAF78DFA0098E062206B4D
:107CD000001D206394F82C003870E06A000AE0620E
:107CE000E089401CE081E089A18A884204D1E581D5
:107CF00001203070032060710120F8BD10B513F031
:107D0000070F04D003F00702022A0DD00AE0012A6F
:107D100005D0002A04BF0120FBF78DF802E0012006
:107D2000FBF77EF8002010BDD64A1268126802F0F8
:107D3000020202700120087010BD70B50D460446A5
:107D400013F0070F04D003F00700022808D005E065
:107D5000002A14BF0120002001F0E8FF002070BDC0
:107D600001F0EBFF002814BF012200222270012045
:107D7000287070BD70B503F00700C14D144601288E
:107D800008BF002016D013F0070F14D1E88900288F
:107D900008BFAA710CD001280AD1A879FBF77DF899
:107DA000A8792040FBF73CF8A879A043FBF743F8FB
:107DB000E889401CE881002070BD2DE9F00103F046
:107DC0000704AF4E059F012C04BF0020F08135D081
:107DD00013F0070FAA4BAC4DDB8903F1010C1FFA1E
:107DE0008CFC02D0022C2DD028E0A8490868C2548F
:107DF000781E834220D10868007830B101280AD06B
:107E000002280ED0032812D016E0086829684078AE
:107E100081F8800110E008682968407881F88101C4
:107E20000AE008682968407881F8820104E008685F
:107E30002968407881F88301A6F80EC0BDE8F001FA
:107E400000207047904A126813B1012B0AD014E049
:107E500092F8801101F00F0392F8811163F31F1162
:107E600001700AE092F8823192F8832103F00F0347
:107E700063F31F12027001200870A6F80EC0BDE85F
:107E8000F0010120704710B4DFF804C213F0070FAF
:107E900004D003F00702022A18D014E0012A01D00E
:107EA0004AB110E0DCF80000806ADCF8001020F035
:107EB0000300886207E0DCF80000806ADCF800104C
:107EC00040F00300886210BC00207047DCF80020FE
:107ED000926A02700120087010BC704770B503F000
:107EE00007000025664C0E46012806D013F0070F48
:107EF00004BF6079022805D019E002206071E58195
:107F0000E56214E0E089A18A884207D261481146FF
:107F10000068FBF702FCE089401CE081A18A80B286
:107F2000884204D1E5810120307003206071002077
:107F300070BD2DE9F04103F007020025504C0E46BC
:107F40000746012A02D0022A06D002E00220607110
:107F5000E5810020BDE8F0816079022814D1E18933
:107F6000A08A814207D24B480068FBF704FC3870B6
:107F7000E089401CE081E089A18A884204D1E58142
:107F800001203070032060710120BDE8F08110B540
:107F900003F007023A4C012A02D0022A27D024E03B
:107FA00003F034FB0023002804BF2363A3821BD00B
:107FB00000F1540121634168B1F5887F90F82010E9
:107FC0000CD390F8212001EB020C01FB02C190F8C8
:107FD000222090F823001044084404E090F8220086
:107FE0000A1801FB0020A082E381002010BDE28975
:107FF000A38A9A4207D2D4F830C01CF802C080F895
:1080000000C0501CE081E089984204BF0120087044
:10801000012010BD10B513F0070F04D003F00702C4
:10802000022A05D002E0104601F0E5FB002010BD59
:10803000194A127802700120087010BD1FB513F0A4
:10804000070F04D1012202A9092001F0A4F904B00C
:10805000002010BD70B503F007000949012804BFD6
:108060000020C88130D013F0070F2DD1C889074CEC
:1080700003283CBF23681A54401C80B2C8810DE01D
:10808000E805002080AE1100F8060020BCAE11000B
:1080900088AE1100A4AE11002D060020032813D1D4
:1080A000F8F7A9FF2068B0F8010045BAF8F7B8FD65
:1080B000040018BFF9F71CF929460020F8F708FD5D
:1080C000002C18BFF9F716F9002070BD70B503F049
:1080D0000700F749012804BF0020C88124D013F00D
:1080E000070F21D1C889F34D02283CBF2B681A54D1
:1080F000401C80B2C881022816D1F8F77CFFF8F73F
:108100008FFD040018BFF9F7F3F82868007818B15C
:1081100028684078F8F7E0FC28684078F8F7DCFC3D
:10812000002C18BFF9F7E6F8002070BD13F0070F18
:1081300004BFDF48C270002070477FB50D4604467B
:1081400013F0070F04D003F00700022808D004E062
:10815000012202A9102001F01EF904B0002070BD18
:1081600004F0C1FF002814BF012200222270012068
:10817000287004B070BD7FB50D46044613F0070F9C
:1081800004D003F00700022808D004E0012202A96D
:10819000112001F000F904B0002070BD04F094FF3C
:1081A00020700120287004B070BD10B503F00700E6
:1081B000DFF8FCC20299012804BF0020ACF80E00D1
:1081C0001AD013F0070F17D1BCF80E00B94B0328D3
:1081D0003CBF1C682254401C80B2ACF80E008842A0
:1081E0000AD118681968B0F80100097840BA00B2DD
:1081F000002908BFFCF75AFF002010BD10B503F09E
:108200000700DFF8ACC20299012804BF0020ACF8D7
:108210000E0017D013F0070F14D1BCF80E00A54BB9
:1082200003283CBF1C682254401C80B2ACF80E00EE
:10823000884207D11868B0F8010041BA1868007880
:10824000F9F7DDFB002010BD70B503F00702984C74
:10825000DDF810C0012A02D0022A07D004E0002075
:10826000E081FBF7ADF8E062002070BDE289624575
:1082700006D2C2F10303E56ADB0025FA03F30370BB
:10828000501C80B2E081604504BF012008700120CD
:1082900070BD70B5044603F0070C0020844DBCF19E
:1082A000010F06D013F0070F07D0BCF1020F13D057
:1082B00010E0E8812882A8710CE0E889002808BF56
:1082C000AA7104D001227C49122001F064F8E889E7
:1082D000401CE881002070BD2A8A3AB1207001203C
:1082E0000870288A401C2882012070BD04F0C6FF57
:1082F0002070F6E770B50D46044613F0070F04D062
:1083000003F00700022805D002E010460AF0F6FF4D
:10831000002070BD0AF0F5FF20700120287070BDAC
:1083200010B5144613F0070F10D1032C0ED8634973
:1083300003200968C86102217F20F8F785F806202C
:1083400040EA041140F21620F8F77EF8002010BD34
:1083500010B513F0070F4FF0010404D003F007022B
:10836000022A56D053E0122A51D2DFE802F0090E59
:10837000122A2A2A2A2F3235383B3E405044474C95
:108380004F4900200968087741E04D4800680477AC
:108390003DE04A4903200968C86101217F20F8F7C0
:1083A00053F815214FF48770F8F74EF875214FF404
:1083B0008470F8F749F84D214FF48570F8F744F8C8
:1083C00025E00021D01E04F09BFF20E0F9F7EAFD34
:1083D0001DE0F9F704FE1AE0F8F73FFF17E0F8F7A1
:1083E000F8FD14E001F040FE11E0012000E0022061
:1083F00004F094FE0BE0FDF711FE08E03049022086
:108400000968088603E02E490020096808860020D4
:1084100010BD274BDFF8ACC0DA8912B1012A05D0B4
:1084200009E0DCF80010090A017004E0DCF800C083
:1084300080F800C00C70501CD881012010BD70B5B0
:10844000144613F0070F5DD103201C49072C11D8E7
:108450000968C86102217F20F7F7F6FF0A2040EA89
:10846000041140F20220F7F7EFFF04F188014FF406
:10847000017019E0A4F10805042D2BD80968C86122
:1084800001217F20F7F7E0FF052D3BD2DFE805F063
:10849000030507091C00362104E0402102E04A21BF
:1084A00000E054214FF48470F7F7CEFF2AE000007B
:1084B000E8050020BCAE1100EE0500208CAE1100D6
:1084C000F80600206C0700205E214FF48470F7F757
:1084D000BBFF17E0A4F10D02022A13D80968C86196
:1084E00001217F20F7F7B0FF0D2C08BF13210BD01F
:1084F0000E2C04BF18214FF48770D5D00F2C08BF65
:108500001D2101D0002070BD4FF48770CCE77FB5EE
:108510000C46054613F0070F04D003F007000228AD
:1085200008D004E0012202A9062000F034FF04B0C4
:10853000002070BDFCF754FA022808BF00200BD0C1
:10854000032808BF022007D0042808BF032003D057
:10855000052814BFFF20012028700120207004B0DE
:1085600070BD10B5104613F0070F08BF04F010FEE1
:10857000002010BD10B5104613F0070F08BF04F01F
:1085800013FE002010BD70B5044603F007000D4631
:1085900002281CBF002070BD04F013FE20700120D3
:1085A000287070BD70B403F007020024F84BDDF8AA
:1085B0000CC0012A05D0022A04BF5A79022A0AD027
:1085C0001BE002205871F348DC816FF07F410068A6
:1085D000081AD86211E0DA89624506D2DE6AD5004F
:1085E00026FA05F50570501CD881D889604504D15C
:1085F000DC81012008700320587170BC0120704795
:1086000013F0070F04BFE44802700020704710B554
:10861000944603F00700DE49029A012804BF0020B7
:10862000C88112D013F0070F0FD1C889DB4B9042DD
:108630003CBF1C6804F800C0401C80B2C881904256
:1086400003D10E20196800F0A6FE002010BD70B501
:1086500003F00704CE4D012C0AD0AC4613F0070FEF
:10866000BCF81230DCF830C006D0022C21D01EE05D
:108670000020E88128821AE0E889002808BF2A63E0
:1086800012D0012804BF501C68820DD0022816BFEA
:10869000C11EAA82994207D2297D0844C01EC1B2D8
:1086A0000CF0FF00F9F775FBE889401CE881002019
:1086B00070BDFF22027093B12A8A9444521CBCF50B
:1086C000807F0BD20CF5801C0CF5F83C9CF800C0A8
:1086D00080F800C09A4204BF012008702A8201205D
:1086E00070BD2DE9F04103F007050026A84C944623
:1086F000012D04BFE681268224D013F0070FA44B7E
:108700005A8A1B6B02D0022D28D01BE0E08900287A
:1087100008BFC4F830C012D0012816D09F49801E6F
:1087200090423CBF0D6805F800C0401C904206D145
:1087300003F58010096800F5F830FAF74FF9E08981
:10874000401CE0810020BDE8F0810CF10100608256
:108750001844B0F5807F88BF6682F0E74FF0FF0CC9
:1087600080F800C09AB1258A03EB050C6B1CBCF5A0
:10877000807F0BD20CF5801C0CF5F83C9CF800C0F7
:1087800080F800C0934204BF0120087023820120BA
:10879000BDE8F08110B5944603F007007C49029AC9
:1087A000012804BF0020C88112D013F0070F0FD199
:1087B000C8897A4B90423CBF1C6804F800C0401C3A
:1087C00080B2C881904203D10220196800F0E3FD15
:1087D000002010BD10B5944603F007006C49029AC2
:1087E000012804BF0020C88112D013F0070F0FD159
:1087F000C8896A4B90423CBF1C6804F800C0401C0A
:1088000080B2C881904203D10320196800F0C3FDF3
:10881000002010BD70B5044603F007005C4D0E4605
:10882000012804BF0020E88140D013F0070F02D0D8
:1088300002283DD03AE0E889584C002804BF21685E
:108840000A7021680978012901D039B123E0002894
:1088500018BF06283CBF21680A541CE00FF0C6FD73
:108860002168000948700FF0CDFDC0F303260FF01A
:10887000BDFD216846EA001088700FF0C3FD216835
:10888000C8700FF09BFD216808710FF09DFD2168F5
:1088900048710520E881E889401C80B2E8810628FB
:1088A00004D106220F20216800F075FD002070BD64
:1088B0000FF0ABFD0246E889002808BF100E10D06B
:1088C000012808BF100C0CD0022808BF100A08D0DD
:1088D000032808BF22700ED0042804D0052805D034
:1088E00009E0207007E00FF069FDFAE70FF06CFD7A
:1088F000207001203070E889401CE881012070BDA3
:1089000013F0070F05D003F00700022804BF012071
:108910007047002070471FB513F0070F04D10122E4
:1089200002A9132000F037FD04B0002010BD03F0B1
:108930000701DFF85CC00098012907D013F0070F8A
:1089400004BF9CF80510012909D01FE001208CF814
:1089500005000020ACF80E00CCF8280014E0BCF8AC
:108960000E10814208D2DCF82830491C42EA03226A
:10897000CCF82820ACF80E1089B2814206D1032031
:108980008CF80500DCF82800CCF830000020704797
:10899000E8050020A005002032050020BCAE110033
:1089A00003F00700FF494FF0010C012806D013F037
:1089B000070F04BF4879012807D014E081F805C0EB
:1089C0000020C881087148620DE0C889002804BFF2
:1089D0000A71A1F80EC006D0012806D00323022890
:1089E00018BF4B7106D00020704710024862022069
:1089F000C881F8E7486A104348624B71F3E770B5E5
:108A0000154613F0070F19D1E64C20462179406A2C
:108A100003290DD8E44A1268D161C0F307217F20F1
:108A2000F7F712FD94F824002946F7F70DFD05E04D
:108A3000C3B2081FC0B21946F9F7ABF9002070BDE8
:108A400070B5044603F007000D4602281CBF002045
:108A500070BDD448D3490079496A032803D889B244
:108A6000F7F7A6FC04E0001FC9B2C0B2F9F752F94B
:108A700020700120287070BD03F00701C94801294A
:108A800004BF0021C18103D013F0070F08BF827219
:108A900000207047F8B503F007020023C34EC14F12
:108AA000012A02D0022A24D021E0002402200093CF
:108AB0007871FB81B87A4FF44835834217DA042283
:108AC00069462846F9F78EFB3168009808553168E9
:108AD00000982144000A48700098000C88700098A3
:108AE000000EC870B87A241D2D1D8442E7DB0020DB
:108AF000F8BD7A79022A15D1FA8997F80AC0624539
:108B000007D2D6F800C01CF802C080F800C0501C84
:108B1000F881F889BA7A904204D1FB81012008706B
:108B2000032078710120F8BD10B503F007009D49BE
:108B3000012804BF0020C88118D013F0070F15D1F9
:108B4000C88991F80AC0994B604505D2D3F800C096
:108B50000CF80020401CC8818A7A80B2904205D16E
:108B60008A7A4FF448301968F9F738FF002010BDB1
:108B70001FB513F0070F04D1012202A90D2000F048
:108B80000AFC04B0002010BD13F0070F04BF854895
:108B9000427200207047F8B503F007020027834EA9
:108BA000DFF800C2012A02D0022A2DD02AE09CF868
:108BB0000900002400EB40004FF4443101EB002594
:108BC000022000978CF80500ACF80E704FF410707E
:108BD000ACF81400042269462846F9F703FB316813
:108BE00000982D1D0855316800982144000A4870EE
:108BF0000098241D000C88700098000EC870B4F511
:108C0000107FE7DB0020F8BD9CF80520022A16D172
:108C1000BCF80E20BCF814309A4205D23468A45C2B
:108C20000470501CACF80E00BCF80E00984206D13F
:108C3000ACF80E700120087003208CF805000120AC
:108C4000F8BD70B54FF444324FF4407101FB00247D
:108C50000120F7F7F8FFFDF7E1F9FCF723F80546E7
:108C6000F8F7FBFA4F4B4FF4107220461C639A82C0
:108C70002946BDE87040F9F7B1BE03F00701DFF8FF
:108C800024C10098012907D013F0070F04BF9CF8F6
:108C90000510022909D01FE002208CF805000020F1
:108CA000ACF80E00CCF82C0016E0BCF80E10814297
:108CB00008D2DCF82C30491C42EA0322CCF82C20E4
:108CC000ACF80E1089B2814206D1BCF82C00ACF889
:108CD000140003208CF805000020704770B503F0E5
:108CE000070000252F4C0E46012806D013F0070F71
:108CF00004BF6079022805D023E002206071E5817D
:108D0000E5621EE0E089A18A884211D2E16A090A7F
:108D100041EA0261401CE162E08110F0030F07D1DB
:108D200004222349206BF9F759FE206B001D2063B4
:108D3000E089A18A884204D1E581012030700320B6
:108D40006071002070BDF8B503F007020025154CD6
:108D50000E460746012A02D0022A05D002E0022070
:108D60006071E5810020F8BD607902282BD1E2898D
:108D7000A08A824215D212F0030F09D1042269465B
:108D8000206BF9F72FFA0098E062206B001D20633A
:108D900094F82C003870E06A000AE062E089401C18
:108DA000E08107E0E80500208CAE1100BCAE1100A8
:108DB00014060020E089A18A884204D1E5810120BF
:108DC0003070032060710120F8BD70B403F0070219
:108DD0000025F74C012A02D0022A06D002E0022028
:108DE0006071E58170BC002070476279022A1CD155
:108DF000E289B4F814C062450FD212F0030F04D117
:108E0000236B53F8046BC4E90B6394F82C300370A4
:108E1000E06A000AE062501CE081E089604504D10C
:108E2000E581012008700320607170BC012070474B
:108E300030B403F007000024DFF874C3012807D022
:108E400013F0070F04BF9CF80500022808D025E0A6
:108E500002208CF80500ACF80E40CCF82C401DE048
:108E6000BCF80E00BCF8143098420CD2DCF82C5040
:108E70002D0A45EA0262401CCCF82C20ACF80E000A
:108E800010F0030F0DD0BCF80E00984206D1ACF8DC
:108E90000E400120087003208CF8050030BC002033
:108EA0007047DCF83000B0F5002F28BF0260001DCD
:108EB000CCF83000E7E730B403F007040025DFF812
:108EC000F0C2012C08BFACF80E5033D013F0070FDE
:108ED00002D0022C31D02DE0042A08BF4FF42C30F0
:108EE00026D012DC002A08BF4FF4801020D0012ABF
:108EF00008BFB0481CD0022A08BF4FF48E1017D00C
:108F0000032A08BFAC4813D00FE0052A08BFAB48BE
:108F10000ED0AB48102A00680AD0112A08BFA94811
:108F200006D0202A08BFB43002D0CCF8285001E087
:108F3000CCF8280030BC00207047BCF80E20042A72
:108F400007D2C2F10303DCF82840DB0024FA03F364
:108F50000370501C80B2ACF80E00042824BF01201E
:108F60000870012030BC704710B503F007000128DD
:108F700004D1002211460C2000F00DFA002010BD93
:108F80002DE9F04103F0070C894E069D0F4604467B
:108F9000BCF1010F04BF0020F08117D0844913F009
:108FA000070FCB8903D0BCF1020F12D00EE0864927
:108FB000022B3CBF0868C254581C80B2F081A84202
:108FC00004D102220968052000F0E5F90020BDE87F
:108FD000F08113B1012B04D008E0FBF701FD2070F4
:108FE00004E0FBF700FD207001203870F089401C80
:108FF000F0810120BDE8F08170B503F007006C4DF1
:10900000012803D013F0070F05D024E00020A86248
:10901000E862A8711EE06649EC8991F806C0886A8A
:109020000CEB0201CBB2022C03D242EA0020A86270
:1090300006E05F49042CC96A04D242EA0120E862D2
:10904000AB7105E0052C03D2624508BF00F0D4FFE8
:10905000E889401CE881002070BD10B503F00701CD
:109060001046012905D013F0070F08BF00F059F989
:1090700004E04F49002088628871C881002010BD3B
:1090800010B5104613F0070F08BF00F04AF9002092
:1090900010BD70B5032600244FF48E1505EB043087
:1090A000F9F71EFA022808BF70BD601CC4B2B442B2
:1090B000F4D3012070BD30B403F007030024DFF8BF
:1090C000F0C0029A012B02D0022B0CD008E0052040
:1090D0008CF80500ACF80E409CF808008CF80600EF
:1090E00030BC002070479CF80530052B14D1BCF82B
:1090F0000E30934205D29CF806500570581CACF80F
:109100000E00BCF80E00904206D1ACF80E400120D3
:10911000087003208CF8050030BC012070472DE951
:10912000F0472AA0DDF820C0006803F007050027FB
:109130001F4E254C012D03D013F0070F06D034E04D
:10914000F78120680770206847702EE0F389634537
:1091500003D22568EA545A1CF281F289624524D16F
:10916000F7814FF0010881F800802168C2B20978C8
:1091700091421AD12168C0F307204978814214D165
:10918000032500244FF48E1909EB0430F9F7A8F9F0
:10919000022804D0601CC4B2AC42F5D3404601287A
:1091A00006BF86F80880F77137720020BDE8F087A7
:1091B000E805002000FE110000F8110000F0110089
:1091C000F80600208C100020BCAE110055AC000049
:1091D0002DE9F0414FF0000C03F00700634E644CA2
:1091E0006546012803D013F0070F0CD068E06570C6
:1091F000A5812562A570002046F82050401CC0B211
:109200004028F9D35CE0607805283CBF401C6070C2
:10921000C0B2012808BF100222D055490228CB8ACB
:1092200008BF98181CD024BFA1898B4248D9514F40
:1092300001F0030001F101083A54A7F134004FF4A2
:109240008E12006A984502EB002008BF002109D168
:10925000491CC9B20429FBD34449F9F7E2F926E0D5
:10926000E0822DE0032232EA010120D17A5CCB00BA
:109270009A40491CC9B242EA0C0C0429F6D3A178E1
:1092800001F03F02491CC9B246F822C0A170402932
:109290000DD13649F9F7C5F9A570206A401C206246
:1092A000002046F82050401CC0B24028F9D3A089C5
:1092B000401C80B2A081E18A884204BF0120E07195
:1092C0000020BDE8F08110B503F00700DFF8A0C072
:1092D0000299012804BF0020ACF80E001FD002281C
:1092E00004BF012010BD13F0070F18D1BCF80E0009
:1092F000214B88423CBF1C682254401C80B2ACF811
:109300000E0088420BD118684178408840BA61F35A
:109310001F401968097840EA01600FF028F8002022
:1093200010BD10B5124C2146E2898B6A8979022A58
:1093300005D240EA03220844A262A07112E0B2F50D
:10934000817F08D20C490968114401F8020CA17907
:109350000844A07106E008BF884203D103491846BB
:1093600000F064FEE089401CE08110BD283400203C
:10937000E80500201C060020BCAE1100F5480021C5
:1093800001704170C1700171F34A08461154401CCC
:109390000428FBD3704710B4EE4C6378002B1EBF3B
:1093A000002010BC7047E07022710020002A88BFA6
:1093B000E94B06D911F800C003F800C0401C8242F6
:1093C000F8D80120607010BC7047E24840787047C0
:1093D000E04880787047DF4900208870704770B59A
:1093E0000024FAF7B6FADB4D6878012806D100F0C0
:1093F00012F804462020E87000206870FBF7F0FAAD
:10940000022802D101F0A6FE18B9002C04BF0020EA
:1094100070BD012070BD2DE9F05FCE480024012110
:109420008170C078A046202880F08D81DFE800F0B0
:10943000131F363F104BF04FCAB2B8BDFC2DEEEDF6
:10944000CBD9DEE3CACACACACACACACACACAECEBFC
:10945000FBF728FB16E0FBF7C3FABE4C6071A01DBA
:1094600001780120FBF7CEFA0120A0700AE0BA488B
:10947000007802F0C5F801210320FBF7C3FAB549D3
:1094800001208870012400F05EB9B24880F80180A4
:10949000801D0078FFF7D5FB00F055B9AE48417844
:1094A000007841EA002003F0A4FC00F04CB9AA487F
:1094B000007803F0A3FC04210320FBF7A3FAA549DD
:1094C00001208870DEE7A44841780078A9E0DFF841
:1094D00088B200264FF0010AABF10609012789F88E
:1094E00002A089F8018099F80000E8BB9BF80050C1
:1094F00089F800A015F0100F17D00120F7F7A3FB93
:109500000020F7F71AFCFBF76EFA70B3F8F76CF867
:10951000FF210F20FBF7F1FD074645F00105002074
:10952000F7F7EBFB0120F7F708FC15F0010F1FD050
:10953000FAF74AFB0020FAF7CFFD0120F7F783FB8B
:10954000FAF79CFC01460220FBF758FC0220FBF7CF
:1095500033FCF7F782FEFAF791FCFAF7A0FDFAF771
:109560008DFC4FF4906101E004E00CE010F086F90E
:1095700089F8008089F80280002F1CBF761C032E1A
:10958000ACDB00F0E0B8F8F72FF8FF210F20FBF775
:1095900050FEC1E770480078401E01F045FD71E7BC
:1095A0006D48007803F017FE6CE76B4800780028E0
:1095B00004BF0021032003D003F0AAFD01460220CE
:1095C000FBF720FABFE0644D2878002818BF01207F
:1095D00003F07FFD2878002818BF012000F08EFDE1
:1095E000B1E05D48007803F065FD4BE75A4800782C
:1095F00003F004FEA7E05848007850B1012855D088
:1096000002280AD09FE09AE08FE074E062E00BE06D
:109610004DE05248F8F7ECFE95E001F01CFE002109
:109620000420FBF7EFF92DE74A4880F80180002677
:10963000354672B6F9F780FF48B1FAF73BF80646AF
:10964000FAF718F8FAF73CF80546FAF723F8F7F7AF
:10965000D2FCF7F7E5FA8146F7F7E1FEF9F7A2FE4B
:10966000070018BFF9F79DFE4FF41870F9F775FE63
:1096700062B63B48C0F80080F8F729FB72B6B9F132
:10968000000F03D0F7F7B7FCF7F7E7FDF9F754FF42
:1096900038B1002E18BFF9F751FF002D18BFF9F7A8
:1096A0008CFF002F18BFF9F77AFE62B64BE02A480C
:1096B0000078012804BF02210520B2D0022804BF8F
:1096C00000210320ADD0032819BF02210846002144
:1096D0000420A6E720480178427841EA02218278F6
:1096E000C078120442EA006041EA000262210720C9
:1096F00003F017F927E0184D28780EF068FE687817
:10970000A978000140EA11100EF067FEE878A97808
:1097100001F00F0140EA01200EF06BFE28790EF0F7
:109720004AFE68790EF04DFE0DE0F8F772FC01205C
:10973000F7F789FAFAF7DEFDF7F78FFDA2E606489C
:10974000007800F0F6F8034880F802802046BDE873
:10975000F09F0000200600202606002000FE1100D9
:109760006405002002460020022928BF704752B13C
:10977000012A18BF704701EB810000EBC100FD49D1
:1097800001EB0010704701EB410000EBC100FA490A
:1097900001EBC010704700FB01F2B2F5307F9CBFB7
:1097A000F64AC2E9020170470028F44A926818BFDD
:1097B0000260F2480029C06818BF08605043704733
:1097C000EE4801210171007880F0010000EB4001BA
:1097D00001EBC000E84901EBC0107047E748827810
:1097E000002132B1C27822B9027882F001020270FF
:1097F000817001717047E14910B54C7848701E289E
:1098000008BF002008D01F2808BF012004D00E2860
:1098100008BF812002D000E00870012003F0EEFCB8
:10982000204610BDF0B4D54E96F800C0B5680CEBDC
:109830004C0404EBCC0CD04C8D4204EBCC1C03FB51
:1098400005F40CEB440C34BF2C460C46F768FE1AAA
:10985000964228BF16461A44974224BF0023002E82
:109860009CBFF0BC70470022002C06D930F8127063
:109870002CF81270521C9442F8D85B1C0CEB450C6F
:1098800000EB4100B342EED3F0BC70472DE9F0414C
:10989000BA4F14468C4601467A7806981D468A428D
:1098A00018BFBDE8F0810121F970012802D002281B
:1098B00025D02AE03878BE6800EB400101EBC000FB
:1098C000AD49A64201EBC01134BF32462246F868CA
:1098D000A84238BF05460023002D16D90020002AD3
:1098E00006D91CF8007021F81070401C8242F8D88C
:1098F0005B1C01EB4601A444AB42EFD305E000231F
:109900002A4621466046FFF78DFFBDE8F04100F092
:10991000E9B910B5002808BF10BD01229749CA70E7
:10992000497800230821FFF77DFFBDE8104000F0D3
:10993000D9B9924A01281146D071497808D0002837
:109940000CBF2429704730205070012003F056BC12
:1099500024205070012003F051BC8848C079704722
:1099600070B4DFF81CC2DCF800C0DCF818C01CF0D2
:10997000040F1ABF012424EA0C060CF00106056846
:109980000C68002E1CBF1B1B5C1E1CF0020F1CBFB2
:10999000521B551E1CF0040F19BF04600D600560BA
:1099A0000C6070BC704710B5002808BF10BD0122C4
:1099B0007249CA704A787349DFF8CCC102220B7829
:1099C0009CF80010FFF72EFFBDE8104000F08AB9A8
:1099D0002DE9F04369498BB00122CA706B4A49787E
:1099E0001578684A2529147824BF0BB0BDE8F083A8
:1099F000DFE801F0134D4D4D134D4D4D4D4D4D4D87
:109A00004D4D4DFD4D5555554DFDFDFDFDFDFDFDEE
:109A1000FD4DFDFDFD7C7CFD8400002800F00081F3
:109A200006460027F7F70AFD5FEA000C16D05349F7
:109A300008788F6800EB400202EBC0004E4ABD423E
:109A400002EBC01094BF2B463B46C968A14238BF09
:109A50000C460021002C06D800F0E2B83B46224616
:109A60002946304647E00022002B08D91CF9028025
:109A700036F8188020F81280521C9342F6D8491C00
:109A800000EB470006EB4506A142ECD3C8E00028F6
:109A90006FD0002322462946FFF7C4FEC0E03C48B1
:109AA0000078012884BF3B480478F7F765FB10F085
:109AB000020F18BF641CFBF7F5F8002205FB04F346
:109AC000002BC4BF2D4CDFF8B0C052DD10F8015B95
:109AD000217801EB410606EBC1010CEBC11121F825
:109AE0001250511C8AB29342F0DC99E0002840D019
:109AF0000023A21C2946FFF795FE91E0002838D0EC
:109B000006461F480068007E10F0040F0EBFA946ED
:109B1000A1462C46A9EB9900A208411E0592069287
:109B20004FEA990000914FEA5902CDE901020391F1
:109B3000A4EB940104906208491ECDE90721099124
:109B400023464A4605A96846FFF70AFF23464A46C8
:109B500005AF06A9E84601A8FFF702FF23464A46DB
:109B600007F1080108F10800FFF7FAFE23464A460C
:109B700012E055E028430020283800202C06002061
:109B8000F8060020BB050020C1050020BA05002012
:109B9000BC050020BE05002007F10C0108F10C00F7
:109BA000FFF7DEFE23464A4607F1100108F11000D8
:109BB000FFF7D6FE58480078002200EB400101EB89
:109BC000C0005649914601EBC01020F8129058F899
:109BD0002210A1F1010C491C61451ED357F8221037
:109BE0004B1E491C994211D303FB05C100E01CE048
:109BF00036F9114030F912108C42C8BF20F81240DB
:109C000057F822105B1C491C9942EDD258F82210DB
:109C10000CF1010C491C6145E0D2521C052AD4D339
:109C20000BB0BDE8F04300F05DB80BB0BDE8F083C9
:109C300039491E288A79887108BF002003D01F285F
:109C400008BF012000D148711046704770B50D461D
:109C500031490122CA70324A49781678314A21299D
:109C600014781EBF2229232970BD002818BF002D9B
:109C700011D0002322463146FFF7D4FD631C012298
:109C800021462846FFF7CEFD05EB4400A31C012228
:109C90003146FFF7C7FDBDE8704000F023B810B5AE
:109CA0001D4C6178002904BF4068FFF791FE607881
:109CB000112804BF0020FFF78BFE6078122804BF34
:109CC0000020FFF785FE6078132803D1FCF766FAC1
:109CD000FFF77EFE60781D2818BF10BD1248BDE852
:109CE000104075E670B5F9F734FB00F0080608205F
:109CF000F9F72AFB084C20790025002801BF2078BD
:109D000080F001002070A5701CBF0120A0703046BB
:109D1000F9F716FBE57070BD2C06002028380020EE
:109D2000BA050020BB05002080640020AF49002850
:109D300014BF0020012008707047AC48007800284C
:109D40000CBF0120002070470120A84948707047CF
:109D5000A64800214170017800291ABF40680028F8
:109D600070470120F9F767B810B5A04C207800289B
:109D70001CBF0120F9F754F800206060A060E0608B
:109D80002061606110BD10B5984C207800281CBF80
:109D90000120F9F745F800206060A060E0602061D4
:109DA000606110BD70B50446F9F7D3FA00F00805FC
:109DB0000820F9F7C9FA8D4A8D490023106901EB93
:109DC000C001401C1061B0F5807F28BF136120786E
:109DD000087060784870A0788870E078C870207942
:109DE000087160794871A0798871E079C87150690B
:109DF000B0F5807F3CBF401C506116D31D20087019
:109E000001204870207888706078C870A078087148
:109E1000E0784871207988716079C871D068401CF9
:109E2000D060B0F5807F28BFD360506840F001005B
:109E30005060107828B15078002804BF0120F8F74E
:109E4000FAFF2846F9F77CFA012070BD10B50178B9
:109E5000022211F003011CBF0129022902D1FFF7E0
:109E6000A1FF0246104610BD2DE9F0415F4E0446A9
:109E70003046726803780025002A1CBF00204FF08E
:109E8000010C54D0B1680CFA01F7174207D1491CF4
:109E9000B1600D2928BFB560401C0D28F2D3B16810
:109EA00009B3544800EBC1000CFA01F122EA0101A8
:109EB00008387160317D0278227042786270827851
:109EC000A270C278E270027922714279627182795D
:109ED000A271C07901F03F0100F0C0000843E071B9
:109EE0007068D8B915E0716909B34148D6F80CC05B
:109EF00000EBCC000CF1010CC6F80CC0BCF5807F67
:109F000028BFF560491E716104BF22F00101716034
:109F1000D0E7002B1CBF0120F8F782FFB068401C7F
:109F2000B0600D2828BFB5600120BDE8F081002B8E
:109F30001CBF0120F8F774FF25706570A570E570EF
:109F400025716571A571E5710220BDE8F081274991
:109F500010B44A6800204C69002A19BF01210B4641
:109F600010BC704703FA01FC1CEA020F18BF401C2A
:109F7000491C0D29F6D312F0010F18BF204410BC64
:109F8000704700B50178427883B0890102F007027A
:109F900041EA82018DF80010418809098DF801100D
:109FA000818809098DF80210817801F00F0201798A
:109FB00062F31F118DF80310017A8DF80410417AB5
:109FC0008DF80510C2798379C02101EA021203F0ED
:109FD0003F031A438DF80620C07901EA80108DF8FE
:109FE00007006846FFF7DEFE03B000BD3C06002018
:109FF00028450020C844002070B50E4680280CD2A9
:10A000008119491E802908D205030024002E04D995
:10A010002846F8F765FA012801D0002070BD641CBD
:10A0200005F58055B442F3D3012070BDB0F5006F43
:10A0300024BF0020704710B50002F8F7F2FA01289B
:10A0400018BF002010BD10B5064CFFF7C8F9012855
:10A0500008BF10BD206801F0D0F9002818BFFAF73A
:10A06000FCFCF2E7F806002010B5FE4C2068006802
:10A07000216820F0010008600020F6F7C3FAFA48D2
:10A080000168496C026841F40061516400BF00BF7F
:10A0900000BF0168496C026821F40061516400BF8F
:10A0A00000BF00BF0168D1F82C13026841F0020123
:10A0B000C2F82C1300BF00BF00BF0168D1F82C13F9
:10A0C000006821F00201C0F82C1300BF00BF00BFE0
:10A0D0000F210020FAF753FD002808BF10BD5F20B4
:10A0E00021688860216802204860F7F7B6F8206888
:10A0F0000068216840F00100086010BDDB4A0028BC
:10A10000916814BF41F0010021F001009060704798
:10A1100010F0010F08BF7047D448816841F0010179
:10A1200081607047D14B99680A0E120721F07F4178
:10A1300042EA0060084398607047CC488068C0F3EA
:10A140000360704770B5C94D2A69521C2A6100230B
:10A150000028C8BF6B610CD0AA6812F0010F38D07C
:10A16000C2F30362140008D0022A18BF002409D0E9
:10A170001FE06A69521C6A61EEE70028C8BF02242A
:10A1800019DC16E0002918BF0A2402D00EF0EDF801
:10A1900011E058B9B64869690068B0F81201884200
:10A1A00038BF0024F2D3A86901280FD068780128AD
:10A1B0000CD094420DD0A868010E090720F07F4012
:10A1C00041EA04610843A860012070BD0024AB612E
:10A1D000F1E7002070BD2DE9F041A44D04460026B2
:10A1E000686A3746012806D16068F9F74BFEA86A0D
:10A1F000032808BF6F626068B0B103F08BFD0028D0
:10A20000C8BF01260FDCA888401CA88098480068B9
:10A21000017F11F0010F07D0807FA988814203D907
:10A220006068F9F72FFEAF803046BDE8F0410021AD
:10A2300088E78E490120C87070472DE9F04F8DB036
:10A2400080468A4E00200C90B0680024C0F303655D
:10A250004FF0FF3005900490F06AD8F804B0A146A2
:10A260000DF1180AB0F5000F07DB4FF07E5110F02A
:10A2700013FDF0625846F9F705FE0027BBF1000F09
:10A280000ED004980097CDE902700023524605A92C
:10A290000197584600F017FC814600F00EFC04467A
:10A2A00005980028C8BFB78002DCB088401CB08089
:10A2B0006F480068017F11F0010F1DD0B0F8140144
:10A2C000B188814206D8B069012803D0B07801284E
:10A2D00003D011E0B078012803D10220B070C01E75
:10A2E00005903B46B780CDE90074DDE90410029784
:10A2F0004A460397FAF752FBBCB1022D0AD015B1BA
:10A30000042D04D016E00598012814D102E0059828
:10A31000012811D1D8F80000CDE900045549CDF845
:10A320000CA068460EF07AF80C90022D04BF642051
:10A33000208001D005B927804F480078012804BF4C
:10A340002046FFF745FB059800281CBF7478022CB7
:10A3500013D0F068B0F5000F07DB4FF07E5110F01E
:10A360009BFCF060B0F5000F04DA002C04BF012064
:10A37000707007D0012C06D104E04048F06077707F
:10A38000B77000E005970598012818BF00200C99C8
:10A39000FFF7D8FE0DB0BDE8F08F394801680969B4
:10A3A000006841F0010101613648016849690268AD
:10A3B00041F40071516101680969026841F00401CA
:10A3C000116101680969006841F0100101612E48BE
:10A3D00001680968006841F0010101602B480078BC
:10A3E0000022224900281CBFCA807047C888B0F5E7
:10A3F0007A7F87BFCA8030BF401CC88070472DE974
:10A40000F04F87B04FF0000B0524FAF7ECFA054641
:10A4100000F086FD1348282102689160006804213D
:10A42000416008200EF00BF8104F4FF00008184E56
:10A430004FF00309DFF830A0FEF7D1FF012807D065
:10A44000B868C0F30360A84208BFBBF1000F2CD06E
:10A4500000F066FDFAF7C4FA05281ED0FAF7C0FA34
:10A46000044617E090AE11008CAE11005406002097
:10A47000F8060020550600202D0600200000344379
:10A4800088AE110078AE1100A8AE11003006002091
:10A49000410700200520FAF7B2FA052C1CBF204620
:10A4A000FAF7ADFA07B0BDE8F08F6846F7F7ABF9F9
:10A4B000A0B3307830B3DAF80000C0F81C90022165
:10A4C0007F20F5F7C1FF0C214FF40070F5F7BCFFBA
:10A4D00000BF00BF00BF0C214FF40070F5F7B4FFC0
:10A4E00000BF00BF00BF002140F20120F5F7ACFF24
:10A4F00000BF00BF00BF002140F20120F5F7A4FF1C
:10A5000086F800806846FFF7CAFB6846FFF795FEAD
:10A510008346F7F795F9FAF7B6FA8DE7FFE7FAF70A
:10A5200091FA89E72DE9F04F87B0F6F752FDF8F779
:10A5300093FF814D0124286A10B9F7F7D0FC2C62F3
:10A540007E4E3068B0F90E11B0F90C0100F054FAEB
:10A550000DF007FF7A48EC61E862002002F0DEFDB2
:10A56000FAF73EFA052804BF4FF00008DFF8D4914F
:10A5700023D17248AA680068C2F303618B00D0F847
:10A58000F800C5F81080D84000F00F00C5F814801E
:10A5900000297CD0022915D0042979D0090722F09E
:10A5A0007F4041F000710843A860FEF718FF0128C2
:10A5B00003D0FAF715FA0528DBD007B0BDE8F04F55
:10A5C0000DF0D1BE834600240526FAF70CFADFF819
:10A5D00078A10746C5F80CA02878012805D10F21DD
:10A5E0005846FAF7CCFA0028DFD000F099FCDFF8E3
:10A5F0005CB12820DBF800108860DBF80010022036
:10A600004860287801281ED1D9F80000406CD9F89C
:10A61000001040F400604864012002F006FCD9F804
:10A620000000406CD9F8001020F400604864F6F790
:10A6300014FEDBF800000068DBF8001040F00100B9
:10A64000086085F8008040F6FF7BC5F830B0042034
:10A65000C5F80CA00DF0F3FEDFF8F4A0FEF7BFFE86
:10A66000012806D0A868C0F30360B84208BF002CD8
:10A6700014D000F055FCFAF7B3F9052805D0FAF725
:10A68000AFF906460520FAF7BAF9052E01E04CE0CD
:10A690004EE01CBF3046FAF7B2F986E76846F7F796
:10A6A000B2F8C8B39AF8000030B3D9F8001003200C
:10A6B000C86102217F20F5F7C7FE0C214FF400701E
:10A6C000F5F7C2FE00BF00BF00BF0C214FF40070C1
:10A6D000F5F7BAFE00BF00BF00BF002140F2012025
:10A6E000F5F7B2FE00BF00BF00BF002140F201201D
:10A6F000F5F7AAFE8AF80080C5F830B0F7F789FCB4
:10A700006846FFF7CCFA6846FFF797FD0024F7F795
:10A7100097F8FAF7B8F9A1E7FFE7286B411E29631C
:10A720000A2838BFFFF7A0FC98E7FFF768FE3CE770
:10A7300003F0CEF839E7000054060020F8060020A8
:10A74000000040408CAE11000000164390AE110096
:10A7500041070020F0B4FF4EDDE905C43668049DD2
:10A76000B66916F0010F04D01F464B1BCD1BDBB2A0
:10A77000EDB216F0020F06D06746A2EB040CD21B16
:10A780000CF0FF0CD4B216F0040F08D080F800C013
:10A790004A1B84704270C91AC170F0BC70470370C4
:10A7A000857080F801C0C470F0BC70472DE9F0439B
:10A7B000164601FB06F90D46014685B01F464A467E
:10A7C000E5480EF0DCFFE44C02F07EFD4FF000089F
:10A7D00018B108F096FD01281AD002F075FD18B1E5
:10A7E00008F08FFD082842D0B7F5805F1CBF00201D
:10A7F000B9F1000FDCBF05B0BDE8F0832156794305
:10A8000009132154401C8145F8DC05B0BDE8F083F4
:10A8100000210B46002ECEBFDFF838C305B0BDE8DF
:10A82000F0830020002D1CDDDCF8002092F83E9122
:10A830009945DCBF92F83F914B450CDC92F83C9176
:10A840008145DCBF92F83D21904204DC62567A4398
:10A850001213625401E004F80180401C491CA84214
:10A86000E2DB5B1CB342DCDB05B0BDE8F083AE424B
:10A870008CBF701E681EC2B2B54234BF681E701E07
:10A88000C1B20420CDE90002002303A80292FFF721
:10A8900061FF00210A46002EDCBF05B0BDE8F08351
:10A8A0000020002D19DD9DF80D309342DCBF9DF88E
:10A8B0000F309A4209DC9DF80C308342DEBF9DF8D0
:10A8C0000E30984204F8018003DD63567B431B136E
:10A8D0006354401C491CA842E5DB521CB242DFDB3A
:10A8E00005B0BDE8F0832DE9F0411C4615460E4643
:10A8F0000746F8F723FB21462846F8F73EFB0623D8
:10A90000954A31463846F8F74EFCBDE8F041F8F775
:10A9100016BB924A9060D16070472DE9F00F002479
:10A92000DDE90875B7F5805F08BF642D2AD00026E1
:10A93000002B87BFA5F16409C5F16408BDE8F00FDD
:10A9400070470020002A17D9B0FBF2FA31F914C081
:10A95000642D0CFB07FC4FEA2C3C27BF0AFB09FACD
:10A960000CFB0ACC0AFB08FA0CFB1ACC21F814C029
:10A97000401C641C9042E7D3761C9E42E1D3BDE8A4
:10A98000F00F7047884204BFBDE8F00F70475A438C
:10A99000BDE8F00F52000EF0F2BE2DE9F041804606
:10A9A0006C4882B00F4600681D46164690F84C1061
:10A9B000ADF8001090F84D10ADF80210B0F84A1044
:10A9C000ADF80410B0F848000024ADF80600F8F720
:10A9D000B5FA6846F8F7A6FB29463046F8F7C4FAF8
:10A9E00039464046F8F7B0FBF8F7A9FA5B4804612E
:10A9F00002B02046BDE8F0815849088070472DE933
:10AA0000F041574E8AB005465448CDE90056A6F1AC
:10AA100048080C46CDF80880B0F9001003913F2992
:10AA2000C8BF3F2005DC11F1400FB8BF6FF03F00F9
:10AA300000DA039000200490F8F780FA49484A4F62
:10AA400001783878F8F790FA6846F8F724FB089010
:10AA5000F8F775FAC4E90068BDF814002081BDF864
:10AA600016006081BDF81800A081BDF81A00E081D1
:10AA7000BDF81C002082BDF81E006082BDF81C00DD
:10AA8000BDF81E103A7801FB020035F910000AB03B
:10AA9000BDE8F08135487047344B032838BF187043
:10AAA0005970002A08BF7047012A01BF9878022810
:10AAB0000320987018BF9A70704728484069704703
:10AAC0002648806970472DE9FF4FADF2A44D064638
:10AAD0000020DDF8E0A4CDF89C04ADF88804CDF8A2
:10AAE000900493464FF0FF394FF4906102A80EF0A6
:10AAF000E7FEBAF1000F1CBF9AF80000CDF89004F1
:10AB00001948DFF86C80194F047816480578114809
:10AB10000068008ECDF8940408F59060CDF88C6440
:10AB2000CDF89804F9F7B9F8019000284BD03246D7
:10AB30002346009510460199F9F78CF80D480078E6
:10AB4000022804BF0198FEF743FF3878022833D16A
:10AB5000002311E0F8060020284D00208806002080
:10AB6000B04F0020BB050020BA0500208A06002057
:10AB7000305000202D060020002D88BFDFF8A4C330
:10AB80001AD90020002C13D903FB040189B2401C00
:10AB900036F9112080B202EB420292008CFB02E2F5
:10ABA0004FEAA20EAEEBE27226F811208442EBD8F7
:10ABB000581C83B2AB42E4D3DB480078092804BFB9
:10ABC0003046FEF705FFDDF88C040190D748C0F849
:10ABD0001480F9F753F90646787801281FD13878A0
:10ABE00001283CD002280CBFB42300230022002DF2
:10ABF00012D90020002C0BD902FB040189B2401CA1
:10AC000036F811C080B29C4426F811C08442F3D8B3
:10AC1000501C82B2AA42ECD3C54902204870234698
:10AC20003246009502A80199F9F714F8BE4F38781A
:10AC3000032804BF3046FEF7CBFE3878052804BF52
:10AC400002A8FEF7C5FE3E463878062804BF02A8D3
:10AC5000FEF7BEFE02AF307822280CD107E0B878AC
:10AC6000012814BF6FF0D1036FF0B303BEE70021DA
:10AC70003846FEF7EBFFDDF8940410F0010F11D019
:10AC8000F8F75CF929462046F8F777F90623A94A30
:10AC900039464046F8F787FAF8F751F9307808282E
:10ACA0000ED010E064214FF48050CDE900012B4616
:10ACB000224639464046FFF730FE3078082802D158
:10ACC0004046FEF785FEDDF8940410F0060F30D004
:10ACD00002F060F968BB0020CDF894049648006843
:10ACE00090F84C10ADF8001090F84D10ADF802102F
:10ACF000B0F84A10ADF80410B0F84800ADF80600FE
:10AD0000F8F71CF96846F8F70DFA29462046F8F7D7
:10AD10002BF941460846F8F717FAF8F710F9834976
:10AD2000DDF89404086130780A2804BF4046FEF735
:10AD30004FFEDDF8A80410B3BBF1000F28D0DDF8FA
:10AD40009C0400900DF591633A464046DDF8981456
:10AD5000F9F710FC8146BDF88804072806D1600089
:10AD600000FB05F2394640460EF009FDB9F1FF3F00
:10AD700012BFB9F1000F0020ADF8880402E0BBF16A
:10AD8000000F05D059464046FFF739FEABF81400D6
:10AD90003078072804BF4046FEF71AFEDDF8A80405
:10ADA000002818BFC0F80090DDF8D80400281CBFA8
:10ADB000BDF888140180BAF1000F1CBFDDF89004C3
:10ADC0008AF80000DDF88C040DF2B44DBDE8F08F78
:10ADD0005A4870472DE9F05F814659481746884622
:10ADE0000078564C4600F9F76FF9DFF83CB182461F
:10ADF00000259BF80000042804BF4846FEF7D3FD59
:10AE00009BF80000052804BF4846FEF7CCFD9BF8E0
:10AE10000000032804BF5046FEF7C5FD9BF8000064
:10AE2000232804BF4846FEF7BEFD0020002E09D9A6
:10AE300039F810103AF81020891A24F81010401C24
:10AE40008642F5D89BF80000062804BF2046FEF78E
:10AE5000AAFD9BF80000222804BF2046FEF7A3FDB0
:10AE60000020711E18BF0A4612D004EB400134F8CE
:10AE700010304988C91A09B224F810100029B8BF47
:10AE8000494209B2A942C8BF0D46401C9042ECD3CA
:10AE900004EB460020F8025C9BF800000A2804BF7F
:10AEA0002046FEF780FD9BF80000082804BF2046DE
:10AEB000FEF779FD9BF80000072804BF2046FEF747
:10AEC00072FD9BF80000012804BF2046FEF76BFDD1
:10AED0009BF800000E2804BF2046FEF764FD9BF897
:10AEE0000000212804BF2046FEF75DFDB8F1000FE9
:10AEF00010D011494FF0FF300968B1F97220AA4211
:10AF0000B8BF012004DBB1F970108D42B8BF00203A
:10AF1000C8F80000002F18BF3D804846BDE8F09FEC
:10AF200070477047676666662D0600208806002019
:10AF30008A060020284D0020F80600203059002005
:10AF4000C105002008283CBF9A49087070470020BE
:10AF50009849C8609848006890F88100082838BF70
:10AF60000870704793480078704710B50446F6F7AC
:10AF700030F8924A03211268D161052C4ED2DFE8E5
:10AF800004F0031221303F0001217F20F5F75CFA25
:10AF90008C214FF48470F5F757FA5C214FF48570DB
:10AFA000F5F752FA3AE001217F20F5F74DFA8721B3
:10AFB0004FF48470F5F748FA59214FF48570F5F78E
:10AFC00043FA2BE001217F20F5F73EFA75214FF47B
:10AFD0008470F5F739FA4D214FF48570F5F734FA9E
:10AFE0001CE001217F20F5F72FFA67214FF48470D0
:10AFF000F5F72AFA43214FF48570F5F725FA0DE0AD
:10B0000001217F20F5F720FA58214FF48470F5F7DD
:10B010001BFA3A214FF48570F5F716FAF8F7F9FEA6
:10B02000F6F71BF9012010BD012070476248614905
:10B030000068B0F876004242C8688242BCBF401E39
:10B04000C86070472DE9F04FA1B09346884604468A
:10B050004FF0000902F0BAF8574E8246554D30685D
:10B06000B0F96E00A0420DDAA868401EA86009D2AF
:10B070006420A860686803280CBF0020401C68603A
:10B08000FFF773FF4E4F3878072829D14D485946AE
:10B090000078820068460EF072FBADF80040ADF813
:10B0A0000280ADF804A0A889ADF80600A888ADF824
:10B0B00008003068B0F87210ADF80A10B0F87410DB
:10B0C000ADF80C10B0F86E10ADF80E10B0F87600B8
:10B0D000ADF810003878072804BF6846FEF763FC17
:10B0E000484621B0BDE8F08F00207047DFF8C4C0AB
:10B0F00000209CF80210002914BF012200229CF8B5
:10B100000110002918BF01218A4208BF70470A1C9C
:10B1100018BF012210B48CF80220274A1368D3F814
:10B12000A42012F0040F0FD021B1C2F3031008289D
:10B1300009D206E00020CCF80C0093F88100082822
:10B1400001D28CF80000012012F0020F18BF01207C
:10B1500010BC70472DE9F041174F00263868D0F831
:10B16000A40010F4807F21D0124D69780C1C18BF08
:10B170000124C0F30330012101FA00F0F7F785FE46
:10B180003968B1F8A41011F4007F01D028B103E0B0
:10B19000002818BF002000D10120844206D00028DA
:10B1A00018BF01206870FFF7A1FF06463046BDE8D2
:10B1B000F0810000A4060020F80600208CAE1100EB
:10B1C0002D060020C10500207148006800F5407080
:10B1D00070476F48006800F58070704770B56C4C20
:10B1E0006C4922681068884204BF5068B0F5087F37
:10B1F00024D1D2F808C0BCF5405F1FD86649D0689A
:10B2000088420DD0002311461846B3EB9C0F07D29D
:10B2100051F8045B401C6B40B0EB9C0FF8D36BB94A
:10B2200002F5807000F0E9F840B1206800F5407048
:10B2300000F0F2F800281CBF012070BD002070BD96
:10B24000534910B54FF48E100860FFF7C7FF002870
:10B2500018BF012010BD4FF48E10F7F7C9B84C4845
:10B260004C4A00680168914206BF4168B1F5087F09
:10B2700000207047464800680069704744490968E3
:10B280000A6982429CBF00207047C0EBC00001EBFE
:10B29000C00000F5806070473D4A126802EB8003F1
:10B2A0005B6A1A443D4B53F82000FF3020F0FF004A
:10B2B00000FB012070472DE9F0010022344D1746B4
:10B2C0002E1D831893F92840002CB8BF41F8227036
:10B2D00010DBD5F800C0D3B20CEB830856F823304E
:10B2E000D8F82480FF33C44423F0FF0303FB04C3D6
:10B2F00041F82230521C102AE3D3BDE8F001704718
:10B300002DE9F0410025174604460029B8BFBDE8E5
:10B31000F081042C02D0052C10D014E0F9F760FB6A
:10B32000052810D1FEF709FF022808BF03250AD01F
:10B33000FEF703FF002808BF022504E0F9F750FBE1
:10B34000052808BF01251248144E006856F824103D
:10B3500000EB8400FF31406A21F0FF0100F5E0308E
:10B36000503005FB0105F9F73BFB022808D101F03D
:10B37000CAFE28B956F82400FF3020F0FF0005442B
:10B3800056F8242039462846BDE8F041F7F726BB99
:10B39000B406002054465053EFBEADDEB806002080
:10B3A00010B5234CFFF74CFFD8B1FFF70DFF014656
:10B3B000AC2220480EF028FAFFF70BFF01464FF4AD
:10B3C000C47220680EF020FA2068406D01F0DBFDA9
:10B3D000206890F8F400BDE8104000F00100FEF78E
:10B3E00097BE4FF4C47120680EF06AFA0021042061
:10B3F000F9F708FBFEF727FED4E758B10E4A0168BB
:10B40000914207D1406820F00F00B0F50C7F04BFD7
:10B41000012070470020704738B1006820F00F000D
:10B42000B0F5907F04BF01207047002070470000F6
:10B43000F80600208C10002041505352002808BF0D
:10B440007047401E00BF00BF00BF00BF00BF002804
:10B45000F7D1704770B5614D82B00024286804664A
:10B460005F480168D1F82C13006841F00801C0F86A
:10B470002C13F7F7DDFF28680069296840F0010008
:10B480000861601EF7F760FF564880234FF4801272
:10B49000002152F821C040F821C0491CB1EB930FA4
:10B4A000F7D3F7F763FFF8F70DFAF8F737FA00204C
:10B4B000F8F709FA2320F8F7FAF9F7F718FDF8F783
:10B4C000A1F9F8F719F8F7F73BFDF6F7B1FCF5F736
:10B4D000F3FBF7F7E0FEF7F79BFE434E0094019471
:10B4E0000423002207213068F8F7FAF83068F8F7EB
:10B4F00072F90420CDE900043C4C034600220721E8
:10B500002068F8F7EDF82068F8F765F9F6F767FDB9
:10B51000F6F774FE364800683649884218BFF6F7D9
:10B520006DFEF8F7EBFAFDF729FFFEF72CFC62B68B
:10B53000FFF736FF30480CF076FD304C2068B0F94C
:10B540000C010CF00CFFF8F73FFBF9F72DFC20681D
:10B55000418A008AFEF71FF92068806EC0F34E0111
:10B5600061F35F0001F0D0F9FFF7DBFC0022114628
:10B57000022001F0D6F900226421072001F0D1F960
:10B5800029680120086602B0002070BD01F0C0FDEE
:10B5900001460220F9F736FAF9F722FA06281AD2FC
:10B5A000DFE800F019090313160602F03DFAF3E78D
:10B5B000FEF7B8FFF0E7FAF788F8F9F711FA012873
:10B5C00004BF0220F9F71BFAE6E701F0ACFBE3E762
:10B5D000FEF739FDE0E7F9F75DFADDE788AE110027
:10B5E0008CAE110000640020A4AE1100A0AE1100CA
:10B5F00084160020544649538C100020F806002081
:10B60000FD49087070474FF42C30704770B54FF407
:10B610002C3044F264422146F6F7E4FDF74A2168F3
:10B62000204691421BD16168B1F5007F17D3D4F851
:10B6300008C0002344F264418C4588BF44F2644C46
:10B640000022B2EB9C0F28BF70BD54F82250521C50
:10B650002B44B2EB9C0FF8D3002B08BF70BD002029
:10B6600070BDE64901604FF40071416044F26441ED
:10B6700081600021C16080F8201080F8211080F8DE
:10B68000221080F8231040F2FF72C0E9042181618A
:10B69000C161016500F580404FF6FF71A0F85414B8
:10B6A000A0F85614A0F85814A0F85A14A0F85C1486
:10B6B000A0F85E14A0F86014A0F86214012070478E
:10B6C00070B50021C1600B46D0F808C044F2644157
:10B6D00004468C4588BF44F2644C0022B2EB9C0FB8
:10B6E00006D254F82250521C2B44B2EB9C0FF8D3D4
:10B6F0005942C1604FF42C3044F264422146F7F7BE
:10B700006DF9012818BF002070BD2DE9F04F0546E6
:10B7100093B088460020F5F79DFE0990F9F7C2FA2C
:10B720000590B748B84F032690F80090B5480078C8
:10B7300001903868C66102217F20F4F785FE40F24F
:10B740000220F4F79AFEC0F30214B8F1010F7DD085
:10B7500000200290AD480390AD480690AE4800909E
:10B760003868DFF8B0A24FF00008C346C661012177
:10B770007F20F4F769FE4FF48770F4F77EFEC0B2C5
:10B78000119002217F20F4F75FFE40F20720F4F7CA
:10B7900074FEC6B24FF40270F4F76FFE0FF08EF92C
:10B7A00010909E4816F0100F50F8240007909C4807
:10B7B00050F82400049018BFD04616F0200F04D093
:10B7C000514640460FF014F8804616F0400F04D062
:10B7D000404600990FF00CF88046F00904D040462E
:10B7E00000990FF005F8804616F0010F18BFD346F8
:10B7F00016F0020F04D0514658460EF0F9FF83466A
:10B8000016F0040F04D0584600990EF0F1FF83465D
:10B8100016F0080F04D0584600990EF0E9FF834651
:10B8200018F1FF4F2CBF88F0004040467D4CA042ED
:10B83000D8BFA046414658460FF042F808904FF056
:10B84000FF3103980FF0FDFA064600E019E0069973
:10B850000FF04CF90746394630460EF0C9FF0D90FF
:10B86000394630460FF018FA0C90002000900198ED
:10B87000002884BF09FB00F0069020D813B0BDE873
:10B88000F08F0198002609FB00F8B8F1000F8EBF79
:10B89000654F13B0BDE8F08FB5F900000FF00EF959
:10B8A00057F824100FF022F90FF0CCF825F8020B0E
:10B8B000701C86B2B045EFD813B0BDE8F08F0026FB
:10B8C000B9F1000F40F22881009800FB09900E901A
:10B8D000009800FB096087B200200F900998B0F92A
:10B8E00000000B900998801C0990059810F801BB86
:10B8F00005901BF0800F1CBF4FF07E50029000247B
:10B900002BFA04F010F0010F13D00120A0400EF02C
:10B91000BEFC464A464B0EF021FD82460A910F9826
:10B920000EF03AFF52460A9B0EF098FB0EF064FBB5
:10B930000F90601CC4B2072CE2D3049907980FF053
:10B94000ABF90446DDE90C100FF0A6F90A900B984C
:10B950000FF0B4F86FF00A010FF073FA4FF07E5158
:10B960000FF09AF90B90079903980EF041FF029996
:10B970000FF0BCF882464FF07E5002990FF08CF920
:10B980008346DDE903010EF033FF59460FF0AEF8B0
:10B9900051460FF081F912901198401E0FF08EF869
:10B9A000824610F1FF4F28BF8AF000401D498842AF
:10B9B000D8BFDFF870A04FF0804110980EF018FF4C
:10B9C000834651460A980EF07BFF59460FF08EF8D9
:10B9D0000B990FF08BF803990FF054F9824614F18C
:10B9E000FF4F2CBF84F0004020460E498842D8BF4C
:10B9F0000C4618F1FF4F1DE00007002053454C4650
:10BA0000BA050020BB0500208CAE11000000B0403C
:10BA1000CDCC4C3FC3F5A04048E1DA40B8B21100AC
:10BA2000D8B211000AD7233CF8B211009A9999991B
:10BA30009999A93F2CBF88F0004040468842D8BF62
:10BA40008846DDE907100FF051F80EF0A5FECDE9AC
:10BA50000A0141460F980EF033FF12990FF046F895
:10BA60000EF09AFE834650460F910EF095FE4FF071
:10BA7000FF320FF0B8F95A460F9B0EF0EFFADDE9EE
:10BA80000A230EF0EBFA82468B4621464FF07E5099
:10BA90000EF016FF0EF080FE52465B460EF05EFC86
:10BAA0000022FE4B0EF08EFD82460C4640460EF004
:10BAB00073FE524623460EF051FC0EF09DFAF849F3
:10BAC0000FF014F8F7490EF093FE0EF0D7FFF64989
:10BAD00080B20968896911F0180F09D011F0100FB0
:10BAE00001F0080107D061B90699B7EB510F08D3EF
:10BAF00025F817000BE000291CBF0699B7EB510F82
:10BB0000F6D30E99891B05EB410121F8020C701C3C
:10BB100086B24E45FFF4DCAE00980199401C80B21D
:10BB200000908842FFF4CBAE13B0BDE8F08F2DE952
:10BB3000F041ADF5906D0E46804600274FF49061C0
:10BB400068460DF0BDFEF5F7F0F80020F5F7E0F8D7
:10BB50000020F5F7D2F8F5F7C4F86846F8F79FFA31
:10BB6000D2480478D2480578002D18BF002C3BD06D
:10BB70003068002118F0030F80F8204080F8215031
:10BB800080F8221080F823102DD0F5F766FB0020F6
:10BB9000F8F7A2FA0120F5F756F82046F5F716FA5D
:10BBA000FAF73CFA36680020F5F754FC01466C437E
:10BBB00043F25400620030440DF0E1FDF9F772F8F1
:10BBC000014643F65400224630440DF0D8FDB948F2
:10BBD000007910F0010F06D0F6F71BFA002106F1EC
:10BBE0005400FFF792FD0127F5F7BEFA0DF5906DB1
:10BBF0003846BDE8F0812DE9F04FADF5117D0E46D8
:10BC0000044617464FF4107168460DF059FEA948D6
:10BC10004FF000084FF0FF39007910F0020F43F2A7
:10BC2000540007EB000504FB06F0909042D06946F3
:10BC3000AC46C246002E88BFA4F1010B2ED90020CD
:10BC4000002C25D9584508BF81F800801CD03CF94C
:10BC50001020002AD8BF81F8009015DD0CEB4003BE
:10BC6000B3F90230934207DCD31A4FF0640E03FBA2
:10BC70000EF393FBF2F206E09A1A4FF0640E02FB09
:10BC80000EF292FBF3F20A70401C491CA042D9D379
:10BC90000AF1010A0CEB440CB245D0D342F6540031
:10BCA00069463844909A0DF0AFFD4FF41071684624
:10BCB0000DF006FE7F48007910F0040F04BF0DF56B
:10BCC000117DBDE8F08F6B464FF0000A002C88BF55
:10BCD00006FB04FB36D900210846BBF1000F05D84E
:10BCE00029E0112908BF83F800801FD00AEB000C5F
:10BCF00035F91C20002AD8BF83F8009016DDA44433
:10BD000035F91CC0944508DCA2EB0C0C4FF0640E16
:10BD10000CFB0EFC9CFBF2F207E0ACEB02024FF0D6
:10BD2000640E02FB0EF292FBFCF21A702044491CD6
:10BD300023448345D5D804FB1630431C0AF1010A7D
:10BD40005445C8D842F6544069463844909A0DF09C
:10BD50005BFD0DF5117DBDE8F08F70B51446524ABC
:10BD60000546554B10680E4690F8E8201A8000F002
:10BD70009CFE002305FB06F1002984BF4F4ADFF833
:10BD800040C112D9106841F6540630F8135004EB44
:10BD900043003552DCF8005000F5005035F81350E0
:10BDA0005B1CA0F854509942ECD842490120C8606D
:10BDB00070BD30B5054691B000240120F4F743FF73
:10BDC0002046FFF75BFA6946FFF775FA0099079876
:10BDD000F4F74EFD3B4901200968C1F814032846D9
:10BDE000F9F712FFFF20F9F764F9F4F79EFF00203E
:10BDF000F4F78EFF0020F4F780FFF4F772FF0020C5
:10BE0000F8F785F80020FAF7C8F90120F8F764F987
:10BE100011B030BDF0B5ADF2C44D0D460646144626
:10BE200000274FF4906168460DF04AFD0120F4F7B9
:10BE30000AFF3846FFF722FA070008BFF8F70DFEA1
:10BE40000DF590613846FFF736FADDF88014DDF81D
:10BE50009C04F4F70DFD1B4901200968C1F8140387
:10BE6000F9F7D2FEF4F761FF0020F4F751FF00204C
:10BE7000F4F743FFF4F735FF2020F9F71AF9012012
:10BE8000F8F72AF96846F8F70AF90020FAF785F971
:10BE90000020F5F7DFFA06FB05F115E00000F03FA2
:10BEA00000007A440080CE43F8060020BA05002046
:10BEB000BB05002000070020240700202C070020DD
:10BEC000280700208CAE11004A00014641F25400C0
:10BED00020440DF054FC0DF2C44DF0BD70B5044685
:10BEE00015460E460020F4F728FFF7F7C7FF04FBBE
:10BEF00006F14C0021460DF0C1FC0220FFF759FF6E
:10BF0000F9F7CAFF0320FFF754FFF9F7D2FFF7F75D
:10BF1000B5FF0146224605F654000DF030FCF7F758
:10BF2000ADFF21460DF0AAFCBDE870400120F4F7FA
:10BF300004BF2DE9F14FADF5065D01273D464FF4F5
:10BF400010610DF6D8500DF0BBFC14204FF0000A24
:10BF500014901390129011905446CDF840A00120F7
:10BF6000F4F771FE2046FFF789F96946FFF7A3F958
:10BF700000990798F4F77CFCDFF850850120D8F889
:10BF80000010C1F814034FF0120920244FF410766A
:10BF90000020F4F7B2FEF5F753FCD8F800100320A8
:10BFA000C86101217F20F4F74FFA11210E20F4F728
:10BFB0004BFA5A210820F4F747FA36210A20F4F701
:10BFC00043FA02217620F4F73FFA02217F20F4F7AA
:10BFD0003BFA6A210220F4F737FA8E210420F4F7A5
:10BFE00033FAF1210720F4F72FFA07210820F4F79C
:10BFF0002BFA00211620F4F727FA03217F20F4F70B
:10C0000023FA89210520F4F71FFA67210620F4F7A7
:10C010001BFA45210720F4F717FA23210820F4F72B
:10C0200013FAF1210920F4F70FFA4FEA460C04FB4A
:10C0300009F8CDF800C001E0002D4FD00120F4F741
:10C0400002FEF5F7D1FA0020F9F733F8F5F705F914
:10C050000120F4F7F8FDF5F7C7FA1198F9F729F878
:10C06000F5F7FBF8002F1CBF42F2601BEB442ED00B
:10C070005846F5F7C8FB40B30020F4F73EFEF5F74D
:10C08000DFFB0DB30AF101001FFA80FABAF1010FCC
:10C090004FF000000AD0F5F7DDF9014641F65830BF
:10C0A0006844009A0DF06BFB002510E0F5F7D2F91B
:10C0B000014641F2D8606844009A0DF060FB149983
:10C0C0001198084480B2119001E0002FD0D10127CF
:10C0D000002D04BFFE48D0F800B0AFD10025002EDF
:10C0E00084BFBBF8EC700DF59B6A37D941F6583028
:10C0F0006844642130F91520A0F5906030F91500EE
:10C10000101A484300EBD07040104AF8250017F091
:10C11000010F20D0202D18BFB5F5007F05D0E02DF0
:10C1200018BFB5F5A07F0CD015E00EF0B0F84FF0B9
:10C130006632E84B0EF012F90EF04CF84AF8250082
:10C1400009E00EF0A4F8E44AE44B0EF007F90EF013
:10C1500041F84AF825006D1CB542C7D3002739467F
:10C16000002C88BF0DF59B6A2DD900239C461A46EA
:10C170003846B7EB580F38BFBBF8ECE013D21EF0CF
:10C18000010F02D0002900F0E6805AF82050521C1E
:10C19000AC4400EB580592B25AF825502B44204489
:10C1A000B0EB580FEBD3BCFBF2FC41F6D870B3FBFD
:10C1B000F2F268447F1C40F821C0803040F8212012
:10C1C000491CA142D1D30020002E1DD941F6D873BD
:10C1D0000DF59B626B4402F5DC5C16ADB0FBF4F12F
:10C1E00004FB1101B0EB560F34BF53F821105CF87B
:10C1F000211052F82070C91B0029B8BF494225F808
:10C200001010401CB042E9D34FF0000AB9F1000F02
:10C2100084BF42F220156D443AD916A800EB8A116A
:10C220000027402228460DF0AAFA0020B9F1000F9D
:10C2300084BF42F2D80CEC4426D99BF8EC100022C3
:10C2400011F0010F08D0002818BF08287ED0092857
:10C250001CBF1128002779D03946A7420BD235F8E8
:10C2600011E05CF82030521C7344491C4CF820301B
:10C2700092B2A142F3D35CF8201091FBF2F14CF89A
:10C280002010401C4845D8D30AF1010ACA45C4D33E
:10C290000020002E82BF42F2D8056D440DF1580CEB
:10C2A0000CD941093CF8103055F82120D11A48BF6B
:10C2B000991A2CF81010401CB042F2D30020002E26
:10C2C00084BF16AA0DF6D85109D951F8203032F89A
:10C2D00010C0634441F82030401C8642F5D81098C5
:10C2E0000125401CC0B2109012981190139910981B
:10C2F0004FF0000A2F4681423FF69EAE0024002EEA
:10C3000017D9DFF8DC8116AD0DF6D857109857F81D
:10C310002410B1FBF0F00DF0D1FF4FF06632434630
:10C320000EF01CF80DF086FF25F81400641CB442D2
:10C33000ECD30DF5005043F65443D0F8800116A914
:10C34000009A18440DF060FA61B000E011E00DF5BC
:10C35000005DBDE8F08F002818BFB0F5807F3FF486
:10C360001EAFB0F5907F18BFB0F5087F3FF417AF50
:10C370000BE7012770E72DE9F0035A4D4FF0000C51
:10C380006246A5F802C000299CBFBDE8F0037047D3
:10C39000554F40F60558A7F10A066B8837F8134049
:10C3A00094421FD1082B1DD200EB4203841804F5E0
:10C3B0000054A3F8548084F854C884F854CC03F58E
:10C3C000805442F25409A4F854C829F803C0A4F8D0
:10C3D00054C0A3F854C803F54053A3F854CC6B8859
:10C3E0005B1C6B80338893421CBF7388934204D1DB
:10C3F000831803F5005383F854CC521C8A42CCD3E3
:10C40000BDE8F00370472DE9F05FADF5924D44F2C1
:10C4100070456D444FF4906128460DF051FA03AE1B
:10C42000FF2244F2644130460DF020FA2D4F4FF0C8
:10C43000FF300290F8680DF1080AFF2428B9FF22A6
:10C440004FF4006129480DF011FA30460296FFF7CB
:10C4500008F9DFF87C804FF00109D8F8000090F867
:10C46000EA10B98090F8EB00032804BF87F8009029
:10C47000BC800120F4F7E7FB51463878FFF757FB03
:10C480002846F7F70CFE9DF82C409DF82D50002C07
:10C4900012BF002D0DF5924DBDE8F09F4FF0000A40
:10C4A000324629462046CDF81CA0FFF7A4FB387978
:10C4B00010F0080F3ED0D8F800000D4990F8E800C1
:10C4C000088000F0F2FA002014E000008CAE1100A9
:10C4D000F80600206666EE3FCDCCCCCCCCCCEC3F51
:10C4E0006666E63F0007002010070020007100206C
:10C4F0002407002004FB05F3002B84BFDFF8F8C3FA
:10C50000DFF8F8E314D9DCF8001041F6540B31F8E9
:10C51000102006EB40012BF80120DEF8002001F589
:10C52000005132F81020401CA1F854208342EAD870
:10C53000C7F80C90387810F0010F3ED097220421F4
:10C54000F420F5F726FC387910F0200F04D032469D
:10C5500029462046FFF75EFC387910F0400F27D0BF
:10C560000020F4F7EAFBF7F789FC024604FB05F02C
:10C570004FEA4009494610460DF080F90220FFF7C6
:10C5800018FCF9F789FC0320FFF713FCF9F791FC7D
:10C59000F7F774FC01464A4606F654000DF0EFF832
:10C5A000F7F76CFC49460DF069F90120F4F7C5FB7B
:10C5B0008A220421F420F5F7ECFB387910F0800F83
:10C5C0001CBF3046FFF7B5FCD8F8000090F8EC002F
:10C5D00010F0010F04D004FB05F13046FFF7CBFE4D
:10C5E000D8F8009099F8EB0001285AD1B88810F0DB
:10C5F000010F07D04FF4006206F15401C0480DF05E
:10C60000BEF84EE010F0020F08D042F660014FF481
:10C6100000626944BA480DF0B2F842E010F0040F2D
:10C6200008D042F660414FF400626944B4480DF00E
:10C63000A6F836E010F0080F0DD04FF400620DF5AB
:10C64000C351AF480DF09BF842F260014FF4006215
:10C650006944AC4823E043F6544103AB10F0100F9B
:10C66000194419D110F0200F08D041F254014FF4B1
:10C6700000621944A2480DF082F812E010F0400F59
:10C6800007D04FF4006206F654019D480DF077F88C
:10C6900007E010F0800F04D04FF4006298480DF0CE
:10C6A0006EF8387810F0400F7ED10898401C089042
:10C6B0000798002814BF0A98099800F1010014BFD8
:10C6C0000A90099004FB05F0401E58BFB9886CD44D
:10C6D00011F0010F13D006EB4002B9F9D830B2F9CE
:10C6E0005420934203DCB9F9DA30934207DA179AFF
:10C6F0000DF5804342F001021792A3F8680411F08F
:10C70000020F14D0321802F50052B9F9C83092F96C
:10C710005428934203DCB9F9CA30934207DA179AD6
:10C7200042F0020217920DF58042A2F8600411F067
:10C73000040F14D0321802F50052B9F9CC3092F936
:10C74000542C934203DCB9F9CE30934207DA179A9E
:10C750000DF5804342F004021792A3F8620411F031
:10C76000080F15D006EB400202F58052B9F9D0301F
:10C77000B2F95428934203DCB9F9D230934207DA74
:10C78000179A42F0080217920DF58042A2F864044D
:10C7900011F0100F18D006EB400202F50052B9F963
:10C7A000D430B2F9542001E07DE059E0934203DC3B
:10C7B000B9F9D630934207DA179A0DF5804342F063
:10C7C00010021792A3F8660411F0200F15D006EBA3
:10C7D000400202F58052B9F9DC30B2F9542093429C
:10C7E00003DCB9F9DE30934207DA179A42F02002EF
:10C7F00017920DF58042A2F86A0411F0400F13D091
:10C8000006EB4002B9F9E030B2F95428934203DC58
:10C81000B9F9E230934207DA179A0DF5804342F0F6
:10C8200040021792A3F86C0411F0800F15D006EBAC
:10C83000400202F54052B9F9E430B2F9542C934267
:10C8400003DCB9F9E630934207DA179A0DF5804315
:10C8500042F080021792A3F86E04401E7FF538AFB5
:10C8600099F8EB00F8B90598002144F26442334688
:10C87000CDF818A0904294BF024644F264420020D2
:10C88000B0EB920F06D256F820C0401C6144B0EBCA
:10C89000920FF8D34842D8604FF42C3044F26442EF
:10C8A0003146F6F79BF8D8F8000090F8EB00032823
:10C8B00002D11349179808801D208DF800004120EF
:10C8C0008DF801009DF85C008DF802009DF85D0078
:10C8D0008DF803009DF85E008DF804009DF85F0060
:10C8E0008DF8050006226946072000F043F80DF593
:10C8F000924DBDE8F09F00002C0700202807002083
:10C9000000690020007100204949C2B2C0F307202D
:10C910000A804880704746484188008861F31F209C
:10C92000704710B5424C012303FA00FC248882B002
:10C930001CEA040F04BF02B010BD00F00F0043EA70
:10C9400080008DF800008DF801108DF80220100A8B
:10C950008DF80300100C8DF80400100E8DF8050002
:10C9600000208DF806008DF807006846FDF76EFA86
:10C9700002B010BD012303FA00F000B52C4B83B0C8
:10C980001B88184204BF03B000BD072A88BF0722D6
:10C9900000206B46002A08D911F800C003F800C037
:10C9A000401C9042F8D3082804D200211954401C9E
:10C9B0000828FBD31846FDF749FA03B000BD10B5AF
:10C9C00082B000234FF0020C00934CEA80008DF8F7
:10C9D000000001938DF801301846002A88BF6B468D
:10C9E00007D911F800C01C18401C84F802C082420C
:10C9F000F7D86846FDF72AFA02B010BD10B40C4C07
:10CA000040EA01230228A288944602D0052805D0D6
:10CA100009E0002918BF022905D103E0002918BF49
:10CA2000022900D11A46944518BFA28010BC704755
:10CA300018070020F34908707047F24800B5C07825
:10CA400048F6B80183B0484301218DF80110002158
:10CA50004A1E8DF807108DF80010ADF804208DF8EF
:10CA60000810ADF802208DF806108DF80910F6F7C1
:10CA7000D2FEFCF7B4FC01280DD00120F6F7D0F966
:10CA8000F6F7E4FE0028F4D06846FDF77AFA0020B5
:10CA9000F6F7D9FEEDE7F6F7D0FE03B000BDD949B1
:10CAA00048707047D748407870472DE9F04FADF295
:10CAB000B44D4FF4906104A80CF002FFDFF84483FA
:10CAC0000221002088F80110FEF7D8FB002808BFDB
:10CAD000F7F7C3FFF4F77DFAF4F727F90020F4F72E
:10CAE00017F90020F4F709F9F4F7FBF804A8F7F7B1
:10CAF000D6FAF4F741FBCDF8AC0498F8020010F038
:10CB0000100F18BFF4F7CCFFBF4890F80090BF4853
:10CB10000778BF48002F0578BE48067818BFB9F1DE
:10CB2000000F0ED0FEF7FCF90020F7F7F0F998F8A7
:10CB3000020010F0100F0AD00120F7F7CDFA012003
:10CB400009E0002E18BF002DECD100F0E6B800205F
:10CB5000F7F7C2FA0020F7F7BFFA0120F3F7B2FFA8
:10CB6000F4F77BFB1E20FCF746FE00210846FCF78D
:10CB7000F9FDC8F8080001210020FCF7F3FDC8F812
:10CB80000C00002009FB07F4DFF88CA2002C88BF02
:10CB900047F6FF710AD9D8F8082022F810A0D8F873
:10CBA0000C2022F81010401C8442F4D81E20FDF7FF
:10CBB0003FF800210120FCF7D5FD834601210846FE
:10CBC000FCF7D0FD02460020AB1918BF47F6FF71F5
:10CBD00006D02BF810A022F81010401C8342F8D881
:10CBE000B8F804000026864238BF4FF0000B6FD221
:10CBF000FCF7F5FB01286BD00DF59260F4F703FE0E
:10CC000000285FD0DDF89404002857D098F802007F
:10CC100010F0100F0BD0DDF89454F7F72FF92A46D7
:10CC200001464B4610460097F7F714F822E0002320
:10CC3000CDF80CB0CDF800B0CDF804B0CDF808B008
:10CC40001A461946DDF89404FDF73DFF054698F8AD
:10CC5000020010F0200F03D0FDF72FFF054608E07B
:10CC6000F7F70CF92A4601464B4610460097F6F7AF
:10CC7000F1FF1DB30021002C88BF53461ED935F9A2
:10CC80001100B0F5004FA8BF47F6FF7003DA10F5AA
:10CC9000004FB8BF1846D8F8082032F911C08445B3
:10CCA000B8BF22F81100D8F80C2032F911C0844521
:10CCB000C8BF22F81100491C8C42E0D8F4F7C0FD2F
:10CCC000761C01E0F7F7C9FEB8F8040086428FD35E
:10CCD0000120F3F7B8FFFEF723F9B8F80400B042DB
:10CCE0001BD8DDF8AC0410F0020F16D000234FF66D
:10CCF000FF721846002C88BFD8E902C50DD93CF94F
:10CD0000101035F91060891B9942C8BF0B4691423B
:10CD1000B8BF0A46401C8442F1D8F4F725FA0DF258
:10CD2000B44DBDE8F08F2DE9F041364D002484B0BC
:10CD30006C703A4F4FF00108661EFCF750FB01285B
:10CD400006D1F7F74DFE03281CBF04B0BDE8F08103
:10CD5000287810F0010F05D0FFF755FB3C702C70C0
:10CD6000FCF739FB287810F0020F07D0FFF79DFE83
:10CD7000287820F002002870FCF72DFB287810F0AE
:10CD8000040F2FD0E8788DF801808DF8074048F621
:10CD9000B8018DF80040ADF804608DF808404843B4
:10CDA000ADF802608DF806408DF80940F6F733FDC6
:10CDB000FCF715FB01280DD00120F6F731F8F6F746
:10CDC00045FD0028F4D06846FDF7DBF80020F6F7B3
:10CDD0003AFDEDE7F6F731FD287820F002002870E3
:10CDE000FCF7F9FAF7F7FCFD0328A6D004B0BDE87C
:10CDF000F0810B490968A1F8E80070470149C87043
:10CE00007047000020070020BA050020BB05002065
:10CE1000BF050020C00500200080FFFF380700206C
:10CE2000F8060020FD48407A704700220028D8BF4D
:10CE30007047002100BF491C0829FBDB521C8242BD
:10CE4000F7DB70472DE9F04F002283B0F4490092E0
:10CE5000019291F804904F8AB1F810804E79B7FB97
:10CE6000F9FEB8FBF6FBB1F90E5094461446B9F141
:10CE7000000F18DD0021002E11DD01EB421330F907
:10CE80001330AB4207DD0CEB441A30F91AA05345BE
:10CE9000C4BF14468C46491C09B28E42EDDC511CBD
:10CEA0000AB29145E6DC5CEA04004FF0010355D07C
:10CEB000611CDB4A0CF1010000FB0BF0948A00B20C
:10CEC00001FB0EF1D58A09B204FB00FC9CFBF8F0D3
:10CED00005FB01F292FBF7F100B209B28045DCBF1D
:10CEE000A8F1010000B2B942A4BF791E09B2CD4A2F
:10CEF0001268926912F0040F14BF23EA020C02F0C8
:10CF0000010CBCF1000F02D0691A491E09B212F0DF
:10CF1000020F02D0201A401E00B212F0040F12BFFE
:10CF20000A460246084641218DF800108DF801306E
:10CF300011098DF8021001098DF8031002F00F019C
:10CF400061F31F108DF804000A208DF80500684673
:10CF5000FCF77CFF03B00120BDE8F08F43208DF883
:10CF6000000000208DF801308DF802008DF80400DB
:10CF70008DF803008DF805006846FCF767FF03B0E5
:10CF80000020BDE8F08FA54982B26FF30F00C1E920
:10CF900006027047A14800797047A04A0028D1696D
:10CFA00014BF41F0020021F00200D061704710B5BB
:10CFB00004465A20F4F7A9FF24B1012C08D0022C12
:10CFC0000CD010E015220021B120F4F7E2FE0AE0B7
:10CFD00019220021B120F4F7DCFE04E01D2200211B
:10CFE000B120F4F7D6FEBDE81040A520F4F78DBFC0
:10CFF00010B55A20F4F789FF80220021B620F4F7FB
:10D00000C8FE00220121B620F4F7C3FEBDE810409F
:10D01000A520F4F77ABF10B55A20F4F776FF112255
:10D020000021B620F4F7B5FE06220121B620F4F760
:10D03000B0FEBDE81040A520F4F767BF7A4810B5F0
:10D040000068C068754910F0040FC87A16D002282D
:10D0500008BF10BD0220C8725A20F4F756FF802284
:10D060000021B620F4F795FE00220121B620F4F746
:10D0700090FEBDE81040A520F4F747BF022818BF76
:10D0800010BD0120C8725A20F4F73FFF1122002181
:10D09000B620F4F77EFE06220121B620F4F779FED1
:10D0A000BDE81040A520F4F730BF5C48007FC0F316
:10D0B00040007047594AF02303EA0010D16921F07B
:10D0C000F0010843D06170475448007FC0F303105B
:10D0D0007047524A0028D16914BF41F0010021F085
:10D0E0000100D06170474D48007F00F0010070479B
:10D0F0004A4B99690A0E120721F07F4142EA00600B
:10D1000008439861704745488069C0F303607047E1
:10D1100044480068406DC0F30360704770B53F4CF1
:10D1200000256574A574A070F7F75AFC052818BF90
:10D1300070BDA078012804BF01206074A078022887
:10D1400018BF70BD032039490968C86102217F20DA
:10D15000F3F77AF91C210020F3F776F900BF00BF3E
:10D1600000BF1C210020F3F76FF900BF00BF00BF14
:10D1700016210120F3F768F900BF00BF00BF162198
:10D180000120F3F761F9A57470BD244880787047D9
:10D19000012101FA00F04FF47F0101EA00411F482C
:10D1A0008269114381617047012101FA00F04FF457
:10D1B0007F0101EA00411948826922EA0101816187
:10D1C000704716488069C0F3074070471348008BCA
:10D1D000C0F303307047114A4FF4704C0CEA003032
:10D1E0009169C1F3033321F47041084390611846FB
:10D1F00070470A48808BC0F38020704770B5074E97
:10D200000446C0F38000F569C5F30021884218BFC9
:10D21000F6F72FFE14F0040F0AE00000300700209C
:10D220008C100020F806002088AE11008CAE110092
:10D2300014BF45F4807025F4807014F0080F14BFFB
:10D2400040F4007020F4007014F0200F14BF40F47C
:10D25000806020F4806014F0100F14BF40F4006070
:10D2600020F4006014F0800F14BF40F0800020F024
:10D270008000F061BDE87040FDF738BFFA48C16931
:10D28000002011F0400F18BF012011F4807F18BF5B
:10D2900040F0040011F4007F18BF40F0080011F4C2
:10D2A000806F18BF40F0200011F4006F18BF40F0ED
:10D2B000100011F0800F18BF40F080007047EA485E
:10D2C000007FC0F340107047E748808BC0F3002018
:10D2D0007047E548808BC0F300307047E248C06972
:10D2E000C0F3003129B1C0F34010002804BF012071
:10D2F000704700207047DC490A6A10430862704793
:10D300002DE9F04789460446FDF7C4FB0546F4F7CE
:10D3100066FEF3F75EFED54903200968C861D44E66
:10D3200018274FF04A08FCB1012C34D0022C0FD042
:10D3300001217F20F3F788F818210E20F3F784F8F5
:10D340004A210820F3F780F886F8EE7686F8E8861A
:10D35000B9F1010F04BF0020F6F7BEFEF3F77DFF21
:10D36000BDE8F047F4F71EBE01217F20F3F76CF80B
:10D3700018210E20F3F768F84A210820F3F764F823
:10D3800086F8EE7686F8E88628780128E0D0012233
:10D390001146104617E001217F20F3F755F81021C0
:10D3A0000E20F3F751F872210820F3F74DF8102002
:10D3B00086F8EE06722086F8E80628780228C7D09C
:10D3C000012211460220FDF767FBC1E710B5A64C0C
:10D3D0006078002818BF10BD00210A20F4F79AFCDD
:10D3E00020701C2818BF10BD0020F5F724FDF3F7AE
:10D3F000F0FD0120607010BD2DE9F04F0027A3B0B3
:10D400007D1E2097CDE90655ADF84C708DF8507013
:10D410001195466819970446059780681690002074
:10D42000219004901AA8B846DFF83CA2BB4610979A
:10D430001890FDF72FFB1590169838B112AA11A974
:10D44000FDF7C8FC1790FDF7C3FC10909EB1894A08
:10D4500014A913A8069B8DE80F009AF9033007A9B9
:10D460003046189AFDF72FFB0590FDF726FB199023
:10D47000FDF726FB8346DAF81C004FF00109C0F3E4
:10D480004001002900F0CC807B49CDF804808968F8
:10D49000216809911999CDE90A1B1899CDF83080B6
:10D4A000CDE90E8110990D91BDF87C10ADF82010DA
:10D4B000DAF82010054641F4007410F0400FCAF865
:10D4C00020801CBF15F0040F44F0010415F4807F88
:10D4D00018BF44F0040415F4007F18BF44F008049A
:10D4E00015F4806F18BF44F02004FDF7FDFD0028FF
:10D4F00018BF44F0805415F4006F18BF44F01004B6
:10D5000015F4805F18BF44F0400415F0800F18BF79
:10D5100044F08004BAF81800C0F3033144EA014033
:10D52000002918BF40F48060002E08BF20F00100E1
:10D530000799B1F1FF3F08BF0127BDF84C1007293B
:10D5400015BF9AF807108AF807900129072108BF2C
:10D55000ADF84C109AF80F1021B90127B91E0791A8
:10D560008AF80F909AF80510012904BF0421ADF83C
:10D570004C100097BDF84C3001AA08A90AF073FEC0
:10D5800004460198806820F0080110F0080FCAF8DE
:10D59000241014BF8AF804908AF8048010F0100F49
:10D5A0000DD09AF8060050B915984FF00001007898
:10D5B00002280DD00120FFF7A3FE8AF805900198FC
:10D5C000007A10F0200F9AF80D000FD030B116E05D
:10D5D0000020FFF795FE8AF80690EEE78AF80D9096
:10D5E000012264210720FFF79CF908E0012806D1F9
:10D5F0008AF80D80002264210720FFF792F9019834
:10D6000001680029CCBF8AF803908AF80380002CB7
:10D6100006BF416800298AF80C8031D0019805685E
:10D6200007980028C4BFAAF814808AF80E8008DC86
:10D63000BAF81410B0F1FF3F0CBF891C491CAAF8BE
:10D6400014100E4F39680A7F12F0010F74D0497F11
:10D65000BAF814208A422ED8DAF83420012A18BFEA
:10D66000B0F1FF3F68D126E0300700208CAE1100FA
:10D67000B059002040070020A8160020F80600201E
:10D68000007A4FF0640110F0400F04D0CDF81C80F8
:10D690008AF80C10C2E79AF80C0030B1401CC0B2F6
:10D6A0008AF80C006428F1D2B8E70798012808BF6F
:10D6B0008AF80C90B2E7AAF814808AF80780BAF8C2
:10D6C0001400814204D2012299210720FFF729F991
:10D6D000DAF83400012804D1022299210720FFF74B
:10D6E00020F90798B0F1FF3F04D1032299210720C8
:10D6F000FFF717F96EB1DDE92001CDE9001BCDE997
:10D700000250DDE90610DDE90432F7F747F98AF83F
:10D710000C80179828B1DAF82C2001461198F7F7F9
:10D720001BF915980078022807D002228AF8068093
:10D7300011460320FDF7B0F91AE09AF80E00401CDC
:10D74000C0B28AF80E00142809D914208AF80E00F5
:10D7500000218AF806800846FFF7D2FD08E003287A
:10D7600006D902228AF8058011460320FDF794F9B4
:10D77000FE4C2078242804BF1998FCF729F920785A
:10D78000012804BF1998FCF723F920780E2804BF5C
:10D790001998FCF71DF9169800281CBF9AF810007C
:10D7A000022811D0386890F86C0010F0010F0BD0EF
:10D7B000DDE91021BDF94800FDF744FC00281EBF3B
:10D7C000012023B0BDE8F08F0798DAF82810491C33
:10D7D000CAF828100028C8BFCAF82C8010D09AF8C0
:10D7E0001C1011F0010F6FD0DAF81810C1F30364A8
:10D7F0002546062C59D2DFE804F0091118583A3AA8
:10D80000DAF82C10491CCAF82C10E8E700284DDD86
:10D81000022000F0F8FA48B3022449E0002845DD70
:10D82000022000F0F0FA08B3F6E7002818BFCAF8A3
:10D8300034803BD1012000F0E6FA002818BF012413
:10D8400036D13868DAF82C10B0F85C00884206D37C
:10D85000DAF83400012808BFCAF8348026D1002045
:10D8600000F0D1FA002818BF002421D11EE00028C2
:10D8700006DD022000F0C7FA002818BF022415D1E7
:10D88000042D0ED1DAF81C00C0F3003149B1C0F309
:10D89000401030B9052000F0B6FA002818BF052462
:10D8A00006D1002000F0AFFA00B10024AC420BD04A
:10D8B000DAF81800C846010E090720F07F4041EA57
:10D8C00004610843CAF8180023B04046BDE8F08F51
:10D8D000F0B587B00746F7F783F80546F7F783F802
:10D8E000A3490646052D0CBFA24CAFF2F344C8690C
:10D8F000C0F3031118BF052E08D1C0F300322AB1BE
:10D90000C0F34010002808BF41F002013846F7F785
:10D9100036F9002804BF07B0F0BDF6F77AFA0746DB
:10D920000020F3F7CFF8F3F798FCFBF758FD012838
:10D9300009D0F7F755F8A84205D1F7F754F8B042E7
:10D9400008BF002F05D0F3F744FBF7F79BF907B0AA
:10D95000F0BD6846F3F757FF40B16846FCF79FF902
:10D960006846A0470746F3F76BFFDEE7F7F76AF86C
:10D97000DBE7F0B57E4E87B00027B0690225C0F323
:10D980000364306A40F480703062F4F70BFB0220CD
:10D990000AF055FDFBF723FD01280AD0F7F720F820
:10D9A000022806D1B069C0F30360A04208BF002F6F
:10D9B00029D0F7F715F802280BD10120F0746E4832
:10D9C000A0210268116101680968006841F0020144
:10D9D0000160F4F704FBF7F703F8052804BF002003
:10D9E000F2F710FEF6F7FCFF022805D0F6F7F8FF75
:10D9F00005460220F7F703F8022D1CBF2846F6F76C
:10DA0000FEFF07B0F0BD6846F3F7FDFE0028C1D069
:10DA10006846FCF744F96846FFF7EEFC0746F3F763
:10DA20000FFFF4F7F6FAB5E72DE9F04F89B0F5F7F7
:10DA3000FFFC52480AF0F7FAFDF789FA504C2068CB
:10DA4000B0F93610B0F93400FCF7D6FF4D484FF06E
:10DA5000010B80F8C0B64C4880F8C0B62068B0F81A
:10DA60005800C0F303200F2818BFF6F7ECF9DFF8D1
:10DA70000081D8F81C0040F00100C8F81C00F6F73F
:10DA8000AFFF022804BF4FF00009DFF8ECA040F020
:10DA90002C81D8F81800C0F303653948A900006844
:10DAA000806DC8F82890C84000F00F00C8F82C908E
:10DAB000C8F83090062D80F00F81DFE805F0D00324
:10DAC0000303D3D30790D8F81C0000260227C0F325
:10DAD0000314022D0BD1C0F3003131B1C0F340105B
:10DAE000002808BF44F0020401D024F0020498F892
:10DAF0000800012819D021460798F7F740F80028B8
:10DB000000F0EA80F8F78AFAF8F764FB0020F6F7ED
:10DB1000E3FA88F808B01D48F3F7FAF8FDF700FAC1
:10DB200098F80A0001283ED10AE098F80A00012876
:10DB3000F1D1F6F7CEFF21460798F6F7E4FFEAE7C2
:10DB4000D8F81C0040F00200C8F81C00D8F82000EB
:10DB500040F00100C8F820000020F3F7CEF8DAF812
:10DB60000000806840F0020012E000002D06002056
:10DB700030070020EBA11000A8AE11008C1000208F
:10DB8000F8060020B059002078080020C99911003B
:10DB9000DAF800108860F3F760FB88F803900AF069
:10DBA0002BFA88F80A90F4F7FDF901200AF047FCF7
:10DBB000FBF715FC01280BD0F6F712FF022807D15E
:10DBC000D8F81800C0F30360A84208BF002E35D073
:10DBD000F6F706FF02280DD188F813B0DAF8001026
:10DBE000A0200861DAF800000068DAF8001040F0C0
:10DBF00002000860F4F7F3F9F6F7F2FE052804BF17
:10DC00000020F2F7FFFC0020F3F782F8F5F715FE8D
:10DC1000F6F7E6FE022805D0F6F7E2FE07460220F8
:10DC2000F6F7EDFEF6F7DCFE052808BFF7F72AF851
:10DC3000022F1CBF3846F6F7E2FE4DE06846F3F7C8
:10DC4000E2FD0028B4D06846FCF729F86846FFF7E3
:10DC5000D3FB0646F3F7F4FDF4F7DBF9A8E7FFF78B
:10DC600088FE39E00746F6F7BBFE0546F6F7BBFE31
:10DC70000646052D0CBF714CAFF68304D8F81C0086
:10DC8000C0F3031118BF052E08D1C0F300322AB12A
:10DC9000C0F34010002808BF41F002013846F6F7F3
:10DCA0006EFFC8B1F6F7B5F807460020F2F70AFF95
:10DCB000F3F7D3FAFBF793FB012809D0F6F790FEB0
:10DCC000A84205D1F6F78FFEB04208BF002F11D051
:10DCD000F3F77FF9F6F7D6FFFBF781FB012804D0B5
:10DCE000F6F77EFE02283FF4D4AE09B0BDE8F04F4F
:10DCF000FDF72DB96846F3F786FD40B16846FBF79E
:10DD0000CEFF6846A0470746F3F79AFDD2E7F6F73D
:10DD100099FECFE72DE9F04F002485B048490494DF
:10DD200023460E78009401940294224604A9039499
:10DD3000FCF7C9FEFCF7C1FE0546002700940194DC
:10DD4000F6F74EFE3F490528096851D0888FB1F893
:10DD50003EA0C0F30B09000BB9FBF0F80020711EC8
:10DD600004468446EE46029100210CFB06F3002E89
:10DD70002ED935F913203EF91CB0934505DA0DF183
:10DD8000040B2EF81C202BF81C104A451BDD3A44CE
:10DD900031B105EB430737F9027C3A44474500DDD2
:10DDA0000120029FB94206D205EB4307B7F9027082
:10DDB0003A44474500DD012401280CBF012C52459F
:10DDC000A4BF012204920027491C5B1CB142D0D39E
:10DDD0000CF1010CBCF1020FC6D31B4800780128DE
:10DDE00004BF2846FBF7F4FD049805B0BDE8F08FAA
:10DDF000B1F80001B1F802A1C0F30B09000BB9FBA7
:10DE0000F0F8ABE77047114A0228117F9269C1F31D
:10DE10000311C2F3074205D0012808BF11F0020F19
:10DE20000AD002E011F0040F06D0012101FA00F03F
:10DE3000104018BF0120704700207047EBA1100070
:10DE4000BA050020F80600202D060020300700202B
:10DE50004FF6FF71A0F8B410A0F8B610A0F8B810F3
:10DE6000A0F8BA10A0F8BC10A0F8BE10A0F8C0101E
:10DE7000A0F8C21070472DE9F04F85B005F0BCF94D
:10DE8000049005F0AFF900252C46009005F0D2F97A
:10DE90000098007D01280CBF4FF4DE71DE21009850
:10DEA000FF4A4FF00008407C012888BF82F80080BC
:10DEB0001CBF05B0BDE8F08F4FF000070098007C54
:10DEC00000289CBF05B0BDE8F08F049800EB072048
:10DED00090F8FCC0BCF1020F18BFBCF1030F40F07A
:10DEE0007E81EF4E3278039252B3EE4BF27802927B
:10DEF00033F822B0B0F8B630BBEB030954BF4A4642
:10DF0000A3EB0B028A42B8BF0124DFF89CA3E44ACA
:10DF1000127901923AF822A0B0F8B420BAEB0206C6
:10DF20004CBFA2EB0A0EB6468E45B8BF0125BCF128
:10DF3000020F1ED0BCF1030F00F0F38000F0DFB839
:10DF4000BCF1020F40F04B810122D64B3270B0F889
:10DF5000B6C0A3F800C05A80B0F8B430D2480380ED
:10DF600042807270B27086F8038086F8048000F0F8
:10DF700036B954EA050C04D0002C71D0002D6ED0B7
:10DF8000BDE0C74E4FF0000AD44696F80190B9F1B3
:10DF9000000F88BFDFF80CE328D93EF82CB0BBEBAC
:10DFA000030648BFA3EB0B068E4216DABC4E86F87A
:10DFB00003C0019A521CD2B23271B3785B1CDBB23F
:10DFC000B3700F2B28BF86F8008080F00881B64B15
:10DFD00003EB8202A2F8028091E00CF1010C0CF03C
:10DFE000FF0CCC45D9D3BAF1000F51D1DFF8B0C244
:10DFF00000239CF802B0BBF1000F88BFDFF8A8E255
:10E0000028D93EF82360B6EB020C48BFA2EB060C01
:10E010008C4518DADFF888C28CF80430029A09F1CE
:10E020000103521CD2B2DBB28CF803208CF8013011
:10E030000A2B02D38CF80080D1E09A4B03EB8202CA
:10E04000A2F802805BE05B1CDBB25B45D9D3BAF17E
:10E05000000F54D1924880F80080C0E000E02EE02C
:10E06000DFF83CE24FF0000A52469EF80190B9F109
:10E07000000F88BFDFF82CB212D93BF82260B6EB54
:10E08000030C48BFA3EB060C8C4502DA8EF8032084
:10E0900035E0521CD2B24A45EFD3BAF1000F2ED16F
:10E0A000029A09F10103521CD2B2DBB28EF80320AE
:10E0B0008EF801300A2BC0D38EF800808FE0DFF895
:10E0C000E0E14FF0000A53469EF80290B9F1000FCC
:10E0D00088BFDFF8D4B117D93BF82360B6EB020C48
:10E0E00048BFA2EB060C8C4502DA8EF8043006E03D
:10E0F0005B1CDBB24B45EFD3BAF1000F04D0039A9F
:10E10000674E012A1FD06AE0019A09F10103521CEF
:10E11000D2B2DBB28EF804208EF802300F2BCBD2B5
:10E1200055E7DFF87CC1B9F1000F48BFA3EB0B093D
:10E130008945BFF67FAF002E48BFA2EB0A068E428C
:10E14000BFF678AFDBE7DFF85C91F27809EB820C81
:10E15000BCF80230F3B342F2107A53450DD2B0F856
:10E16000B6A039F822B00BFB03AA5B1C9BB2ACF83B
:10E170000230BAFBF3F329F8223039F82230B0F834
:10E18000B6209B1A03EBD37302EB6302A0F8B62010
:10E19000DFF81491327909EB820CBCF8023083B3BA
:10E1A00042F21076B3420DD2B0F8B46039F822A032
:10E1B0000AFB03665B1C9BB2ACF80230B6FBF3F3C0
:10E1C00029F8223039F82230B0F8B4209B1A03EB3A
:10E1D000D37300E00DE002EB6302A0F8B420781CDA
:10E1E000C7B20098007CB8423FF66FAE05B0BDE8FC
:10E1F000F08FB0F8B63029F822300122ACF80220B6
:10E20000C6E7FFE7B0F8B40029F822000120ACF817
:10E210000200E4E72DE9F04704F0EEFF044604F0C5
:10E22000E1FF0246007D01280CBF4FF4DE7078202C
:10E23000517C1E4D0026A5F10C07012907D098BF7F
:10E24000BDE8F0873E722E806E80BDE8F08792F8C0
:10E2500010C04FF00001BCF1000F98BFBDE8F0877F
:10E2600004EB012292F8FC30022B18BF032B05D0DF
:10E27000491CC9B28C45F3D8BDE8F0873B7A012B25
:10E280001ED0002B18BFBDE8F08704EB012090F8EA
:10E29000FC00022818BFBDE8F0870120387207E0B3
:10E2A0007007002000790020287900207C070020DA
:10E2B000B2F8B4002880B2F8B6006880BDE8F087F4
:10E2C00004EB0123B5F80090B3F8B430B5F8028040
:10E2D000A9EB03030FFA83FCB2F8B630BCF1000FD0
:10E2E000A8EB03031BB2B4BFCCF1000AE2465045D1
:10E2F0003ADB002BB4BFC3F1000A9A46824533DCF7
:10E3000092F8FC00022816D042F6AB200CFB00F07D
:10E310000114A1EBE07142F6AB2058430314A3EBC8
:10E32000E070A9EB0101A2F8B410A8EB0000A2F87C
:10E33000B600BDE8F08746F267600CFB00F04114C0
:10E34000A1EBE07C46F2676058434114A1EBE07119
:10E35000A9EB0C00A2F8B400A8EB0101A2F8B610DA
:10E3600028806980BDE8F0873E722E806E808CE741
:10E370002DE9F04F83B004F03FFF044604F032FF74
:10E38000074604F057FF019004F058FF0090787C96
:10E39000FF4E01254FF0000A01280DD09CBF03B0AD
:10E3A000BDE8F08F757186F807A003B04FF001004B
:10E3B000BDE8F04F02F078BA707998B1397C00204E
:10E3C00000299CBF03B0BDE8F08F04EB002292F857
:10E3D000FC20022A71D0401CC0B28142F5D803B0A3
:10E3E000BDE8F08F97F810B00023BBF1000F9CBF81
:10E3F00003B0BDE8F08F4FF0020EDFF8988308F10C
:10E40000060904EB032090F8FB10022905D003292C
:10E4100004BFB17902292BD077E004EB03210978FE
:10E42000012914D9019A921E914210DA41780129EA
:10E430000DD9009A921E914209DA757186F807A0EB
:10E44000012002F031FAB57103B0BDE8F08F86F813
:10E4500006E0B0F8B410A9F80010B0F8B600A9F8BA
:10E46000020088F800A088F801A003B0BDE8F08F92
:10E47000B9F80010B0F8B470B0F8B600CA1BB9F81B
:10E480000210A1EB00014CBFC2F1000C9446BCF19C
:10E49000F00F1CDD98F800C0BCF1000F06D0BCF1F5
:10E4A000010F0BD0BCF1020F0CD00EE0002AB4BF5C
:10E4B00088F8005088F800E007E02EE0002A3FF7D7
:10E4C00071AF02E0002AFFF66DAFA9F800700029D5
:10E4D000B4BF4A420A46F02A17DD98F8012022B15B
:10E4E000012A09D0022A0BD00DE00029B4BF88F818
:10E4F000015088F801E006E000293FF753AF02E041
:10E500000029FFF64FAFA9F80200581CC3B29B4583
:10E510003FF677AF03B0BDE8F08F86F807A003B0F1
:10E52000BDE8F08F2DE9F04104469B480068858ADC
:10E5300004F076FE09F042FF074609F045FF064663
:10E5400009F048FF002808BFBDE8F08194F8FC00FE
:10E5500002281CBF0328BDE8F081B4F8C2000121E5
:10E56000B84202D9AA1B904207DB94F8E8000028C1
:10E5700004BF84F8E710BDE8F081002084F8E700CC
:10E5800084F8E810BDE8F0812DE9F04FADF5197D74
:10E5900004F032FE939004F025FE064604F034FEAB
:10E5A000044604F03DFE929006F1170004F11705B1
:10E5B000909004F03FFE00279190307C3C463B4613
:10E5C00000287BD99398929A00EB032191F85B0085
:10E5D00002EB002A91F8E900012870D191F8FB9034
:10E5E000B9F1020F18BFB9F1030F68D1601CC4B2B2
:10E5F00091F85920694800EB820C3CF8048CA8F58E
:10E600007F40FF381FBF3CF8022CA2F57F40B0F1DD
:10E61000FF00404604BFBAF80600BAF80820B9F176
:10E62000030F6ED1B1F80690CDF8549209F1050AA6
:10E63000DFF86C91A9FB0ABACAF3CF0ECDF860E2FD
:10E64000B1F808E0CDF850E20EF1050AA9FB0ABACC
:10E65000CAF3CF0ACDF85CA200F1050AA9FB0ABAF9
:10E66000CAF3CF0B02F1050AA9FB0AA9C9F3CF0A25
:10E67000DDF854924CF6CD4E09FB0EF94FEAD9491C
:10E68000CDF85892DDF850E24CF6CD490EFB09F971
:10E690004CF6CD4E02FB0EFE4FEAD9494FEADE4E54
:10E6A000CDF85492CDF850E24CF6CD49DDF860E259
:10E6B00000FB09F94FEAD949DE4501E029E020E0F5
:10E6C00004BFDDF85CB2D34507D0DDF858A2CA45D7
:10E6D00004BFDDE9949ACA4513D17F1CDFF8BC90D2
:10E6E0004FF6FF7AFFB2D04504BF3CF8028CD0450C
:10E6F00007D12CF8040C91F8590009EB800020F8A0
:10E70000022C581CC3B2307C98423FF65BAFA74244
:10E710007ED1707C02287BD31D49487A401CC0B250
:10E7200048721E283CBF0DF5197DBDE8F08F1E20F4
:10E7300048724FF41072684690990BF020F8307CC4
:10E740004FF0000B002877D99398929A00EB0B2199
:10E7500091F85B0002EB002291F8E900012864D1F6
:10E7600091F8FB00022818BF03285ED10B7891F8BE
:10E7700001C091980CFB00339098C05C0B7B00F0BB
:10E780003F0A107B984238BF0873507B4B7B09E0EF
:10E79000700700207A0700205808002064790020C4
:10E7A000CDCCCCCC984238BF4873907B8B7B9842C1
:10E7B00088BF8873D07BCB7B984288BFC873087BA7
:10E7C00095904C7B9494137892F801C0919A91F8AB
:10E7D0000F800CFB0232887BAA5C444502F03F09A3
:10E7E0001CD8919A624397B2959A824212D8BB186C
:10E7F00015F803C00CF03F0ECE4505D12CF03F0CB0
:10E800004CEA0A0C0DF803C0521C92B2824200E09E
:10E810001CE0ECD9621C94B24445E2D9959A0A7383
:10E82000949A4A73887381F80F800BF1010000F00D
:10E83000FF0B307C584587D84FF41072694690988A
:10E840000AF09DFF0DF5197DBDE8F08F7B48002192
:10E850007B4A417208464FF6FF7122F8201002EB06
:10E860008003401CC0B259800A28F6D30DF5197DEB
:10E87000BDE8F08F2DE9F35F834604F0BDFC074649
:10E8800004F0CEFC804604F0ADFC054601984FF044
:10E890000009002879D1287C05F1170A002874D0D6
:10E8A000FFF772FE287C0024002888BF4FF6FF7611
:10E8B0001ED907EB042292F8E900012813D1A2F82F
:10E8C000B460A2F8B660A2F8B860A2F8BA60A2F884
:10E8D000BC60A2F8BE60A2F8C060A2F8C260514657
:10E8E000584602F023FC601CC4B2287CA042E0D849
:10E8F000002610F0FF0F18BF4FF0020A45D007EBBB
:10E90000062494F8FC00022818BF03280ED094F8BF
:10E91000FD00022818BF03282AD095F862020128BA
:10E9200004BF94F8FB00022822D029E0204600F022
:10E93000F4FF94F89D00012822D194F85B0008EBC5
:10E94000002090F8FC10022918BF032918D1B43018
:10E95000B434B0E80E10A4E80E10B0E80E10A4E82D
:10E960000E100FC80FC404F860AC04F8809C07E0D8
:10E97000B4F8B400A4F8B800B4F8B600A4F8BA002B
:10E98000701CC6B2287CB042B9D8287C002400286C
:10E9900017D907EB042090F8E91001290CD190F861
:10E9A000FB10022918BF032906D190F8F4100029A2
:10E9B00004BF019901F094FA601CC4B2287CA04203
:10E9C000E7D8002610F0FF0F12BF4FF0010902B088
:10E9D000BDE8F09F07EB06241A480068B0F81480E1
:10E9E00004F01EFC09F0EAFC834609F0EDFC8246C7
:10E9F00009F0F0FCC8B194F8FC00022818BF032805
:10EA000013D1B4F8C200584503D9A8EB0A018842D3
:10EA100006DB94F8E800002808BF84F8E79004D0EB
:10EA2000002084F8E70084F8E890701CC6B2287CC7
:10EA3000B042CFD802B0BDE8F09F000070070020C0
:10EA40006479002058080020F9484078002818BF51
:10EA500001207047F748006890F8580000F0010066
:10EA60007047F44909688A6D60F300028A6570474F
:10EA7000F04B10B4D3F800C0BCF8123003FB00F424
:10EA8000BCF81A005943B4FBF0FCB1FBF0F10CFBED
:10EA90000CF4DFF8A4C34943CCE9084103FB02F1BD
:10EAA000B1FBF0F04043CCF8280010BC70474FF6A3
:10EAB000FF7202EA0023E04802EA0121C3850186D1
:10EAC0004FF4A05141864910818670472022DA49CF
:10EAD00006280ED2DFE800F00D030D05080A10200D
:10EAE00000E04020888570478020FBE74FF480706D
:10EAF000F8E78A85704700B5022205210B20FFF751
:10EB0000B7FFDFF830C30A231422DCF8000090F8C6
:10EB10005C00C0F3031100F00F00FFF7C8FFDCF842
:10EB20000000B0F85C005DF804EBC0F30330CDE703
:10EB30002DE9F04190460D46044604F053FBBF48D2
:10EB4000BC4E47190A380544BCB1012C3AD0022CFE
:10EB50004DD0032C18BFBDE8F08104220E210F20F8
:10EB6000FFF786FF30680A231422B0F85C00C0F378
:10EB700003200146FFF79BFF1CE0022205210B202A
:10EB8000FFF776FF15F8010C002801BF17F8010CFC
:10EB9000002898F8FB00032830684FF00A034FF074
:10EBA000140290F85C00C0F3031100F00F00E1D1F3
:10EBB000FFF77DFF3068B0F85C00BDE8F041C0F3BE
:10EBC000033083E702220E210F20FFF751FF306848
:10EBD0000A231422B0F85C00C0F3032100F00F00F8
:10EBE000491CFFF764FFBDE8F04104206EE715F80B
:10EBF000010C012804BF17F8010C01284FF0040292
:10EC000019BF112112200C210D20FFF731FF15F83B
:10EC1000010C02283068C06D18BFC0F30351C0F367
:10EC200003404FF00A034FF0140208BF0321FFF71F
:10EC30003EFF3068C06DBDE8F041000F46E730B5DB
:10EC40007C4C7B4D02222068418A408B8900B1FBBD
:10EC5000F0F04043A86005210B20FFF709FF206872
:10EC60000A23142290F85C00C0F3031100F00F0097
:10EC7000FFF71DFF2068B0F85C00C0F30330FFF71A
:10EC800025FF05F110014FF6FF700880488005F15F
:10EC90000C004FF0FF31018041800020287030BD12
:10ECA000654B03EB400003898B4288BF991A38BF3C
:10ECB000991808BF7047018170472DE9F04F83B064
:10ECC0001F460E46044604F08DFA04F0A9FA844665
:10ECD000584894F85950564B0068574A4FF0000B6B
:10ECE000418A408BC1EB0111890091FBF0F094F84F
:10ECF000FC104043022911D0A2F1500101EBC501E3
:10ED000051E902A9318801917188009194F8581055
:10ED1000022994F8E11012D011B331E05119B6F87C
:10ED200000A0B6F8029001F801BC02EB4508918EF4
:10ED3000A8F80810012D08BF83F801B0E2E7F9B187
:10ED400094F85B100CEB012191F8E110C1B902EBD2
:10ED50004501B2F830C0B1F80880E04510D90DE0A7
:10ED6000874224BF94F8FC10032909D102EB450126
:10ED7000B2F830C0B1F80880E04501D9A1F808C068
:10ED80002179022918BF032906D094F8E11019B996
:10ED9000874238BF918E00D3518E518694F8E1108E
:10EDA00041B9874294F8FC0002D2032810D101E057
:10EDB00002280DD08846D2F828C0BC4588BF4FF045
:10EDC00002085878002804BF012D03290CD102E065
:10EDD0004FF00208EFE70120587017484189108E64
:10EDE000814284BF144948813846136A0C991746FA
:10EDF0004FF0030E834204D8B8F1020F01D001296D
:10EE000006D07A6A824227D9B8F1020F34D123E0C2
:10EE100094F8E000032804BF94F8C40000280FD041
:10EE20007919012001F8010C042084F8E00031E098
:10EE30008407002058080020DC7900201E7A00207A
:10EE40007919022001F8010C84F8E0E094F8C4007C
:10EE5000411C84F8C4103CE071B1824298BF9842D2
:10EE60002ED2B8F1020F2ED0781984F8C4B010F861
:10EE7000011C03291ED02CE094F8E000042804BFF4
:10EE800094F8C400002808D00220791901F8010C78
:10EE900084F8E0E084F8C4B01BE07919012001F89F
:10EEA000010C042084F8E00094F8C400401C84F8AD
:10EEB000C4000EE0022100F8011C84F8E0E008E044
:10EEC000B8F1020F05D1781900F801EC022084F89E
:10EED000E00004F087F97A19864612F8012CB88D03
:10EEE000398EB7F82EC07B8E022A04D0012A19D0A1
:10EEF000032A6BD02CE007EB450201EB4103B2F88B
:10EF000008C09C4505D99EF80AC0BCF1000F08BF97
:10EF1000138113898B4288BF181A38BF184417D041
:10EF2000108115E007EB45031A89914209D2501A66
:10EF3000A2EB6000000A4FF6FF7101EA0020188181
:10EF400006E0624588BF101A38BF104400D018810F
:10EF500007EB45000089002804BF0021084623D0A4
:10EF60000146B0F5807F36BF4FF480720A464FF4F9
:10EF70008070FE4994F85930B8F1020F18BF03F8B9
:10EF800001B02DD0A2F5807101FB0AF3019903EBCA
:10EF90000121B1FBF2F1A0F5807202FB09F3009AA6
:10EFA00003EB0222B2FBF0F094F85930F04A02EB86
:10EFB000C30343F8081C94F8593002EBC30242F82B
:10EFC000040CB180F08003B0BDE8F08F07EB450280
:10EFD0001189994288BF081A38BF0844A0D1B7E701
:10EFE00013F801C0BCF1FA0F3CBF0CF1010C03F89F
:10EFF00001C0C7E72DE9F04F90F859C08FB04FF42A
:10F00000806300290CBFDB4CDB4C04EB4C14DB4D64
:10F01000029205EB4C1705F5A5756544203C15F8E3
:10F02000015C07EB051606EBC10858F8206C921B33
:10F03000039290F8FC0002287ED058F81C8C04EB58
:10F04000051206EB0809CDF83090D2F80490D66886
:10F050009568106809EB0602DFF8249328441044F1
:10F06000D9F800A035445044D9F804A05244D9F846
:10F0700008A0D9F80C9055444E44DDF808A0DDF8FE
:10F080003090AAEB0909CDF82090DDF80C90DFF85C
:10F09000F4A2A9EB0809CDF82C90DAF8009009EB5E
:10F0A000000ECDF828E0DAF80490DAF808B0DAF8C3
:10F0B0000CA09144B244AB440EFB0AFE09FB1BEECC
:10F0C0009EFBF3FEBEF1000F08BF4FF0010E4FEAAA
:10F0D0008A2A9AFBFEFA4FEA892999FBFEF9CDF8B4
:10F0E00038A0C9F1000A4FEA8B29CDF834A0DDF829
:10F0F00028A099FBFEF94FEA8A2A9AFBFEFBDDF86D
:10F1000038A0C9F1000900FB0AFA02FB09AA9AFB20
:10F11000F3FEDDF834A0CDF828E000FB0AFA02FB8C
:10F120000BAA9AFBF3FECDF824E0DDF838A005FB2E
:10F130000AFA06FB09A900E05DE099FBF3F9DDF8A6
:10F1400034A0CDF8389005FB0AF906FB0B9999FB22
:10F15000F3FADDF828E0DDF820900EFB09FBDDF87E
:10F1600024E0DDF82C900EFB09BEDDF820B0DDF8C0
:10F1700038909EFBF3FE09FB0BFBDDF82C900AFB9D
:10F1800009B999FBF3F9C844DDF830B0DDF83890DF
:10F19000F344CDE900B8DDF828E0C9F10009CEF567
:10F1A0008068DDF824E0CAF5806ACEF1000B08FB28
:10F1B00000FE0BFB05EE08FB02F809FB00F00BFB61
:10F1C00006880AFB05009EFBF3FE98FBF3F890FB14
:10F1D000F3F0CDF810E0CDE9058009FB02F00AFB61
:10F1E000060090FBF3F0079067480022E84604AE63
:10F1F00000EB0C0315E0644A00206244039012F80F
:10F20000012C02AB07EB021202EBC10253F82040C3
:10F2100002EB8005401C00B245F8204C0228F5DBCB
:10F2200020E013F8015C58F8220007EB051505EB08
:10F23000C10505EB820545F8200C002006EBC20550
:10F2400013F801AC55F8209004EB0A1A0AEBC20A35
:10F250004AF82090401C00B20228F1DB501C02B298
:10F26000022ADEDB4848604410F8010C07EB00106E
:10F2700000EBC10050F8200C0FB0BDE8F08F70B467
:10F28000012803BF022401204FF0000C04241CBFFE
:10F2900003204FF0010C00263C4D0029C8BF20463A
:10F2A00009D00CEB8C0105EB810101EB420121F847
:10F2B000026C70BC704736480CEB8C0100EB4100CF
:10F2C000104405EB810101EB420210F8010C32F809
:10F2D000021C642924BF70BC7047491C22F8021C20
:10F2E0000121197070BC70472DE9F0010128DDE99A
:10F2F000055614BF0120002000EB8000DFF890C00D
:10F300000CEB400C8C441CF801CCBCF1000F04BF8A
:10F31000BDE8F0017047DFF87C80002408F13C076D
:10F32000944548D1A7F1280202EB800202EB41028A
:10F3300032F8022C9A4207D908EB4000084400F842
:10F34000014CBDE8F001704708EB40020A4412F896
:10F35000013C642B24BFBDE8F0017047002E1CBFA8
:10F36000BDE8F00170475B1CDBB215E0D17A0020EC
:10F370008C790020DC7A00201C7C00205C7D002041
:10F38000C0070020D00700209C7E00209A8000202B
:10F39000728000208680002002F8013C0A2B3CBFCE
:10F3A000BDE8F001704707EB4000084400F8014C4D
:10F3B000BDE8F001704708EB40020A4407EB40004B
:10F3C00012F8013C0844052B36BF10F8011C00F868
:10F3D000014C642904D20A2DA4BF491C00F8011C69
:10F3E00002F8014CBDE8F00170472DE9F04F89B0FB
:10F3F00082460888ADF8100048888946ADF81400A8
:10F4000003F0F0FE00909AF8FC009AF859400228A8
:10F4100004BF204600F0BBFDF948FD4A2044089097
:10F4200010F8015CF748F949204402F1080C00F893
:10F43000015CF54800EB040818F8010CD8B1681C11
:10F44000C0B2142821D304EB840001EBC00000EB10
:10F45000450330F828EC33F828BCAEEB0B0B02EB7D
:10F46000840E4EF804BC1B8D008DC01A0CEB840377
:10F4700043F8040C20E002EB8403002043F8040C62
:10F480000CEB840343F8040C16E004EB840301EB5B
:10F49000C30303EB400030F8283C30F82ABCA3EB50
:10F4A0000B0302EB840B4BF8043C038DC08C181A41
:10F4B0000CEB840343F8040C04EB840001EBC00064
:10F4C000079000EB4500BDF8103020F8283CBDF84F
:10F4D00014B0A0F828B0132D04BF012008F8010CC7
:10F4E0009AF8FC0003284FD1002D1CBF681EC0B243
:10F4F0005AD0079901EB400030F8281C008DA3EB8F
:10F50000010118F8013CABEB00000193002B52D035
:10F51000C04B002903EB840656F8047CACBF0B46B5
:10F520004B4207EB030BBC4B46F804BC03EB8403D4
:10F53000002853F804ECB4BF47420746774402EB77
:10F54000840243F8047C52F8042C002AB8BF5242CB
:10F55000ABEB020246F8042C0CEB840252F8042CAC
:10F56000002AB8BF5242BA1A43F8042CAB4A1268B8
:10F57000138B5943138A91FBF3F6518B4843518AFD
:10F5800090FBF1F7019878B3A5480221204406903A
:10F5900000F8011CA34800EB040B0BF8011C9AF8BF
:10F5A000E100032842D13EE018F8010C01280CBF0D
:10F5B000132028469DE7974A002902EB840252F85F
:10F5C00004CCB4BF4B420B46634442F8043C924A1D
:10F5D000002802EB840252F804CCB4BF4342034635
:10F5E000634442F8043CC1E7FFE78F48002E00EB7C
:10F5F000440030F8022CB4BF714231468A4205DA29
:10F60000002EACBF3146714220F8021C4288002F08
:10F61000B4BF794239468A42B6DA002FACBF3946C8
:10F6200079424180B0E703F086FE68B1204600F0E1
:10F63000AEFCBDF81000A9F80400BDF81400A9F84C
:10F64000060009B0BDE8F08F18F8010C012803D0BE
:10F65000D8B9691C072918D3282ED8BF282F09DC50
:10F66000714901EB440131F8022C282A9CBF4988DA
:10F67000282919D9009890F85A02012805D106992D
:10F68000032001F8010C0BF8010C0898089910F8F8
:10F69000010C401CC0B201F8010C1428C9D3089910
:10F6A000002001F8010CC4E75A494FF0000C01EBAF
:10F6B000840151F8042C584901EB840151F8041CD1
:10F6C0008A42C8BF4FF0010C05A904AA1423CDE952
:10F6D0000003CDE9022107982B4600F12802A0F192
:10F6E0002801604600F07BFC01280CBF01200020AF
:10F6F000069901F8010C0BF8010CC6E7DDF800C013
:10F700008A4204BF4FF0FF307047ACEB030C401A45
:10F710000CFB00F0511A90FBF1F0184470472DE9F2
:10F72000F04F5F1ADDE90A45DDF824C0161ADDF84E
:10F7300030800CEBDC7C4FF0FF39012C07BF4FEA27
:10F740006C03A0EB030C4FEA6C02A1EB020C4FF030
:10F7500000041CD08B4208BFCA4607D0ACEB010A9C
:10F7600006FB0AFA9AFBF7FB0BEB000AA0EB0A0B6D
:10F770000BFB0BFEA1EB0C0B0BFB0BEBC34532DAC7
:10F7800002EBD2724FEA6202ACEB020C30E0824232
:10F7900008BFCA4607D0ACEB000A07FB0AFA9AFB7F
:10F7A000F6FB0BEB010AA0EB0C0B0BFB0BFBA1EB2D
:10F7B0000A0E0EFB0EBBC34506DA03EBD3734FEA0A
:10F7C0006303ACEB030C05E009DD03EBD3734FEAF5
:10F7D00063039C4404F10104E4B2052CD7D3C5E9CA
:10F7E00000CABDE8F08F07DD02EBD27252109444DC
:10F7F000641CE4B2052CADD3C5E900ACBDE8F08FC4
:10F8000086070020880700208A070020287A002029
:10F8100098070020B0070020B807002058080020F3
:10F82000147A00201E7A0020A80700202DE9F04F4E
:10F830000D4687B0014600200490059091F85900CC
:10F8400091F8FC20401EC4B228886E88FE49022A26
:10F850003CD031F8242001EB8407831A0FFA83FC93
:10F860007B880CFB0CF8F11A09B201FB0188B8F592
:10F87000C86FDCBF104619464ADD4FF028094FF427
:10F88000C8686FF0270ABCF1000FB4BFCCF1000BC1
:10F89000E3460029B4BFC1F1000E8E46F3451CDDDE
:10F8A000BCF1280FC8BF494604DC1CF1280FB4BFC7
:10F8B000514661460DF1100C4FF00109CDE90019D8
:10F8C000CDE902C83146FFF72AFF19E021F82400EC
:10F8D00001EB84014E8031461AE02829C8BF494611
:10F8E00003DC11F1280FB8BF51460DF1100C4FF099
:10F8F0000209CDE90019CDE902C83146FFF70FFF33
:10F90000D148049920F8241005987880DDE9040195
:10F91000A880E98007B0BDE8F08F2DE9F04F8DB0E9
:10F92000044600F01FFF049000F01FFF089003F052
:10F9300077FC814603F056FC079094F8596003F079
:10F9400051FC827A94F859100127002A04BF427DA5
:10F95000002A06D1027D012A1CBF90F85D22012AEF
:10F9600001D180F85A7200258DF819508DF8187061
:10F970008DF8175090F86322DFF8D082022A06D063
:10F9800090F85A020028D8F8000013D029E0D8F8DF
:10F990000000826DC2F3C0438DF81430C2F34042C0
:10F9A0008DF81520806D2246C0F380408DF816003A
:10F9B000032026E090F85820C2F3C0038DF81430DD
:10F9C000C2F340028DF8152090F85820C2F380024F
:10F9D0008DF816202279022A1EBF032A2246002013
:10F9E0000FD1826DC2F3C0438DF81430C2F3404290
:10F9F0008DF81520806D2246C0F380408DF81600EA
:10FA00000220FFF795F89148D0F8008098F8580048
:10FA100010F0010F00F00F8294F85B10B4F8B400FE
:10FA2000ADF80800B4F8B63009EB0121ADF80A30A2
:10FA30000B9194F8591094F8FCC0854A01EB4101F0
:10FA4000BCF1020F02EB810155D031F80AAC21F86C
:10FA500008AC31F80C2C21F80A2C21F80C0C31F8E8
:10FA6000049C21F8029C31F806CC21F804CC21F842
:10FA7000063C81B261F30F0062F31F40914284BFE4
:10FA800062F30F0061F31F40010C514588BF6AF318
:10FA90001F4082B2010C8A4284BF61F30F0062F3FF
:10FAA0001F40000C63F30F016CF31F41634584BFDB
:10FAB0006CF30F0163F31F410A0C4A4588BF69F3D9
:10FAC0001F418AB20B0C9A4284BF63F30F0162F3A9
:10FAD0001F410B0C9DF81410ADF80C00ADF80E3062
:10FAE000012904BFADF80800ADF80A3094F8FC0015
:10FAF00002280DD083E021F8080C21F80A0C21F827
:10FB00000C0C21F8023C21F8043C21F8063CE1E70A
:10FB100050484FF0000C304400F8015C4E4801950D
:10FB2000304400F8017C4D4800EB46100A904C48E8
:10FB300000EB461009904B4800EB461000900999E5
:10FB4000002001EB0C1E009901EB0C1B0A9901EB44
:10FB50000C1900210EEBC0020BEBC00309EBC00730
:10FB600002EB810A4AF8205C03EB810A4AF8205C28
:10FB700007EB810A491C09B24AF8205C0229EFDB35
:10FB8000401C00B20228E4DB0CF101000FFA80FCFB
:10FB9000BCF1020FD3DB019A0998DFF8CCE000EB4F
:10FBA000021ADDE90002002100EB02192F4A0020B1
:10FBB00002EBC1070AEBC10C09EBC1050EEBC10357
:10FBC000814207D1B8F8622043F82020B8F86020BD
:10FBD00047F8202053F820200CEB800B02EB820228
:10FBE00052004BF8202C05EB800B401C00B24BF868
:10FBF000202C0228E4DB481C01B20229D6DBBDF828
:10FC0000082000212046FFF7F5F90546BDF80A2037
:10FC100001212046FFF7EEF9002DB8BF002500288E
:10FC2000B8BF0020094F3A68B2F910104B1EAB4222
:10FC3000B8BF1D46B2F912104A1E8242B8BF104624
:10FC4000AAB2ADF80C2013E0E08000205808002094
:10FC5000B07E00209C7E0020A67E00205C7D0020DF
:10FC6000DC7A00201C7C0020C0070020D007002088
:10FC700083B2FF48ADF80E3081190A30304411F8D4
:10FC800001CC10F8015C01F8015C00F801CC9DF892
:10FC90001600012804BFADF80820ADF80A30204650
:10FCA0000B9900F08FFA94F858100B98022918BF9E
:10FCB000002529D0C4F8C850B4F8B410B0F8B42066
:10FCC000DFF8B083891AC4F8CC10B4F8B610B0F8D5
:10FCD000B60008F10A09081AC4F8D000022E9CBF29
:10FCE0009DF81700012823D008EB0601022001F837
:10FCF000010C09EB060101F8010C08EB06010020DC
:10FD000011F8011CB1BB36E0B4F8B430B0F8B4104F
:10FD10005A1A48BFCA1AB4F8B630B0F8B6C0B3EB36
:10FD20000C0148BFACEB0301524301FB0125C1E7C5
:10FD30002A4602A92046FFF758FB079890F85A0276
:10FD40000028DAD1CC48304410F8010C012808D042
:10FD50000028D2D1C948304410F8010C401C1428A6
:10FD6000CBD9BDF80C00ADF80800BDF80E00ADF819
:10FD70000A00C2E704E009EB060111F8011C01B119
:10FD80000120009007982B4602A9427C2046FEF7EE
:10FD900094FF9DF81500012840D0BDF80800A4F894
:10FDA000B800BDF80A00A4F8BA00BDF80800049A2B
:10FDB000BDF80A109042B8BF1046089A9142B8BFE9
:10FDC00011463A68049BB2F910C0ACEB0303A3F1EF
:10FDD000010C8445B8BF6046B2F91230089A9A1AED
:10FDE000531E8B42B8BF194682B2A4F8B82088B21D
:10FDF000A4F8BA000B99B1F8B810511AC4F8D81089
:10FE00000B9AB2F8BA20801A4943C4F8DC0000FB10
:10FE10000010C4F8D4000DB0BDE8F08FBDF80C00A0
:10FE2000ADF80800BDF80E10ADF80A10A4F8B8003F
:10FE3000BDF80E00B7E7B4F8B400A4F8B800B4F801
:10FE4000B600A4F8BA000DB0BDE8F08F8C4A30B40B
:10FE5000146894F8542012F0040F1ABF012323EA07
:10FE6000020502F00105B0F900C0B1F900301DB182
:10FE7000E58AEB1A5B1E1BB212F0020F06D0A48AB1
:10FE8000A4EB0C0CACF1010C0FFA8CFC12F0040F7B
:10FE900019BF0380A1F800C0A0F800C00B8030BCDF
:10FEA0007047774A30B41268B2F8983013F0FF0206
:10FEB0004FEA132308BF6422002B08BF6423048881
:10FEC000B1F800C062436F4CA4FB02525209028099
:10FED0000CFB03F0A4FB00204009088030BC7047F5
:10FEE0002DE9F0470446664882B00068B0F818A0D3
:10FEF000B0F81A90858AC68A078AB0F81280002066
:10FF0000ADF80000ADF8040003F06CF9B4F8B810D7
:10FF1000B4F8BA0001FB0AF292FBF7F2A4F8BC2095
:10FF200000FB09F292FBF8F26943704391FBF7F191
:10FF300090FBF8F0A4F8BE20ADF80010ADF8040076
:10FF400001A96846FFF782FFBDF90000711E8842D3
:10FF5000A8BF084600B2BDF904106A1EADF8000043
:10FF60009142A8BF114609B2ADF804100028D8BFCD
:10FF70000020ADF800000029D8BF0021ADF8041022
:10FF8000A4F8C000A4F8C21002B0BDE8F0873B4A54
:10FF90000021024402F8011C3B4A024402F8011C01
:10FFA000354A024402F8011C384A02EB800242F84A
:10FFB000041C374A02EB800242F8041C354A02EB6B
:10FFC000800242F8041C344A02EB800242F8041C0E
:10FFD000324A02EB400020F8021C418070472DE9B4
:10FFE000F0439BB01F468C46DDE923350021DDF848
:10FFF00088800646259C12911391149115911691B3
:020000021000EC
:100000001791189138461991B8F1000F14BFA3F158
:100010000A07471C052F40F2D1804FFA80F909F1F9
:10002000010189B28B4298BF0021B8F1000F7DD049
:100030003CF81180CDF8488032F811101391A9EBEB
:10004000530109B2002901DA194409B23CF81180C0
:10005000CDF8508032F811101591F9B2CDE9003188
:100060000DF110081346CDF808806246014617E0EE
:100070009C7E0020147A00208A0700208807002038
:10008000580800201F85EB5186070020B00700208C
:10009000B807002098070020A0070020A80700202C
:1000A000304600F0F0F916902A880392FE49208825
:1000B000069009684B8AB1F81AC0C3EB0313B3FB6F
:1000C000FCF317934B8AB1F81AC0C3EB0313B3FBCD
:1000D000FCF318934B8A498B03EB83035B00B3FB60
:1000E000F1F11991DDF85CC0002E4FF0000139D01C
:1000F000129B059A5A43049B03EB2242139BD31A8B
:1001000044BF139B9B1A634554D2149B059ADDF898
:1001100060C05A43049B03EB2242159BD31A44BF91
:10012000159B9B1A634545D2199B00E00AE0169A7D
:10013000821A44BF169A121A9A423BD2169880B27B
:10014000069036E0BCF80080CDF84880B2F8008018
:1001500021F00101CDF84C803CF80180CDF85080B1
:10016000515A79E7139B05985843049B03EB2040B1
:10017000129BC31A44BF129B1B1A63451AD2159BCC
:100180000598DDF860C05843049B03EB2040149BA6
:10019000C31A44BF149B1B1A63450BD21698199BB4
:1001A000101A44BF1698801A984203D2169880B24B
:1001B0000390012103982880069820801BB00846F0
:1001C000BDE8F0832DE9FF4F8BB09B468A4605467C
:1001D00003F008F890F85A22BAB114204FF0020840
:1001E0000290287995F85940AF49022818BF032892
:1001F00015D0012A1CBFAD4886681AD095F8FC00BE
:10020000AB4A0027022840D11DE03C210291407CEE
:1002100002282CBF4FF003084FF00F08E1E70868F1
:100220006423428A408B5A43B2FBF0F000FB00F695
:10023000E4E70868428A408BC2EB0212B2FBF0F09E
:1002400000FB00F6DAE7101900F8017C9948204419
:1002500000F8017C47729848204400F8017C4772FE
:10026000964800EB440020F8027C4782944885F8C9
:10027000E170204400F8017C47729248204400F865
:10028000017C9148204400F8017C904802EB04096D
:1002900000EB041319F8010CDDF834C003EB400245
:1002A00022F810CCA2F890B095F8FC20032A46D191
:1002B000C01D00F007008DF8207003EB40008DF8A2
:1002C000247030F8102C0D9BB0F890009A1AABEB0C
:1002D00000030868018B5143028A91FBF2F10791F8
:1002E000418B408A594391FBF0FB08AB2246012029
:1002F0000799FEF7C4FF059009AB22465946022034
:10030000FEF7BDFF03909DF820100798CDE900018E
:1003100021460120029B059AFEF7E6FF9DF8240086
:10032000DDE90232CDE900B021460220FEF7DCFF14
:1003300061480599204400F8011C0399417219F89D
:10034000010C0122401CC0B209F8010C082808D396
:1003500009F8017C9AF8E100002808BF8AF8E1203A
:1003600002E09AF8E10018B195F85800022809D087
:1003700085F8E1705248204400F8017C47720FB0C4
:10038000BDE8F08F514B0021084603EB041C0CEB39
:100390004003401C33F8103C80B219440828F6D3BF
:1003A0004FEAD10A00210846E9460CEB400333F836
:1003B000103CA3EB0A035B4349F82030401C80B299
:1003C00019440828F1D34FEAD109414B00210846CE
:1003D00003EB041C0CEB4003401C33F8103C80B2D0
:1003E00019440828F6D34FEAD10A00210846EB4603
:1003F0000CEB400333F8103CA3EB0A035B434BF8D0
:100400002030401C80B219440828F1D3C8080323C7
:100410004E4528BF864208D32648204410F8011CC8
:1004200008299CBF407A082811D9264885F8E13070
:10043000204400F8017C2448204400F8012C95F861
:10044000E100032804BF0FB0BDE8F08F92E71D481C
:10045000204410F8011CC8293CBF491C00F8011CAD
:100460001949214411F8011C012908D110F8010C87
:1004700040459EBF85F8E1300FB0BDE8F08F022007
:1004800085F8E10076E72DE9F04FAFB00FFA81F97A
:10049000DDE9388C0124CA466946002860D032F86C
:1004A0001A002B9016E00000580800208407002056
:1004B0006880002086800020728000209A800020C2
:1004C000C2800020D6800020C87A0020287F00202B
:1004D000C87F0020BCF1010011D441F8204001EB9D
:1004E000800632F81A503565AAF101050FFA85FA2F
:1004F000BAF1000FB8BFA8F1010A401EEDD50024E3
:1005000025464846BCF101020FD433F8107051F86B
:100510002260401E7E43341900B245EBE675002888
:10052000B8BFA8F10100521EEFD500263746BCF136
:1005300001005DD401EB800233F819A0126DA9F11E
:10054000010902FB0AF296190FFA89F947EBE277E3
:10055000B9F1000FB8BFA8F10109401EEAD547E084
:1005600033F81A002B90BCF1010011D441F820405F
:1005700001EB800633F81A503565AAF101050FFA30
:1005800085FABAF1000FB8BFA8F1010A401EEDD5F7
:10059000002425464846BCF101030FD432F8107000
:1005A00051F82360401E7E43341900B245EBE675D6
:1005B0000028B8BFA8F101005B1EEFD50026374622
:1005C000BCF1010014D401EB800332F819A01B6DBB
:1005D000A9F1010903FB0AF39E190FFA89F947EB08
:1005E000E377B9F1000FB8BFA8F10109401EEAD5C1
:1005F0004FF000084046CDF8A080BCF1000F0CDDA4
:1006000051F82020289B524312EB080843EBE2727A
:1006100000F1010028928445F2DC00229646104643
:100620002992BCF1000F11DD01EB800351F820206D
:100630001B6DDDF8A4905A434FEAE27A12EB0E0EDE
:100640004AEB0903401C29938445EDDC4FF0000977
:10065000CA464846BCF1000F0DDD01EB800251F89F
:100660002030126D00F101005A4312EB09094AEBE8
:10067000E27A8445F1DC002003460246BCF1000F1B
:100680000CDD694601EB8001096D49434FEAE17BCE
:100690008A184BEB0303401C8445F2DC1046A8FB90
:1006A000002C2899CDE92C0301FB00C0AEFB09CB3F
:1006B00029992E9108FB030301FB09B10EFB0A10D7
:1006C000B2EB0C0163EB0000CDE92901084333D004
:1006D000DDE92C02A0FB0413AEFB06CB02FB0432C7
:1006E0002E9B00FB052203FB06B30EFB0733B1EB89
:1006F0000C0062EB0301DDE9293209F01CF83A999C
:100700000860A8FB0602289901FB0621A9FB042327
:100710000AFB043308FB071109FB0533801A61EB60
:1007200003010904DDE9293241EA1041000409F01E
:1007300002F83A99486004E03A99002008603A9932
:1007400048603A98D0E900122B98504311EB2040B2
:1007500048BF00202FB0BDE8F08F0000FE48704772
:10076000FE487047FE4800787047FD484078704763
:100770000346002002460029D8BF704753F822C024
:10078000521C60449142F9DC70472DE9F05F0E463F
:10079000054602F053FD044602F04CFD310291FB88
:1007A000F0FC290291FBF4F3DFF8B4E3EB4D5E12A9
:1007B000BEF80490BEF8068000214FEA6C2705F5CC
:1007C000907A002C0BDD01FB03F206EB222245F8A8
:1007D00021204AF82120491C09B28C42F3DCDE4E6C
:1007E000002106F5907B00280BDD01FB0CF207EBE6
:1007F000222246F821204BF82120491C09B28842C8
:10080000F3DC0CFB09FC03FB08F34FEA6C315A13D1
:100810005F13CEF80C102B684FEA6C3C9B1A2B60D0
:1008200005EB840353F8045C154443F8045C336817
:100830005B1A336006EB800353F8045C0D4443F805
:10084000045C9EF80330002BDAF8003017D09B1AB6
:10085000CAF800300AEB84030BEB800053F804CC99
:10086000624443F8042CDBF80020521ACBF8002035
:1008700050F8042C114440F8041CBDE8F09F9A1A6B
:10088000CAF800200AEB84020BEB800052F8043C0B
:100890003B4442F8043CDBF80020511ACBF800102E
:1008A00050F8041C6144E6E7AE4930B40968AC4A2C
:1008B0004FF0040C4C8A098A0723A2F804C0D380A5
:1008C0004020108170205081204630BC5DE7A44854
:1008D000C078012818BF002070475FEA000C30B4D0
:1008E000A0489F4B0268508A118A14D092F854C0D5
:1008F000528B4FEADC0404FB00FCBCFBF2F21A70E2
:100900005A7004229A800722DA8040221A817022CB
:100910005A8130BC39E700221A705A70F1E79148C9
:10092000026892F85430508AB2F81AC0DB08434388
:10093000B3FBFCF3118A8A4A13705370042393802B
:100940000723D3804023138170235381C0EB00130E
:10095000B3FBFCF393700023D37016E72DE9F04F3F
:10096000B3B00D460446CC227F49684608F04CFFE0
:100970007C48B5F902200068012A90F805C090F87B
:100980000480478A068A687800FB0CF109B2D8BF58
:1009900001222B78DFF8D4E1EB4683B1ACF10109F9
:1009A0004B45194417D104EB410131F9021C0129CF
:1009B000D8BF0121C902494291FBF2F140E004EBAA
:1009C0004101B1F902100129D8BF0121C90291FBEF
:1009D000F2F109B235E004EB410939F9021C0129B1
:1009E000D8BF0121B9F90290B9F1010FD8BF4FF07A
:1009F00001094FF0640A01FB0AF109FB0AF901EB56
:100A0000620109EB620991FBF2F199FBF2F93BF902
:100A100011103BF91990494508BF002111D001EB95
:100A2000090A1AF5004FB8BFF24604DBBAF5004FC9
:100A3000A8BF47F6FF7AA1EB0901C90291FBFAF1C1
:100A400009B2A0B1A8F101094845A0F1010909FBCB
:100A50000CF90FFA89F9994415D134F91940012C90
:100A6000D8BF0124E402644294FBF2F246E003EBB7
:100A70000C0934F91940012CD8BF0124E40294FB7D
:100A8000F2F212B23BE034F91990B9F1010FD8BF7C
:100A90004FF0010900F1010A0AFB0CFA0FFA8AFA79
:100AA0009A4434F91AA0BAF1010FD8BF4FF0010AE5
:100AB000642409FB04F404EB620494FBF2F44FF0A9
:100AC00064090AFB09F909EB620999FBF2F23BF9A7
:100AD00014403BF91220944208BF00220FD004EBCF
:100AE000020919F5004F05DBB9F5004FB4BFCE463A
:100AF00047F6FF7EA21AD20292FBFEF212B21B044C
:100B0000000403EB011100EB021201F5004002F5B5
:100B1000004190FBFCF091FBF8F1704301FB07F101
:100B200000144FEA21414CBF00220246B242C8BF26
:100B3000304602DC0028B8BF00200029B4BF0022E4
:100B40000A46BA42C8BF394602DC0029B8BF0021B4
:100B5000A5F8B4000CE00000088100209881002076
:100B6000E00700205808002018B311000080FFFFA4
:100B7000A5F8B61033B0BDE8F08F531A48BF8B1AF2
:100B800064225343421A48BF0A1A93FBF2F070479B
:100B900070B4FA4A8DB004AEB2E838108DE838105F
:100BA000B2E8381086E8381092E81C1008AD85E8E5
:100BB0001C10002201290CBF022100216E465DF8A5
:100BC0002130EF4C0DF1200C04AD83421CDB55F8B5
:100BD00021205CF821109042D8BF421A37DDB1EBDA
:100BE000020C48BFA2EB010C64210CFB01FC991A1A
:100BF00048BFD11A9CFBF1F1181A484384FB00103E
:100C00004111A1EBE07222E006EB81035B689842A0
:100C10001DDB05EB81020CEB8101526849688242C1
:100C2000D8BF0A1A13DDB1EB020C48BFA2EB010CCE
:100C300064210CFB01FC991A48BFD11A9CFBF1F10D
:100C4000C01A484384FB00104111A1EBE0720DB0C3
:100C5000104670BC70474FF0000C00686246634657
:100C6000B0F5107FC8BF7047B0F5C87F13DCD1F86E
:100C700000C00823ACF53462002ACCBF01224FF03B
:100C8000FF32C0F5C870ACF5346C00FB0CF04FF4CB
:100C9000346C90FBFCFC086803FB020060440860B5
:100CA000704770472DE9FF4FADF5177D0E4607469B
:100CB00014469021684608F003FE902124A808F00D
:100CC000FFFD902148A808F0FBFD90216CA808F0DA
:100CD000F7FD02F087FA02F097FA02F0B3FA959066
:100CE00002F0A8FA054602F0A9FA9090A5484FF044
:100CF00064090068418A9191008A92906278207814
:100D0000A149949102FB050090399391305C00F069
:100D10003F0A207B969094F80DC094F80FB0A17B09
:100D2000DC4533D8969B0CFB05F01FFA80F88B420C
:100D300026D808EB0302B4F902E037F91200F145B6
:100D400007DAB4F83AE0A0EB0E0000B20028B8BF12
:100D50000020B25C02F03F0252450DD1959A9042BC
:100D60000ADB5DF823E024AA86444DF823E052F81C
:100D70002CE0704442F82C00581C83B28B42D8D926
:100D80000CF101001FFA80FCDC45CBD900216A463A
:100D90000846002D7EDD52F82030401C1944A84240
:100DA000F9DB002976DD0021909A24AB0846002A61
:100DB00070DD53F820C0401C61448242F9DC0029F8
:100DC00068DD69462846939A00F0DCF9064624A9B6
:100DD000949A909800F0D6F96C4F0446F878002861
:100DE00048D1B046939EA946CDF854D206EB89056A
:100DF000002155F804BC4046D6F800A0FFF7C8FE15
:100E000000280DDB31683246091A316055F8041CA0
:100E1000084445F8040C4846959900F0B3F980461B
:100E2000C6F800A045F804BC4646A046DDF840924E
:100E300024A8949C909004EB8905012155F804ACFA
:100E40004046D4F800B0FFF7A3FE00280DDB216870
:100E50002246091A216055F8041C084445F8040C80
:100E60004846909900F08EF98046C4F800B045F8E5
:100E700004AC44463878F0B1002210461146B6F56D
:100E8000107F1BDCB6F5C87F12DC0821A4F53460A6
:100E9000002800E022E0CCBF01204FF0FF30C6F573
:100EA000C872A4F534635A434FF4346392FBF3F2EF
:100EB00001FB00408418002EB8BF0026002CB8BFEC
:100EC00000249298401E8642C4BF9298461E919874
:100ED000401E8442C4BF9198441E01E0002634465F
:100EE0009A980680A49804800DF51B7DBDE8F08FCC
:100EF00010B4274992B0B1E81C108DE81C10B1E87D
:100F00001C10CDE90423CDE9064C51F8042B0892BE
:100F1000B1E81C10CDE90923CDE90B4CB1E81C1058
:100F2000CDE90D23CDE90F4C096811910479B0F892
:100F3000B42041786B460DF1240C012C05D0B0F99A
:100F40003640B4F5E17F25DD07E0B0F93440B4F573
:100F50002F7F02DC0478142C07D833F811101144C9
:100F6000A0F8B41012B010BC70473CF81110114436
:100F7000A0F8B41012B010BC70470000E4B3110028
:100F80001F85EB5158080020B8820020E0070020A0
:100F900014B411000478142CE7D8DEE72DE9F74FDC
:100FA00091488B4684B00068144690F8561090F82B
:100FB000550001F07F0A00F07F08CF09C60902F052
:100FC00011F902F021F902F02BF994F85B1000EB13
:100FD000012502F033F9814602A8009001AB2246B8
:100FE00059460498FFF75EFE0AEB8A00C1B208EB8F
:100FF0008800C2B2002F1CBF4842C1B2002E1CBFE5
:101000005042C2B2BDF804000844A4F8B400BDF8D0
:1010100008001044A4F8B60095F8E400012804BFC5
:10102000287800280AD1687800281CBFA9F101019E
:10103000884203DA94F8E500012807D095F8F80013
:1010400001280BD1E088E988884207D3B5F8B400BD
:10105000A4F8B400B5F8B600A4F8B60094F8FB0004
:1010600001210222022813D003281CBF07B0BDE8CB
:10107000F08F84F8FD1095F8FD00012820D002289B
:1010800012BF0328032084F8FD0007B0BDE8F08FED
:1010900084F8FD1094F8E40000281CBF07B0BDE8F8
:1010A000F08F94F8F20000281FBF94F8F500002894
:1010B00007B0BDE8F08F84F8FD2007B0BDE8F08FE1
:1010C00094F8F200002804BF94F8E4000028F2D05D
:1010D00007B0BDE8F08F10B5044602F083F802F0C7
:1010E0009FF8014694F85B00022201EB00210120E9
:1010F00084F8FC0094F8FD0002280FD0032818BFE4
:1011000010BD91F8FC00022811BF0328032084F8C9
:10111000FC0010BD94F8E60028B110BD94F8E6007C
:10112000002818BF10BD84F8FC2010BD10B514466F
:10113000FFF734FF02F056F802F072F894F85B10F3
:10114000022200EB0121012084F8FC0094F8FD004C
:1011500002280FD0032818BF10BD91F8FC00022808
:1011600011BF0328032084F8FC0010BD94F8E600AA
:1011700028B110BD94F8E600002818BF10BD84F80F
:10118000FC2010BD70B5A4B00D4604461646902153
:10119000684608F095FB0023002CC8BF684609DDAF
:1011A00055F8231056F82320514340F823105B1CB8
:1011B0009C42F5DC002368461A46002C05DD50F8F9
:1011C0002210521C0B449442F9DC4FF0000C624692
:1011D000002C05DD55F82200521C84449442F9DCB1
:1011E00093FBFCF024B070BD5808002070B5144685
:1011F0000D46064602F01EF88446D5E90720A96987
:10120000002904BF002319460AD002EB8202920093
:101210004900B2FBF1F300EB80008000B0FBF1F17C
:101220002380FF486180A0FB0332A0FB0110D2089D
:10123000C00800FB0C2036F81000A08070BDF0B490
:10124000DDE905C4049D002D1CBF002081F8390094
:1012500002D0F0BC002070470D6840F8045B8D8818
:1012600020F8085BD1F8065040F80C5B156840F890
:10127000125C928820F80E2CE4CBE4C0E4CBE4C0EE
:10128000E4CBE4C06CCB6CC0D1F80A2040F8482C09
:10129000D1F80E2040F8442C8A6940F83C2C8A8A08
:1012A00020F8402C91F8262000F8092C8A6A40F892
:1012B000042C91F8332000F8082C91F8342020F801
:1012C0001E2C91F8382080F8922091F83A2080F86E
:1012D0009320012280F8912080F8944091F83210F8
:1012E00080F89F109CF80000401CC0B28CF80000F1
:1012F0000A2828BF0120ACD3F0BC70470028DCBF0F
:10130000002070474FF480714FEA002C00200B1230
:101310009CFBF3F30A46991801EBD1714910531A5B
:1013200048BF8B1A802B02DB401C6428EFD30812C5
:1013300070472DE9FF4F89B017468946002401F018
:1013400051FF00F1170601F075FF054601F076FF29
:101350000590B7F900000790B7F90200069099F8D8
:101360000600009099F80800019099F8073099F864
:101370000900039099F8000099F80110A44601FBB8
:1013800005003221305C0291B9F902106746E0464F
:1013900000F03F00C829C4BF5021029103998B423D
:1013A0003BDCDDE90012914232DC03FB05F20492E2
:1013B000069A03EB8309C2EB490909FB09FB03FB0E
:1013C000051A099A32F91A20DDF808A052451ADDEB
:1013D000DDF810A006EB010E1AF80EA00AF03F0A85
:1013E000824510D1DDF81CA001EB810ECAEB4E0A3C
:1013F0000AFB0AFE09FB0AFA0EFB02CC0BFB027782
:101400000AFB02881444491C019A09B29142D6DDB4
:10141000591C0BB203998B42C3DDDFF8089289FB9C
:101420000C214A11A2EBE17289FB07314B11A3EBAE
:10143000E17389FB08C14FEA611CACEBE17C54B15C
:1014400011021A024FEA0C2391FBF4F192FBF4F221
:1014500093FBF4F302E000210A460B4601FB02FC79
:1014600003FB13C311444C421F12B90004FB04F2E6
:10147000C1EB222109124A00002AD8BF00211ADD3F
:101480004FEA02284FF4807100224FEA212C98FB8A
:10149000FCFC0B460CEB030101EBD1714910B3EBE3
:1014A000010C48BFA1EB030CBCF1800F02DB521C06
:1014B000642AEAD30912090201EBD1710C9BD4EB27
:1014C000610204EB6101C1F100011F614CBFC2F177
:1014D000000C94460C9B0029C3F808C0B4BF4C42D2
:1014E0000C460C9BDC600CEB8C035B0089FB0373EC
:1014F000DF10A7EBE373FF2BC8BFFF234FEA6C1C81
:101500006411BCF1FF0F88BF4FF0FF0CFF2C88BFA8
:10151000FF24BCF1000F12BF002C4FF0010C6446F9
:10152000002B08BF0123DB00DFF8FC8088FB03737E
:101530005F10A7EBE373377807F03F07874207D0C8
:10154000059F7F1E6F43F75D07F03F07874204D179
:10155000980088FB0030431011E005EBC507F75DEC
:1015600007F03F07874205D016F8355005F03F05D4
:10157000854206D12B20584389FB00300311A3EB91
:10158000E0730C9880F834300C9880F832C00C98D6
:1015900080F8334090104FEAA20048BF40428B10C1
:1015A0004FEAA10348BF5B42C01A0FD588104FEA2B
:1015B000A10048BF404291104FEAA20100D5494224
:1015C000401A0C9948610DB0BDE8F08F90104FEAB9
:1015D000A20048BF40428A104FEAA101F0D5EEE7D1
:1015E0002DE9FF4F07461148164693B0D0E9031284
:1015F000CDE90412D0E90512209CCDE90612D0E90C
:101600000712CDE90812D0E90910CDE90A1001F05E
:10161000E9FD17300F9001F00DFE039008E0000087
:10162000CDCCCCCC1F85EB51676666665CB41100EF
:1016300001F004FE024614980021521EB0F9020087
:101640000090149889468A4600781190149888462C
:101650000D46407801911090009802910302CDE967
:101660000D23039A8C46521E0C92002224F811205E
:1016700004AA32F81C30119A1A4413B206AA32F89E
:101680001CB0109A5A440FFA82FB039ABBF1000F68
:101690000BFB023212B2A4BFDDF834E0DE453BDBC7
:1016A000002BA4BFDDF830B09B4535DB37F9123095
:1016B00024F81130002BDCBF012324F8113034F959
:1016C00011300A2B0DDDDDF838B0DDF808E0BBFB8A
:1016D000F3FBF34409F1010909F0FF09CDF808B063
:1016E00001E0002B08DDDDF838B008F10108BBFB94
:1016F000F3FBDA4408F0FF08DDF804B05B45C8BF2F
:101700000193DDF83CB01BF802B0BBF1000F1CBF29
:101710006D1CEDB2184400B2491C0CF1010202F03C
:10172000FF0CC9B2BCF1040F9FD30023002224F8A0
:10173000112008AA32F813C0119A62440DF1280C46
:1017400012B23CF813B0DDF840C0DC440FFA8CFC58
:10175000DDF80CB0BCF1000F0CFB0B2B0FFA8BFB70
:10176000A4BFDDF834E0E64515DB002AA4BFDDF8B0
:1017700030C094450FDB37F91B2024F81120002AD4
:10178000DCBF012224F811200F9A12F80B20002A46
:101790001CBF6A1CD5B2491C5A1CD3B2C9B2042B57
:1017A000C4D31699B9F1000F0D70DDE90012114490
:1017B0000AB21ABF0299B1FBF9F30023B8F1000F86
:1017C00014BFBAFBF8F10021002A1ABF4FEA002C1F
:1017D000BCFBF2FC4FF0000C4FEA0C2C002914BFAC
:1017E000BCFBF1FC4FF0000CDB09C909F283C6E930
:1017F0000931B083C6F82CC01499898A90FBF1F0A6
:10180000308617B0BDE8F08FF0B40546B0F902405D
:101810000020D22C29DAB2F90060002EC4BFB2F940
:1018200002C0BCF1000F04DDB444A4440FFA8CFCE8
:1018300012E0B2F904C0BCF1000FC1BFB2F90670EA
:10184000002FBC44A44405DC5788A4443E44B4445F
:10185000D688B4440FFA8CFCBCF5AF7F05DAB5F836
:1018600024C0BCF1060F38BF01204FF0000C32F845
:101870001C600CF1010C34440FFA8CFC24B2BCF156
:10188000040FF4DB30B15A1C94FBF2F292B20A86D8
:10189000F0BC7047AA8A002A1CBF94FBF2F292B2F5
:1018A000F5E72DE9F04F0446FF480F4683B0D0E935
:1018B0000112CDE900120068029001F0BBFC054660
:1018C00001F0BCFC8146B7F90200397997F800A015
:1018D0007E784FEA6008012935D1502833DD4FF07A
:1018E000000CEE460DF1080B3EF81C00504402B20D
:1018F000002AA8BF95421BDD06FB052087B2002108
:101900003BF81100304400B20028A8BF81450BDD30
:1019100000FB052034F9173080B24345A4BF34F9E9
:101920001000B3EB400F0EDB481CC1B20229E7D315
:101930000CF1010000F0FF0CBCF1030FD4D303B095
:101940000120BDE8F08F03B00020BDE8F08F70B536
:1019500086B015460C46064601F044FC02A90091EB
:1019600001AB2A4621463046FFF73AFE2146304673
:10197000FFF797FF002804BF06B070BD94F832004F
:10198000002804BF022084F8320006B070BD2DE9A3
:10199000F04F89B01F4615460E46129C01F022FCFE
:1019A000034606EB851C0022DD7B10461146002D08
:1019B0000BD906EB811393F83930012B04BF521C6D
:1019C000D2B2491CC9B28D42F3D8B849096891F81E
:1019D000581011F0800F04BF09B0BDE8F08FBCF8BB
:1019E00014102388994213D997F83280B4F80490E0
:1019F000C8450DD9BCF82690B4F802A0D14584BFE3
:101A0000C844B8F1580F03D909B00120BDE8F08FE0
:101A1000022A1CBF09B0BDE8F08FA3F11E0291425B
:101A2000DCBF09B0BDE8F08F97F83210A288263AE3
:101A30009142DCBF09B0BDE8F08FBCF82610628887
:101A40001E3A9142DCBF09B0BDE8F08F4FF0010AA9
:101A50000021009101910291039104910591069159
:101A60000B46E9460791002D88BF01242DD906EBCE
:101A7000831292F839C0BCF1010F1FD1002912BFA7
:101A80005778012192F8018092F811C092F80FB0B6
:101A9000ACEB0B0C0CEB4C0B92F810C0927B0BEBED
:101AA000DB7BACEB020EBEEB6B0F2ADD944505D35E
:101AB00009F80240521CD2B29445F9D25A1CD3B252
:101AC0009D42D4D8BAF1000F1BD0B8EB070148BF34
:101AD000A7EB08010329D9BF0022114609B0BDE8D0
:101AE000F08F19F80130012B04BF521CD2B2491CEF
:101AF000C9B22029F5D3152A9CBF09B0BDE8F08FE3
:101B000082E709B00020BDE8F08F2DE9F74F82464B
:101B100000209EB093460446039018908146199089
:101B200001F06AFB064601F05DFB074601F06CFB25
:101B300014903220ADF860002320ADF862002D2013
:101B40004FF000088DF85440ADF864004546BBF1F5
:101B5000000F0ADD1F9800EB851494F83900012866
:101B60001DD0681C05B25D45F4DBA7F8048014980D
:101B70004F4B407C18B19DF85410022901D200212E
:101B80001970022806D29DF85400022804BF187864
:101B900000287DD09DF8540021B0BDE8F08F0020D2
:101BA0000490079008900590069009900C900D9075
:101BB0000A900B900E90119012900F90109013902D
:101BC0001690179004A8019001F00CFB1AA8009041
:101BD00002AB21465046019AFFF702FD21465046CE
:101BE000FFF75FFE30B194F83200002804BF0220F6
:101BF00084F8320001F01EFB0346D4E90601226A94
:101C0000002804BF002108460AD001EB81018900A9
